:020000040800F2
:1000000000060020B5050008212A0008A1290008E3
:10001000F9290008A1290008CD290008B705000822
:10002000B7050008B7050008B705000875380008CF
:10003000B7050008B7050008B7050008B7050008B0
:10004000B7050008B7050008B7050008B7050008A0
:10005000B7050008B7050008D9470008054800089B
:10006000314800085D48000889480008B7050008C5
:10007000B7050008B7050008B7050008B705000870
:10008000B7050008B7050008B705000819260008DD
:10009000B705000829260008B7050008B54800087C
:1000A000B7050008B7050008B7050008B705000840
:1000B000B7050008B7050008B7050008B705000830
:1000C000B7050008B7050008B7050008B705000820
:1000D000B7050008B7050008B7050008B705000810
:1000E00019490008B7050008B7050008B70500085A
:1000F000B7050008B7050008B7050008B7050008F0
:10010000B7050008B70500088D490008B7050008C5
:10011000B7050008B7050008B7050008B7050008CF
:10012000B7050008B7050008B7050008B7050008BF
:10013000B7050008B7050008B7050008B7050008AF
:10014000B7050008B7050008B7050008B70500089F
:10015000B7050008B7050008B7050008B70500088F
:10016000B7050008B7050008B7050008B70500087F
:10017000B7050008B7050008B7050008B70500086F
:10018000B7050008B7050008B7050008B70500085F
:10019000B7050008B7050008B7050008B70500084F
:1001A000B7050008B7050008B7050008B70500083F
:1001B000B7050008B7050008B7050008B70500082F
:1001C000B7050008B7050008B7050008B70500081F
:1001D000B7050008B7050008B7050008B70500080F
:1001E000B7050008B7050008B7050008B7050008FF
:1001F000B7050008B7050008B7050008B7050008EF
:10020000B7050008B7050008B7050008B7050008DE
:10021000B7050008B7050008B7050008B7050008CE
:10022000B7050008B7050008B7050008B7050008BE
:10023000B7050008B7050008B7050008B7050008AE
:10024000B7050008B7050008B7050008B70500089E
:10025000B7050008B7050008B7050008B70500088E
:10026000B7050008B7050008B7050008B70500087E
:10027000B7050008B7050008B7050008B70500086E
:10028000B7050008B7050008B7050008B70500085E
:10029000B7050008B7050008B7050008B70500084E
:1002A00069150008000000000000000000000000C8
:1002B00053B94AB9002908BF00281CBF4FF0FF31CD
:1002C0004FF0FF3000F074B9ADF1080C6DE904CEC9
:1002D00000F006F8DDF804E0DDE9022304B0704721
:1002E0002DE9F047089D04468E46002B4DD18A42E9
:1002F000944669D9B2FA82F252B101FA02F3C2F11C
:10030000200120FA01F10CFA02FC41EA030E9440AC
:100310004FEA1C48210CBEFBF8F61FFA8CF708FBCD
:1003200016E341EA034306FB07F199420AD91CEBA5
:10033000030306F1FF3080F01F81994240F21C81D7
:10034000023E63445B1AA4B2B3FBF8F008FB10331F
:1003500044EA034400FB07F7A7420AD91CEB040454
:1003600000F1FF3380F00A81A74240F20781644424
:10037000023840EA0640E41B00261DB1D4400023A9
:10038000C5E900433146BDE8F0878B4209D9002D0D
:1003900000F0EF800026C5E9000130463146BDE897
:1003A000F087B3FA83F6002E4AD18B4202D3824201
:1003B00000F2F980841A61EB030301209E46002DB0
:1003C000E0D0C5E9004EDDE702B9FFDEB2FA82F205
:1003D000002A40F09280A1EB0C014FEA1C471FFA63
:1003E0008CFE0126200CB1FBF7F307FB131140EA4A
:1003F00001410EFB03F0884208D91CEB010103F117
:10040000FF3802D2884200F2CB804346091AA4B2D8
:10041000B1FBF7F007FB101144EA01440EFB00FEAC
:10042000A64508D91CEB040400F1FF3102D2A64511
:1004300000F2BB800846A4EB0E0440EA03409CE7B0
:10044000C6F12007B34022FA07FC4CEA030C20FA5D
:1004500007F401FA06F31C43F9404FEA1C4900FA7D
:1004600006F3B1FBF9F8200C1FFA8CFE09FB1811FA
:1004700040EA014108FB0EF0884202FA06F20BD96D
:100480001CEB010108F1FF3A80F08880884240F2BD
:100490008580A8F102086144091AA4B2B1FBF9F001
:1004A00009FB101144EA014100FB0EFE8E4508D9FC
:1004B0001CEB010100F1FF346CD28E456AD9023881
:1004C000614440EA0840A0FB0294A1EB0E01A14266
:1004D000C846A64656D353D05DB1B3EB080261EBD4
:1004E0000E0101FA07F722FA06F3F1401F43C5E9AE
:1004F000007100263146BDE8F087C2F12003D840E4
:100500000CFA02FC21FA03F3914001434FEA1C4725
:100510001FFA8CFEB3FBF7F007FB10360B0C43EA17
:10052000064300FB0EF69E4204FA02F408D91CEBC7
:10053000030300F1FF382FD29E422DD902386344C5
:100540009B1B89B2B3FBF7F607FB163341EA034165
:1005500006FB0EF38B4208D91CEB010106F1FF38B4
:1005600016D28B4214D9023E6144C91A46EA0046AB
:1005700038E72E46284605E70646E3E61846F8E63D
:100580004B45A9D2B9EB020864EB0C0E0138A3E786
:100590004646EAE7204694E74046D1E7D0467BE767
:1005A000023B614432E7304609E76444023842E7DF
:1005B000704700BF02E000F000F8FEE772B63A486C
:1005C00080F30888394880F3098839484EF6085185
:1005D000CEF20001086040F20000CCF200004EF6BE
:1005E0003471CEF200010860BFF34F8FBFF36F8FFD
:1005F00040F20000C0F2F0004EF68851CEF2000149
:100600000860BFF34F8FBFF36F8F4FF00000E1EE34
:10061000100A4EF63C71CEF200010860062080F30D
:100620001488BFF36F8F03F06FFE03F011FE03F029
:100630009BFE4FF055301F491B4A91423CBF41F889
:10064000040BFAE71C49194A91423CBF41F8040BDC
:10065000FAE71A491A4A1B4B9A423EBF51F8040B5B
:1006600042F8040BF8E700201749184A91423CBFB2
:1006700041F8040BFAE703F029FE03F0EDFE144CF9
:10068000144DAC4203DA54F8041B8847F9E700F034
:1006900041F8114C114DAC4203DA54F8041B884761
:1006A000F9E703F011BE0000000600200022002040
:1006B000000000080000002000060020704E000826
:1006C000002200208022002080220020004B0020F9
:1006D000A0020008A4020008A4020008A402000866
:1006E0002DE9F04F2DED108AC1F80CD0D0F80CD0C8
:1006F000BDEC108ABDE8F08F002383F311882846F3
:10070000A047002003F068FAFEE703F0E1F900DFFC
:10071000FEE700002DE9F04100F09AFF30B12F4BC9
:1007200000220C211A725A729972DA7203F014FDC7
:10073000074603F083FD0546C0BB294B9F4235D0D9
:1007400001339F4235D027F0FF02264B9A4234D125
:10075000A84642F21074F8B200F0EEFA00F0F6FC8F
:1007600008B10024A04600F0EDFA064648B354BB99
:10077000464635B11C4B9F4203D0002403F056FD82
:100780002646002003F0F2FC0EB100F02FF800F036
:1007900001FD00F0FBFE02F04BF90546B4B900F094
:1007A0003FFD4FF47A7003F01DFAF7E7A8460024E6
:1007B000D4E704464FF00108D0E7804641F2883480
:1007C000CCE70446D5E74FF47A74D2E702F030F96B
:1007D000431BA342E3D900F009F8DCE70022002024
:1007E000010007B0000008B0263A09B0F8B5444B44
:1007F000444A1C461968013100F081800433934259
:10080000F8D16268404B9A4279D9404B9B6803F11A
:10081000006303F580239A4271D203F0DBFC03F0FE
:10082000EDFC002000F0D8FE0220394B187000F0DB
:1008300011FF384B0021D3F8E820C3F8E810D3F8B3
:100840001021C3F81011D3F81021D3F8EC20C3F80D
:10085000EC10D3F81421C3F81411D3F81421D3F8F1
:10086000F020C3F8F010D3F81821C3F81811D3F80A
:10087000183172B64FF0E023C3F8084DD4E90004F4
:10088000BFF34F8FBFF36F8F234AC2F88410BFF3BB
:100890004F8F536923F480335361BFF34F8FD2F8E6
:1008A000803043F6E076C3F3C905C3F34E335B01F2
:1008B00003EA060C29464CEA81770139C2F87472C2
:1008C000F9D2203B13F1200FF2D1BFF34F8FBFF3CA
:1008D0006F8FBFF34F8FBFF36F8F536923F40033D4
:1008E00053610023C2F85032BFF34F8FBFF36F8FB5
:1008F000202383F31188854680F308882047F8BDBC
:100900000000040820000408FFFF03080022002064
:10091000802200200044025800ED00E0094A49F21C
:100920006900136899B21B0C00FB013344F250615B
:100930001360054B186882B2000C01FB02001860BE
:1009400080B27047182200201422002000211022BB
:1009500010B5044600F092FE034B03CB20606160AB
:100960001868A06010BD00BF00E8F11F2DE9F0433A
:10097000204DBBB002F05CF8AB68C31AF92B32D93A
:1009800006AF2B4628220021A860384602F02EFD33
:1009900005F10E0000F06AFE002604465FFA80F9B9
:1009A00005F10E08F3B2F100994501F1280107D9CC
:1009B00008EB060308223846013602F017FDF1E77E
:1009C000082301220534297B0B48A4B2CDE9023269
:1009D0000A4B01933023CDE90474009303A3D3E9B8
:1009E000002302F01BFB3BB0BDE8F08378F6339F99
:1009F00093CACD8D784700209C3200208547002087
:100A000070B50D4614461E4602F09EFA50B9022EED
:100A100010D1012C0ED112A3D3E900230120C5E986
:100A2000002307E0282C10D005D8012C09D0052C74
:100A30000FD0002070BD302CFBD10BA3D3E90023D5
:100A4000ECE70BA3D3E90023E8E70BA3D3E90023EA
:100A5000E4E70BA3D3E90023E0E700BFAFF3008096
:100A6000401DA12026812A0B78F6339F93CACD8D95
:100A70009E6AC421818A46EE26417272DF25D7B76D
:100A8000F017304A39059E5613B501F0D1FF1949C8
:100A90000B68C31A642B184B08D9184A1C8892F9A2
:100AA00000200860C2EB021222441A80B3F9002031
:100AB000002A1BDA00221A8011490A68821AB2F54C
:100AC0007A7F04D90D4C0860227852422270B3F923
:100AD00000300322002093FBF2F3DBB263F3070044
:100AE00063F30F2063F3174002B010BD962AE3DDD5
:100AF0009622E0E75C480020644800201022002095
:100B00006048002013B504460846202200212346F1
:100B1000019002F06BFC227923460198032A4FF0E2
:100B2000200128BF032203F8042F022202F05EFCFA
:100B3000627923460198072A4FF0220128BF072235
:100B400003F8052F032202F051FCA27923460198F5
:100B5000072A4FF0250128BF072203F8062F03229A
:100B600002F044FC019804F108031022282102F04D
:100B70003DFC382002B010BD2DE9F04FFFB00F460C
:100B8000002140F275120CAE804620A81F9100F0A3
:100B900075FD48220021304600F070FD1FAD01F0C8
:100BA00047FF4FF47A72544B0DF15209B0FBF2F04B
:100BB000186093E80700012386E807000DF1520052
:100BC0003382FFF7C3FE41F204334C49338406AB52
:100BD000184603F0C1FF142229463064304686F8D7
:100BE0003C20FFF78FFF10AB044601460822284641
:100BF00002F0FCFB08220DF141032846A11804F184
:100C0000880A02F0F3FB0DF14203082204F11001FF
:100C1000284604F5847B02F0E9FB11AB202204F1A5
:100C20001801284602F0E2FB12AB402204F1380121
:100C3000284602F0DBFB14AB082204F178012846B9
:100C400002F0D4FB0DF15103082204F18001284683
:100C500002F0CCFB51460AF1080A4B46082228460E
:100C600009F1010902F0C2FBD345F3D104F5887400
:100C70004FF0000919AB08225946284602F0B6FB8E
:100C800096F834304B450AD9B36B214608222846E2
:100C90004B44083409F1010902F0A8FBF0E74FF0DA
:100CA000000996F83C3004EBC9014B4508D9336C78
:100CB000082228464B4409F1010902F097FBF0E7AE
:100CC0000023073140460393C1F3CF01BB7E02935B
:100CD00007F1190301930123CDE904510093F97E33
:100CE00003A3D3E9002302F099F97FB0BDE8F08FA8
:100CF0009E6AC421818A46EE84220020884B000827
:100D00000A4B0B4A10B51A6003F5805393F848203C
:100D10003AB95C6C2CB1204601F006FD204603F088
:100D200085FE0448BDE8104001F0FEBCC83200203A
:100D30007C4C0008F8420020014B1870704700BF3F
:100D400090220020334BF0B51C7B85B034B1324B80
:100D50000E221A810024204605B0F0BD2F4A02ABB6
:100D60001068516803C308232D492E480DEB030278
:100D700003F084FE054630B9274B0A222A481A811F
:100D800001F05AFCE6E70169B1F5E01F06D9224BF4
:100D90000B2226481A8101F04FFCDCE7438B40F21E
:100DA0001342934207D01C490C2008811946204861
:100DB00001F042FCCFE71F4A024402F110039942BE
:100DC00004D2154B10221C481A81E4E71039204642
:100DD0008E1A144901F032FE05F118010746324619
:100DE000204601F02BFEAB689F4202D1EB6898428F
:100DF0000AD0094B0D221A813B4600900F48D5E9D5
:100E0000021201F019FCA5E70D48012401F014FCC1
:100E1000A1E700BF7847002084220020314C000861
:100E2000DCFF1B0000000408A04B0008AC4B0008CE
:100E3000BE4B00080800FCF7DC4B0008F94B00082B
:100E4000224C00082DE9F04FADB080460C4606AFAD
:100E500002F07AF80546002859D1237E022B1BD1D7
:100E6000E38A012B18D101F0E3FD0646FFF756FD9A
:100E700003464FF4C87006F51676DFF8CC92B3FB44
:100E8000F0F202FB103316FA83F3C9F80030E37E68
:100E900033B9A84B00221A709C37BD46BDE8F08FCD
:100EA000A38AEEB20135013BB3420BD93B1DE900E9
:100EB000082220461E4401F0F8010023009602F0AB
:100EC00059F9EDE707F11400FFF740FD324607F14D
:100ED0001401381D03F0C2FD0028DAD10F2E08D806
:100EE000944B1E70D9F80030A3F51673C9F8003082
:100EF000D2E7FB1CF8700146072200930346204608
:100F000002F038F9F978404602F016F8C4E7E38AAF
:100F1000282B26D010D8012B1ED0052BBCD1BFF317
:100F20004F8F8549854BCA6802F4E0621343CB605A
:100F3000BFF34F8F00BFFDE7302BADD1637EE94695
:100F40007F4D01336A7BDBB2934203D1E27E2B7B80
:100F50009A4265D0CD469FE721464046FFF70CFEFA
:100F60009AE7A38A013B9BB2C92B95D8744D2E7B7F
:100F700026BB05F10C030822314600933346204678
:100F800002F0F8F8731CF2B2D9001E46A38A013BA6
:100F90009A4205DA0E3200232A4400920822EEE734
:100FA00000230022C5E900230023AB6085F8D73079
:100FB000C5F8D8302B7B0BB9E37E2B73002507F1E6
:100FC00014093B1D082229464846FD60C7E9015522
:100FD00002F00CFA3B7A05F1010AAB424FEACA066D
:100FE00008D9FB680822314648462B44554602F092
:100FF000FDF9EFE7C6F3CF060023E17E1934039332
:101000004046CDE904966378019402932823009327
:1010100046A3D3E9002302F001F8FFF7A7FC3BE762
:101020004FF0000807F1140310222046A7F814809F
:1010300041460093012302F09DF8A68A023EB6B213
:10104000F31C9B109B000733DB08A9EBC3039D46F1
:101050000DF1180A1FFA88F34FEAC801B34201F1F3
:1010600010010AD20AEB08030822204608F1010801
:101070000093002302F07EF8ECE795F8D70000F02B
:10108000B5FAD5F8D83004461BB995F8D70000F06A
:10109000BDFAD5F8D83033449C4204D295F8D70035
:1010A000013000F0B3FA4FEA960B4FF000081FFA38
:1010B00088F18B45D5E9003209D90AEB8801012274
:1010C00003EB880008F1010800F0E0FAEFE7F318FD
:1010D00095F8D70042F10002C5E90032D5F8D830C2
:1010E00006EB0308C5F8D88000F080FA804509D3E4
:1010F00095F8D730D5F8D8000133001B85F8D730E4
:10110000C5F8D800FF2E08D800232B7300F090FA02
:10111000FFF718FE08B1FFF769FB2B68094A9B0A25
:10112000013313810023AB6014E700BF26417272C4
:10113000DF25D7B79532002000ED00E00400FA0566
:1011400078470020842200209832002010B54FF00C
:1011500040540C4B22689A4212D1627D0A4B0B48D4
:101160001A70C922237D0E30094900F8023C00F0B4
:1011700073FAE0220021204600F080FA012010BD21
:101180000020FCE79AAD44C590220020784700205B
:101190001600003037B50223184D002218496B7134
:1011A0000123184800F05AFE002317494FF48052DB
:1011B0000193164B16480093164B01F097FE164B01
:1011C000197811B1124801F0B7FE01F031FC044664
:1011D000FFF7A4FB4FF4C873B0FBF3F202FB130359
:1011E00004F5167010FA83F00C4B186003F026F823
:1011F00008B10F232B8103B030BD00BF8422002033
:1012000040420F00C832002094220020010A00084A
:101210009C320020450E00089022002098320020C9
:101220002DE9F04FC44D2DED028BBDA7D7E9006726
:1012300095B00FF2F429D9E90089DFF81CA3DFF893
:101240001CB3284601F04EFF034650B3002410940F
:10125000ADF84C40CDE91144027B8DF84C2011AA29
:101260009968406803C21B6843F00043109301F083
:10127000E1FB10EB0A020094584641F1000310A96B
:1012800000F092FAA042AD4A05DD284601F02EFF9B
:10129000AA4A1470D5E71378072B00F2188101339E
:1012A000137000230DACDFF8B4B20C93ADF83C30F2
:1012B0000D9363609FED9E8B00234FF0010A0DF1AB
:1012C000250209A958468DF825308DF824A08DED0A
:1012D000008B01F047F99DF824200023002A40F0FC
:1012E000FA80284601F030FE0446002847D1DFF896
:1012F00070B201F09DFBDBF8003098423FD301F063
:1013000097FB0790FFF70AFB4FF4C873079AB0FBEF
:10131000F3F102F5167201FB130310A812FA83F31E
:10132000CBF80030DFF83CB29BF80010002914BF66
:101330002346534607918DF83030FFF707FB079996
:1013400010AB0DF13100C1F110021944D2B2062ADE
:1013500028BF0622079200F07FF9079A0CAB2846B7
:10136000039301321823D2B20293754B0492324692
:10137000CDE900A33B4601F0E9FD8BF8004001F008
:1013800057FB704A1368C31AB3F57A7F31D31060E4
:1013900001F050FB02460B46284601F0B1FE2846FC
:1013A00001F0D2FD28B3684B0DF1400A674C1B7B5E
:1013B000002B14BF03230223637101F039FB4FF4A8
:1013C0007A735146B0FBF3F020602046FFF79AFB9A
:1013D00018230730424602935D4BC0F3CF000193C0
:1013E00040F25513CDE903A0009328464B4601F087
:1013F000ADFDFFF749FBC0F307238DF84000C0F3B4
:1014000007404FF0080A534A8DF842004FF48071AC
:1014100000208DF84130AAF1080BBBF1330F78D9C9
:10142000ABF134041923B4FBF3FC03FB1C43002B86
:1014300071D0A4EB0C041823B4FBF3F3984210D042
:101440000793FFF721FB4FF48071C0F3072C8DF851
:101450004000C0F307403F4A079B8DF841C08DF81C
:1014600042004FF0180CB4FBFCF00CFB10400DF1E7
:10147000500C04F007040CEBD000C4F1080410F881
:10148000100C40FA04F4184604F00104002C0BF18F
:10149000010B51830CBF4FF000730023DA4543EA80
:1014A000442494611183B8D10AF1080ABAF1A00F5B
:1014B000B1D1254C237B2BB1FFF758FA237B002BAE
:1014C0007FF4BBAE15B0BDEC028BBDE8F08F2846B3
:1014D00001F00CFEE5E61946102210A800F0CEF847
:1014E0000DF126030AAA0CA9584600F065FB11ABC2
:1014F00094E8030083E803009DF83C3010A92846D7
:101500008DF84C300C9B1093DDE90A2301F0B6FFF7
:10151000D2E60024BAE70124B8E700BFAFF30080A9
:10152000401DA12026812A0BF1C6A7C1D068080F53
:1015300000000000000000009C32002067480020EE
:101540009432002058480020784700208422002050
:10155000664800200004025840420F00C8320020B4
:10156000983200209532002008B5054800F0CAFBEB
:10157000044A05490020BDE8084003F051BA00BF05
:10158000C8320020A4480020010D000870B5104C9E
:101590000025104E02F05AFC2080306823888342D8
:1015A0000CD800252088013802F04CFC2388054423
:1015B000013BB5F5802F2380F4D370BD02F042FCCF
:1015C000336805440133B5F5802F3360E5D3E8E790
:1015D000944800206848002002F016BD00F1006029
:1015E000920000F5802002F093BC0000054B1A68C1
:1015F000054B1B889B1A834202D9104402F022BC7F
:1016000000207047684800209448002038B5074DF6
:1016100004462868204402F01BFC28B928682044AE
:10162000BDE8384002F026BC38BD00BF6848002045
:10163000064991F8243033B100230822086A81F862
:101640002430FFF7CBBF0120704700BF6C4800205B
:101650000020704770470000002310B5934203D06C
:10166000CC5CC4540133F9E710BD000003460246C8
:10167000D01A12F9011B0029FAD17047024403461F
:10168000934202D003F8011BFAE770472DE9F843B3
:101690001F4D14460746884695F8242052BBDFF8B4
:1016A00070909CB395F824302BB92022FF21484636
:1016B0002F62FFF7E3FF95F824004146C0F10802CE
:1016C00005EB8000A24228BF2246D6B29200FFF767
:1016D000C3FF95F82430A41B17441E449044E4B281
:1016E000F6B2082E85F82460DBD1FFF7A1FF0028B1
:1016F000D7D108E02B6A03EB82038342CFD0FFF7F8
:1017000097FF0028CBD10020BDE8F8830120FBE73C
:101710006C480020202383F3118862B670470000D4
:10172000002383F3118862B67047000001207047E0
:10173000704700007047000010B413460268146838
:101740000022A4465DF8044B6047000000F580507D
:1017500090F859047047000000F5805090F852044A
:101760007047000000F5805090F958047047000061
:101770004E20704700F5805208B5FFF7CBFFD2F836
:101780009834D2F894041844D2F890341844D2F81B
:1017900078341844D2F888341844D2F88434184481
:1017A000FFF7BEFF08BD00002DE9F74F0C4600F51E
:1017B00080511F46054691F852349046BDF830904E
:1017C0009BB1D1F874340133C1F8743423689A00A2
:1017D00006D4237B082B0BD9627B0AB10F2B07D9C8
:1017E000D1F878340133C1F878344FF0FF300FE08E
:1017F000FFF790FFEB6AD3F8C42012F4001A0AD066
:10180000D1F87C3400200133C1F87C34FFF788FF25
:1018100003B0BDE8F08F22684FF0480BD3F8C460E6
:10182000002A6B6AC6F30446B4BF42F080429204B9
:101830001BFB063BCBF8002023685B004FEA0663E6
:1018400044BF42F00052CBF80020227B43EA02431F
:101850007201CBF80430607B18B343F44013CBF82B
:101860000430D1F8A4340133C1F8A434AB1803F523
:101870008353197B41F020011973207B019200F002
:1018800037FF0330019A80105FFA8AF30AF1010AE8
:1018900083420DDA04EB83010BEB83034968996003
:1018A000F2E7AB1803F58353197B60F34511E3E7C7
:1018B0000121EB6A04F10C00B140C3F8D010AB1861
:1018C000214603F58253C3E9048705EB461303F56C
:1018D0008253183351F804CB814243F804CBF9D139
:1018E00009882A442846198041F26803D65002F537
:1018F000805209F0030392F86C1043F0100321F0BA
:101900001F010B43214682F86C304246FFF708FF67
:101910003B46CDF8309003B0BDE8F04F00F0AEBECE
:101920002DE9F04700F58056044696F85254002DF4
:1019300040F00181037C032B40F092802B46284627
:101940002F465FFA83FC944510DA01EBCC0E51F878
:101950003CC0BCF1000F04DBDEF804C0BCF1000F9A
:1019600002DB01370133ECE70130FBE7FFF7D2FE82
:10197000E36AF0B9D3F8800040F00200C3F88000B9
:101980004E23E06A002F6ED1D0F8803043F001037F
:10199000C0F88030694B6A4A1B6803F1805303F535
:1019A0002C539B009342A36240F2AF80654801F044
:1019B00039F84D2842D8DFF884814FEA004EDFF82D
:1019C0008891D8F800C04EEA8C0EC3F884E00CF180
:1019D000805303F52C539B00636100EB0C03D4F898
:1019E0002CC0C8F80030C0F14E03DCF8800040F095
:1019F0003000CCF880004FF0000CD4F81480E6469C
:101A00005FFA8CF08242BCDD01EBC00A51F8300075
:101A1000002810DBDAF804A0BAF1000F0BDA09EAAB
:101A200000400AF07F0A40EA0A0040F0084048F807
:101A30002E000EF1010E0CF1010CE1E79A6922F083
:101A400001029A6100F0F4FF0646E36A9B69D90738
:101A500004D500F0EDFF831BFA2BF6D9FFF760FEEB
:101A60002846BDE8F087B7EB530F3DD2DFF8CCE056
:101A70004FEA074CDEF800304CEA830CC0F888C00F
:101A800003F1805003EB4703002700F52C50CEF8FC
:101A90000030BC468000A061E06AD0F8803043F09E
:101AA0000C03C0F88030D4F818E0FBB29A427FF7FC
:101AB00071AF51F8330001EBC3080028D8F80430A7
:101AC00001DB002B0EDB20F0604023F0604340F090
:101AD000005043F000434EF83C000EEBCC000CF1FC
:101AE000010C43600137E0E7836923F00103836160
:101AF00000F09EFF0646E36A9B69DA07AED500F068
:101B000097FF831BFA2BF6D9A8E7E26A936923F0C3
:101B10000103936100F08CFF0746E36A9B69DB07D2
:101B200005D500F085FFC31BFA2BF6D996E70125F2
:101B300086F8525492E7002592E700BFA0480020A3
:101B4000FCB500403C4C00080000FF0713B500F551
:101B500080540191606C00F01DFE1F280AD92022DC
:101B60000199606C00F08CFEA0F1200358425841AE
:101B700002B010BD0020FBE700F5805008B5FFF76C
:101B8000C9FD406C00F0DAFDBDE80840FFF7C8BDB4
:101B9000002202608281426082607047002200233E
:101BA00010B5C0E90023002304460C3020F8043CA3
:101BB000FFF7EEFF204610BD2DE9F047074688B03D
:101BC0009A46884607F5805468469146FFF7A2FD7D
:101BD000FFF7E4FF606C00F0C3FD1F282DD9202221
:101BE0006946606C00F0D0FE202826D194F852346B
:101BF0001BB303AD444605AB2E46083403CE9E42CC
:101C000044F8080C44F8041C3546F5D130684146C8
:101C100020603846B388A380DDE90023C9E90023AA
:101C2000BDF808304A46AAF80030FFF779FD534660
:101C300008B0BDE8F04700F00FBD0020FFF770FDD1
:101C400008B0BDE8F08700002DE9F84F00230646F4
:101C500000F58154054688461034C0E90133264B0F
:101C600046F8303B374638462037FFF797FFA74204
:101C7000F9D105F580544FF4805305F5A3594FF081
:101C8000000A26630026676405F5835709F11009E9
:101C90004FF0000B1037E663C4E90D36012384F8DA
:101CA000403084F84830A7F11800203747E910ABDE
:101CB000FFF76EFF47F8286C4F45F4D184F858843D
:101CC000A4F85A64A4F85C64A4F85E6484F86064C0
:101CD000A4F86264A4F86464A4F8666484F8686490
:101CE000B8F1000F02D0054800F09CFE044B2846D6
:101CF000EB62BDE8F88F00BF7C4C0008604C000828
:101D000000A00040044B10B5197804464A1C1A7014
:101D1000FFF79AFF204610BD9D4800202DE9F047AF
:101D200000295FD0304F3148B7FBF1F581428CBFBD
:101D30000A201120431EB5FBF0FC00FB1C50DCB256
:101D400020B1022B1846F5D8002037E00CF1FF3502
:101D5000B5F5806F32D2C4EBC4094FF47A7009F143
:101D600003034FEAE308C3F3C70308F1010AA4EB36
:101D7000030E08FB00085FFA8EF65AFA8EFEB8FBD7
:101D8000FEFEBEF5617F1BDC1FFA8EF4581C56FA6E
:101D900080F00CFB00FCB7FBFCFC6145D4D1013B9F
:101DA000DBB20F2BD0D8711E0020C9B2072905D88D
:101DB000107101201480558053719171BDE8F08736
:101DC00009F1FF334FEAE30EC3F3C7030EF1010835
:101DD000E41A0EFB0000E6B258FA84F4B0FBF4F407
:101DE000A4B2D3E70846E9E700B4C4043F420F00B9
:101DF00038B540F27772C36A154CC3F8BC2007228D
:101E0000C36AC3F8C8202268C16A930043F4C023A0
:101E1000C1F8A03002F1805302F16C01C56A03F5EC
:101E20002C53EA3289009B00226041F0E061094AAC
:101E3000C361C5F8C01003F5D87103F56A73416238
:101E40009342836202D9044800F0ECFD38BD00BF24
:101E5000A0480020FCB500403C4C00082DE9F04FA4
:101E600000F58055994689B0044695F858348A465D
:101E70009046012B04D90027384609B0BDE8F08F01
:101E8000974A52F8231009B942F823009549C4F83B
:101E90000CA00B7884F81090C3B9FFF73BFC924B71
:101EA000D3F8EC2042F48072C3F8EC20D3F89420ED
:101EB00042F48072C3F89420D3F8942022F4807204
:101EC000C3F8942001230B70FFF72AFC95F85134D6
:101ED00073B902211320FFF71DFC01F02DFD022133
:101EE000152001F029FD012385F85134FFF718FC76
:101EF000FFF710FCE26A936923F01003936100F08E
:101F000097FD0746E36A9E6916F0080607D000F0C1
:101F10008FFDC31BFA2BF5D9FFF702FCABE79A69DB
:101F200042F001029A6100F083FD0746E36A9A6974
:101F3000D00705D400F07CFDC31BFA2BF6D9EBE7E4
:101F40009A69002704F5825B42F002020BF1100B44
:101F50009A61E36A5F65FFF7E3FB686C00F0EEFBF4
:101F6000202200216846FFF789FB02A8FFF710FE38
:101F70006A460BEB06030DF1180E069794460833DC
:101F8000BCE80300F44543F8080C43F8041C62461F
:101F9000F4D1DCF8000020361860B6F5806F9CF8AC
:101FA00004201A71DCD1002304F5A25251462046C8
:101FB0001A3285F8503485F85334FFF7AFFE0746E0
:101FC00090B9E26A936923F00103936100F030FD58
:101FD0000546E36A9B69D9077FF54DAF00F028FD00
:101FE000431BFA2BF5D946E795F85F6495F85E2414
:101FF0003602C5F86CA4E36A46EA426695F86024A6
:102000001643B5F85C2446EA0246DE61B8F1000FDB
:1020100029D004F5A352414620460232FFF77EFE46
:1020200090B9E26A936923F00103936100F000FD27
:102030000546E36A9B69DA077FF51DAF00F0F8FCFF
:10204000431BFA2BF5D916E795F8683495F8671411
:102050001B01C5F87084E26A43EA0123B5F86414F1
:1020600043EA0143D360E36A00262046C3F8BC601C
:10207000FFF7BEFE85F859646FF04042E36AB9F19C
:10208000030F1A65194AE36A5A654FF00222E36AA0
:102090009A654FF0FF32E36AC3F8E0204FF0030285
:1020A000E36ADA65E26A936943F4407393613FF44B
:1020B000E3AEE26A936923F00103936100F0B8FC98
:1020C0000646E36A9B69DB0705D500F0B1FC831B7C
:1020D000FA2BF6D9CFE6012385F85234CCE600BFBF
:1020E000984800209C4800200044025855020002F5
:1020F0002DE9F04F054689B090469946002741F2F8
:10210000680A00F58056EB6AD3F8D830FB40D80750
:102110004AD505EB47124FEA471B5244137919077A
:1021200042D4D6F880340133C6F8803413799A0645
:1021300005EB0B0248BFD6F8A834524444BF013324
:10214000C6F8A834137943F008031371DB0723D5CD
:1021500096F8533403B305F582546846FFF71EFD25
:1021600003AB18345C4404F1080C2068083454F8BC
:10217000041C1A46644503C21346F6D1206869461A
:1021800010602846A2889A800123ADF808302B6899
:10219000CDE900891B6C9847D6F8543423B1D6F8A2
:1021A0009C340133C6F89C340137202FABD109B0E1
:1021B000BDE8F08F2DE9F04F0F468DB0044600F0DA
:1021C00039FC82468946002F5BD1E36AD3F8A02010
:1021D00012F4FE0F03D100200DB0BDE8F08FD3F84C
:1021E000A420920141BF04F58051D1F8942401321A
:1021F000C1F89424D3F8A4205606ECD0D3F8A45008
:10220000E669C5F305254823E8464FF0000B03FBBC
:1022100005664046FFF7BCFC326851004ABF22F019
:102220006043C2F38A4343F00043920048BF43F047
:1022300080430093736813F400131BBF012304F55C
:1022400080528DF80D308DF80D301EBFD2F8AC34B1
:102250000133C2F8AC34F38803F00F038DF80C306F
:102260009DF80C0000F044FA5FFA8BF3984225D9F0
:10227000F2180CA90BF1010B127A0B4403F82C2C69
:10228000EEE7012FA7D1E36AD3F8B02012F4FE0FD6
:10229000A1D0D3F8B420950141BF04F58051D1F805
:1022A00094240132C1F89424D3F8B420500692D07B
:1022B000D3F8B450266AC5F30525A4E7EFB9E36A5D
:1022C000C3F8A85004A807ADFFF768FC98E80F0012
:1022D00007C52B800023204604A9ADF818302368D9
:1022E00004F580541B6CCDE904A9984758B1D4F883
:1022F0008C340133C4F88C346EE7012FE2D1E36AE9
:10230000C3F8B850DEE7D4F8903401200133C4F8A4
:10231000903461E7F8B505460F4600F58054012674
:1023200039462846FFF746FF10B184F85364F7E7B3
:10233000D4F8543423B1D4F89C340133C4F89C3419
:10234000F8BD0000C36AF0B51A6C12F47F0F2BD0F1
:102350001B6C00F5805441F268054FF0010CC4F885
:10236000A0340023471900EB43125E012A4411797F
:1023700011F0020F15D0490713D4B959C66A0CFAE7
:1023800001F1D6F8CCE011EA0E0F0AD0C6F8D4104D
:10239000117941F004011171D4F888240132C4F894
:1023A00088240133202BDED1F0BD000010B5264C6F
:1023B000264B22680AB340B31A6D92050FD54FF42D
:1023C00000721A6500F036FB50EA01020B4602D09B
:1023D000013861F1000302462068FFF789FE1B4ABD
:1023E000136D9B012AD523684FF0007103F58053CC
:1023F0001165012283F8592420E001221A65102278
:102400001A654FF480521A6510BD196DC80702D4C1
:10241000196D490705D50521104619650021FFF7FB
:1024200079FF0A4B1A6DD00602D41A6D510605D5F4
:10243000502201211A652068FFF76CFF2068BDE873
:102440001040FFF77FBF00BF9848002000A0004069
:1024500008B5FFF75FF9FFF775FFBDE80840FFF724
:102460005FB90000C36AD3F8C00010F07C5005D0FB
:10247000D3F8C40080F40010C0F34050704700004F
:1024800000F5805008B5FFF745F9406C00F068F999
:10249000FFF746F943090CBF0120002008BD0000EA
:1024A00000F5805393F8592462B1C16A8A6922F019
:1024B00001028A61D3F898240132C3F898240022DB
:1024C00083F85924704700002DE9F74300F5825145
:1024D00098460025FFF71EF9103141F2680E4FF0C3
:1024E000010900F5805C00EB4514744423795E0714
:1024F0001CD4DB061AD58E69C36A09FA06F6D3F82E
:10250000CC703E4212D04F6801970F689742019FEE
:1025100077EB08070AD2C3F8D460237943F00403A9
:102520002371DCF884340133CCF884340135203154
:10253000202DD8D103B0BDE8F043FFF7F1B800007B
:10254000F8B51E4600230F46054613701446FFF7E4
:1025500097FF80F0010038701EB12846FFF782FF18
:102560002070F8BD2DE9F04F994685B00B780E46E6
:102570008046174601931378DDE90EBA029300F006
:1025800059FA337804460D4613B93B78002B41D0F5
:1025900022462B464046FFF797FFFFF759FFFFF70C
:1025A0007FFF4B463A463146FFF7CAFF33782BB1DF
:1025B000019B1BB1012005B0BDE8F08F3B7813B142
:1025C000029B002BF6D108F5805303935C4575EB15
:1025D0000A031FD2039BD3F85404D8B1BBEB040207
:1025E0000368D9686AEB050388474B463A4631468B
:1025F0004046FFF7A5FF337813B1019B002BD9D1DB
:102600003B7813B1029B002BD4D100F013FA04469F
:102610000D46DBE70020CEE708B50020FFF7C6FE39
:10262000BDE8084001F05EB908B50120FFF7BEFE25
:10263000BDE8084001F056B90FB4002004B070475F
:1026400013B56C46031D84E8060094E8030083E894
:102650000500012002B010BD73B58568019155B128
:102660001B885B0707D4D0E90036DB6B9847019ADB
:10267000C1B23046A847012002B070BDF0B58668EF
:1026800089B005460C465EB1BDF838305B070AD408
:10269000D0E90037DB6B98472246C1B23846B047D5
:1026A000012009B0F0BD0022002301F10806CDE9A8
:1026B000002300230A46ADF8083003AB1068083247
:1026C00052F8041C1C46B24203C42346F6D11068DB
:1026D00020609288A28000F0AFF90423ADF80830A2
:1026E0002B68CDE900011B6C694628469847D7E75F
:1026F000082817D909280CD00A280CD00B280CD090
:102700000C280CD00D280CD00E2814BF40203020EF
:1027100070470C2070471020704714207047182015
:10272000704720207047000010B5037C044613B9A1
:10273000006802F08BF9204610BD00000023BFF3B3
:102740005B8FC360BFF35B8FBFF35B8F8360BFF3AF
:102750005B8F7047BFF35B8F0068BFF35B8F704781
:1027600070B505460C30FFF7F5FF044605F1080685
:102770003046FFF7EFFFA04206D96D683046FFF7FD
:10278000E9FF2544281A70BD3046FFF7E3FF201A01
:10279000F9E7000070B505464068A0B105F10C06E8
:1027A00005F10800FFF7D6FF04463046FFF7D2FFD9
:1027B000844204F1FF34304694BF6D680025FFF772
:1027C000C9FF2C44201A70BD38B50C460546FFF7EA
:1027D000C7FFA04210D305F10800FFF7BBFF044478
:1027E0006868BFF35B8FB4FBF0F100FB114401207C
:1027F000AC60BFF35B8F38BD0020FCE72DE9F041F2
:10280000144607460D46FFF7C5FF844228BF04461D
:10281000D4B1B84658F80C6B4046FFF79BFF3044E4
:10282000286040467E68FFF795FF331A9C4203D824
:1028300001206C60BDE8F081A41B6B603B68204404
:10284000AB60E8600220F5E72046F3E738B50C46B8
:102850000546FFF79FFFA04210D305F10C00FFF7DC
:1028600079FF04446868BFF35B8FB4FBF0F100FBB1
:1028700011440120EC60BFF35B8F38BD0020FCE702
:102880002DE9FF418846694607466C46FFF7B6FFCB
:10289000002506B204EBC606B4420AD0626808EB13
:1028A000050120680834FEF7D7FE54F8043C1D44A7
:1028B000F2E729463846FFF7C9FF284604B0BDE8CD
:1028C000F0810000F8B505460C300F46FFF742FFD7
:1028D00005F1080604463046FFF73CFFA0423046AB
:1028E00088BF6C68FFF736FF201A386020B12C686B
:1028F0003046FFF72FFF2044F8BD000073B51446A3
:1029000006460D46FFF72CFF8442019028BF04467F
:10291000DCB101A93046FFF7D5FF019B33B932681E
:10292000C5E90233C5E9002401200CE09C4228607F
:1029300038BF0194019884426860F5D93368241A3D
:102940000220AB60EC6002B070BD2046FBE70000E7
:102950002DE9FF410F4669466C46FFF7CFFF00B2F5
:10296000002604EBC005AC4209D0D4F80480B819A5
:1029700054F8081B42464644FEF76EFEF3E7304625
:1029800004B0BDE8F081000038B50546FFF7E0FF70
:10299000044601462846FFF717FF204638BD0000D1
:1029A00000B59BB0EFF3098168226846FEF754FE3C
:1029B000EFF30583044B9A6BDA6A9A6A9A6A9A6A09
:1029C0009A6A9A6A9B6AFEE700ED00E000B59BB048
:1029D000EFF3098168226846FEF73EFEEFF30583B8
:1029E000044B9A6B9A6A9A6A9A6A9A6A9A6A9B6A7A
:1029F000FEE700BF00ED00E000B59BB0EFF30981FA
:102A000068226846FEF728FEEFF30583034B5A6BF6
:102A10009A6A9A6A9A6A9A6A9B6AFEE700ED00E0EF
:102A2000FEE700000FB408B5029801F075F8FEE764
:102A300001F032BB01F00ABB01F008BB30B50A441B
:102A4000084D91420DD011F8013B5840082340F346
:102A50000004013B2C4013F0FF0384EA5000F6D140
:102A6000EFE730BD2083B8ED2DE9F041C56915B918
:102A7000C161BDE8F0814B68AC4623F06047C3F309
:102A80008A464FEAD37EC3F3807816EA230638BF1E
:102A90003E462B465A68BEEBD27F22F060440AD0F5
:102AA000002A18DAA40CB44217D19D420FD10D6050
:102AB000DEE71346EEE7A74207D102F08044C2F3F7
:102AC000807242450BD054B1EFE708D2EDE7CCF865
:102AD00000100B60CDE7B44201D0B442E5D81A68CB
:102AE0009C46002AE5D11960C3E700002DE9F047B4
:102AF000089D01F0070400EBD1004FF47F494FEA35
:102B0000D508224405F00705944201D1BDE8F087BD
:102B100004F0070705F0070A111B08EBD50E57450F
:102B20003E4613F80EC038BF5646C6F108068E4220
:102B300028BF0E46E108415C34443544B94029FAC7
:102B400006F721FA0AF1FFB28CEA010147FA0AF707
:102B500039408CEA010C03F80EC0D5E780EA012069
:102B6000082341F2210201B2013B4000002980B25A
:102B7000B8BF504013F0FF03F5D1704738B50C468D
:102B80008D18A54200D138BD14F8011BFFF7E6FFF0
:102B9000F7E7000002684AB1136801890360C3883F
:102BA00001339BB29942C38038BF038110467047FE
:102BB00070B588B0044620220D4668460021FEF715
:102BC0005DFD20460495FFF7E5FF024660B16B46C8
:102BD000054608AE1C46083503CCB44245F8080C3F
:102BE00045F8041C2346F5D1104608B070BD00001E
:102BF000082817D909280CD00A280CD00B280CD08B
:102C00000C280CD00D280CD00E2814BF40203020EA
:102C100070470C2070471020704714207047182010
:102C20007047202070470000082817D90C280CD9BD
:102C300010280CD914280CD918280CD920280CD904
:102C400030288CBF0F200E207047092070470A20C3
:102C500070470B2070470C2070470D207047000014
:102C600010B54B6823B9CA8A63F30902CA8210BD42
:102C7000C4681A681C60C360438A013B43824A608F
:102C8000EFE700002DE9F84F1D46CB8A0F4681463D
:102C9000C3F30901924606290B4630D00020AAB2A0
:102CA00007F119049EB21FFA80F8052E0FD890453F
:102CB00003F1010306D30A44FB8A62F309030120EE
:102CC000FB821AE01AF800600130E654EAE790450A
:102CD000F1D2A1F1060B1C237C68BBFBF3F203FBD2
:102CE00012BB1FFA8BF6002C45D14846FFF752FF66
:102CF000044638B978606FF00200BDE8F88F4FF0F5
:102D00000008E6E7002606607860ADB24FF0000BE1
:102D1000454510D90AEB0803221D13F8011B08F1E1
:102D200001089155B1B21FFA88F81B292BD04545EF
:102D300006F10106F1D8FB8AC3F30902154465F3D5
:102D40000903BCE701321C4692B22368002BF9D17B
:102D5000AB1F0B441C21B3FBF1F301339BB29A422E
:102D6000D3D2BBF1000FD0D14846FFF713FF20B9F3
:102D7000C4F800B0BFE70122E7E7C0F800B05E4644
:102D800020600446C1E74545D5D94846FFF702FF14
:102D900008B92060AFE7C0F800B000262060044604
:102DA000B6E700002DE9F04F2DED028B83B007460A
:102DB0009146BDF83C50CDE90013002A00F0928006
:102DC0002DB10E9B002B00F08D80072D32D807F11E
:102DD0000C00FFF7DFFE044638B96FF0020420460E
:102DE00003B0BDEC028BBDE8F08F14220021FEF78A
:102DF00045FC2A460E9904F10800FEF72DFC681CDC
:102E0000C0B2FFF711FFFFF7F3FE207499F800300E
:102E1000013803F01F0314FA80F063F03F030372DC
:102E20003846009B43F0004161602146FFF71CFEDD
:102E30000124D4E74FF0000800F10C034FF0800AA2
:102E40004646444608EE103A18EE100AFFF7A2FE76
:102E500083460028C1D014220021FEF70FFCC6BB18
:102E6000019B0220ABF808300E9B00F10802991973
:102E70005BFA82F20130C0B2082801D0AE422AD3F8
:102E8000FFF7D2FEAE4208BF4FF0400AFFF7B0FE98
:102E900099F80020411E009B02F01F0201345BFAEA
:102EA00081F142EA481288F0010824B24AEA020A93
:102EB00043F0004281F808A059468BF810003846CC
:102EC000CBF804204FF0000AFFF7CEFDAE42BBD195
:102ED00085E70020C8E711F801CB013602F801CBE5
:102EE000B6B2C7E76FF0010479E70000F8B5154600
:102EF0000E462822002104461F46FEF7BFFB069B14
:102F0000B5F5001FA760636004F10C00079B34BF98
:102F10006A094FF6FF722362002397B29A4205D8DE
:102F20000023036027826382A382F8BD0660013319
:102F300030462036F2E7000003781BB94BB2002B75
:102F4000C8BF017070470000007870472DE9F74F47
:102F5000DDF83C90804692469B46BDF830500D9E71
:102F60009DF83840BDF84070B9F1000F01D1002F35
:102F700051D11F2C4FD898F80000B0B9072F47D86F
:102F800035F0030347D13A4649464FF6FF702D020C
:102F9000FFF7F4FD20F0010045EA04644004400C12
:102FA00044EA40244FF6FF7321E040EA0520072F52
:102FB00040EA0464F6D900254FF6FF73C5F12000FE
:102FC000A5F120022AFA05F108350BFA00F02BFAD8
:102FD00002F2014318461143C9B2FFF7BFFD402D6D
:102FE0000346EBD13A464946FFF7C8FD0346324651
:102FF00021464046CDE90097FFF7D4FE33780133F0
:10300000DBB21F2B88BF0023337003B0BDE8F08F05
:103010006FF00300F9E76FF00100F6E72DE9F04FDC
:1030200085B0924606469B46DDF848800F9D9DF888
:1030300040209DF84490BDF84C70B8F1000F01D1CC
:10304000002F49D11F2A47D83378002B47D00C02D4
:103050009DF83810072F44EA026444EAC93444EA70
:10306000014444EA030444F0800432D900234FF6BB
:10307000FF72C3F1200CA3F120002AFA03F103939D
:103080000BFA0CFC2BFA00F041EA0C01014310464C
:10309000C9B2FFF763FD039B02460833402BE8D11A
:1030A0003A464146FFF76AFD03462A462146304626
:1030B000CDE90087FFF776FEB9F1010F06D12B7835
:1030C0000133DBB21F2B88BF00232B7005B0BDE896
:1030D000F08F4FF6FF73E8E76FF00100F6E76FF04F
:1030E0000300F3E7C06900B104307047C3691A6890
:1030F000C261C2681A60C360438A013B4382704761
:103100002DE9F041D0F8188014461D46184E41466E
:10311000002709B9BDE8F081D1E90223A21A65EBC5
:103120000303964277EB03031ED283698B420DD1D2
:10313000FFF796FD83691B688361C3680B60438A50
:10314000C160013B816943828846E2E7FFF788FD61
:103150000B68C8F80030C3680B60438AC160013B4C
:103160004382D8F80010D4E788460968D1E700BF49
:1031700080841E002DE9F04F8BB00D4614469B460F
:10318000DDF850908046002800F01881B9F1000F5A
:1031900000F01481531E3F2B00F21081012A03D14D
:1031A000BBF1000F40F00A810023CDE90833B8F8E5
:1031B0001430B5EBC30F4FEAC30703D300200BB0A5
:1031C000BDE8F08F2B199F42D8F80C3036BF7F1B1B
:1031D0002746FFB21BB9D8F81030002B7AD02F2D1C
:1031E0004DD8C5F1300600232946B742009308ABFD
:1031F000D8F808002CBFF6B23E46A7EB060A3544C5
:1032000032465FFA8AFAFFF771FCB8F814303021C1
:1032100003F10053063BDB000493D8F80C30039312
:10322000039B13B1BAF1000F2CD1D8F8100040B1B4
:10323000BAF1000F05D008AB5246691A0096FFF7A5
:1032400055FC38B2002FB9D066070AD00AAB6242EB
:1032500003EBD40102F0070211F8083C134101F816
:10326000083C082C3DD9102C40F2B580202C40F2AF
:10327000B780BBF1000F00F09C80082335E0BA4610
:103280000026C2E7049BE02B28BFE02306930B44F3
:10329000AB42059315D95A1B0398691A00969245BB
:1032A00008AB00F1040034BF5246D2B20792FFF7D8
:1032B0001DFC079A1644AAEB020A1544F6B25FFAFF
:1032C0008AFA049B069A05999B1A0493039B1B6830
:1032D0000393A5E700933A4608AB2946D8F80800BF
:1032E000ADE7BBF1000F13D00123B4EBC30F6BD0DC
:1032F000082C12D89DF82030621E23FA02F2D5075E
:1033000006D54FF0FF3202FA04F423438DF8203043
:103310009DF8203089F8003051E7102C12D8BDF804
:103320002030621E23FA02F2D10706D54FF0FF3299
:1033300002FA04F42343ADF82030BDF82030A9F898
:1033400000303CE7202C0FD80899631E21FA03F3C4
:10335000DA0705D54FF0FF3202FA04F40C43089463
:10336000089BC9F800302AE7402C2AD0611EC4F11E
:103370002102A4F12103DDE9086526FA01F105FA2D
:1033800002F225FA03F311431943CB0711D50122A9
:10339000A4F12003C4F1200102FA03F322FA01F19F
:1033A000A2400B43524263EB430332432B43CDE92C
:1033B0000823DDE90823C9E9002300E76FF00100D5
:1033C000FDE66FF00800FAE6082CA1D9102CB4D95C
:1033D000202CEED8C4E7BBF1000FAED0022384E767
:1033E000BBF1000FBCD004237FE70000012A30B5F9
:1033F000144638BF012485B00025402C28BF402446
:10340000012ACDE9025518D81B788DF808306307DA
:103410000AD004AB624203EBD40502F0070215F8B0
:10342000083C934005F8083C0346009122460021E1
:1034300002A8FFF75BFB05B030BD082AE4D9102ACB
:1034400003D81B88ADF80830E1E7202A95BF1B6838
:10345000D3E900230293CDE90223D8E710B5CB6866
:103460001BB98B600B618B8210BDC4681A681C602D
:10347000C360438A013B4382CA60F0E72DE9F04F05
:10348000D1F8008093B004460D4618F0800FCDE9C6
:103490000323C8F3C01219BFC8F3C03BC8F3062604
:1034A0004FF0020B1646B8F1000F80F2D18118F0F0
:1034B000C043059340F0CC810B7B002B00F0C8810A
:1034C000BBF1020F03D00178B14240F0C48108F093
:1034D0007F0106916AB3C8F3074A2B447606069A21
:1034E00046EA0B4693F8039046EA82465FEAD91310
:1034F00046EA0A06079300F09080002200236768DE
:103500000AA92046CDE90A23069B524600935B4652
:10351000B84700287ED0A7699FB9314604F10C0056
:10352000FFF746FB0746E0B96FF0020013B0BDE8B5
:10353000F08FC8F30F2A18F07F0F08BF0AF0030AB4
:10354000CBE73B699E420DD03F68002FF9D1314651
:1035500004F10C00FFF72CFB07460028E4D0A36918
:103560003B60A76100264FF6FF70DDE90A23C6F134
:10357000200E22FA06F1A6F1200C083603FA0EFE00
:10358000099223FA0CFC089341EA0E0141EA0C016E
:10359000C9B2FFF7E3FA402EDDE90832E7D1B8827D
:1035A000FB7D09F01F06C8F30468C3F384039B1B6B
:1035B00098B2002BD7E90221BCBF00F120031BB257
:1035C00052EA01000FD00398821A049860EB0101BF
:1035D000A74890424FF000028A4104D3079A002A7C
:1035E0005BD0012B23DDFA7D4FEA89033946204663
:1035F00002F0030203F07C031343FB75FFF730FB7B
:10360000079BA3B9FB7DC3F38402013262F38603F7
:10361000FB7504E06FF00B0088E7A76917B96FF03E
:103620000C0083E73B699E42BAD03F68F6E719F089
:10363000400F32D0039B142200210DA8BB60049BD5
:10364000FB60FEF71BF8039B0AA920460A93049B24
:10365000ADF83EA00B932B1D8DF840B00C932B7B47
:103660008DF84160013B8DF84280DBB2ADF83C3013
:10367000069B8DF8433094F8243083F001038DF8D5
:103680004430A3689847FB7DC3F38403013303F000
:103690001F039B02FB82002048E7FB7DC9F3401219
:1036A000B2EBD31F40F0DA80C3F38403B34240F09F
:1036B000D88007994FEA99122B7B002934D0D20782
:1036C00041D4032B40F2D080039BAE1D394604F158
:1036D0000C00BB603246049BFB602B7B033BDBB2E0
:1036E000FFF7D0FA00280DDA20463946FFF7B8FA7E
:1036F000FB7D0320C3F38403013303F01F039B020C
:10370000FB8213E7AB883B832A7B033AD2B2B88AA9
:103710003146FFF733FAFB7DB882DA43C2F3C012B9
:1037200062F3C713FB75B6E76AB92E1D013B394634
:1037300004F10C00DBB23246FFF7A4FA0028D3DB19
:103740002A7B013AE2E7F98A013BC1F30901DAB2C7
:10375000052959D8281D002307F11A0C9A4208D9C7
:1037600010F801EB01330CF801E00131DBB206295E
:10377000F4D1039993420A9138BF043304992CBFC2
:10378000002355FA83F30B9107F11A010C91796824
:103790000E930D91291DFB8AADF83EA0C3F30903DA
:1037A0008DF840B08DF841601A44069B8DF8428038
:1037B0008DF8433094F82430ADF83C2083F00103B9
:1037C0008DF844300023B88A7B602A7B013AFFF7EA
:1037D000D5F93B8BB882834203D1A3680AA920465E
:1037E000984720460AA9FFF739FEFB7DB88AC3F344
:1037F0008403013303F01F039B02FB823B8B98423F
:1038000014BF1120002091E67B68002BB1D0062068
:1038100001E01C306346D3F800C0BCF1000FF8D1C2
:10382000091A05F1040C081D00EB030905989DF821
:10383000143001EB000EBEF11B0F9AD89A4298D9B2
:103840001CF8013B09F8013B059B01330593EDE7AB
:103850006FF009006AE66FF00A0067E66FF00D008E
:1038600064E66FF00E0061E66FF00F005EE600BFE9
:1038700080841E00EFF30983054968334A6B22F008
:1038800001024A6383F30988002383F31188704798
:1038900000EF00E0202080F3118862B60D4B0E4A45
:1038A000D96821F4E0610904090C0A430B49DA6084
:1038B000D3F8FC2042F08072C3F8FC20084AC2F81A
:1038C000B01F116841F0010111601022DA7783F80E
:1038D0002200704700ED00E00003FA0555CEACC5AC
:1038E000001000E0202310B583F311880E4B5B68B5
:1038F00013F4006314D0F1EE103AEFF309844FF0A3
:103900008073683CE361094BDB6B236684F30988B1
:1039100000F0B4F810B1064BA36110BD054BFBE7F6
:1039200083F31188F9E700BF00ED00E000EF00E04D
:103930000B0700080E070008090100F1604301228F
:1039400003F56143C9B283F8001300F01F039A40E6
:1039500043099B0003F1604303F56143C3F88021F1
:103960001A607047024B0022C3E900339A60704727
:10397000A8480020002382680374054B1B689968DF
:103980009142FBD25A6803604260106058607047F1
:10399000A848002008B5202383F31188037C032B5B
:1039A00005D0042B0DD02BB983F3118808BD4369D2
:1039B00000221A604FF0FF334361FFF7DBFF002363
:1039C000F2E7D0E9003213605A60F3E7002382681F
:1039D0000374054B1B6899689142FBD85A680360D1
:1039E0004260106058607047A8480020054B196974
:1039F00008741868026853601A6018610123037420
:103A0000FCF76EBEA84800204B1C30B5044687B0BA
:103A10000A4D10D02B6901A8094A00F0FDF8204694
:103A2000FFF7E4FF049B13B101A800F031F92B6903
:103A3000586907B030BDFFF7D9FFF8E7A848002064
:103A40009539000838B50C4D044641612B698168F1
:103A50009A68914203D8BDE83840FFF78BBF1846FB
:103A6000FFF7B4FF01232C61014623742046BDE813
:103A70003840FCF735BE00BFA8480020044B1A6848
:103A80001B6990689B68984294BF00200120704792
:103A9000A848002010B5084C236820691A685460B3
:103AA0002260012223611A74FFF790FF014620690A
:103AB000BDE81040FCF714BEA848002008B5FFF789
:103AC000DDFF18B1BDE80840FFF7E4BF08BD000006
:103AD000FFF7E0BFFEE7000010B50C4CFFF742FF18
:103AE00000F08CF880220A49204600F03DF80123BE
:103AF00044F8180C0374FFF7CDFE002383F31188FC
:103B000062B60448BDE8104000F04EB8D04800202E
:103B1000C04C0008D04C000808B572B6034B586280
:103B200000F086FA00F054FBFEE700BFA848002032
:103B300000F0E8B8EFF3118020B9EFF305832022FD
:103B400082F311887047000010B530B9EFF3058497
:103B5000C4F3080414B180F3118810BDFFF7AEFF61
:103B600084F31188F9E70000826002220282704724
:103B70008368A3F17C0243F80C2C026943F83C2CC7
:103B8000426943F8382C074A43F81C2CC268A3F159
:103B9000180043F8102C022203F8082C002203F826
:103BA000072C7047F906000810B5202383F311880D
:103BB000FFF7DEFF00210446FFF744FF002383F3F5
:103BC0001188204610BD0000024B1B6958610F2070
:103BD000FFF70CBFA8480020202383F31188FFF7CC
:103BE000F3BF000008B50146202383F311880820A5
:103BF000FFF70AFF002383F3118808BD054B4FF040
:103C0000FF3103F11402C3E905220022C3E90712C0
:103C1000704700BFA848002070B51C4E05460C46F2
:103C2000C0E9032300F08AFB334653F8142F9A426D
:103C30000DD130620A2C2CBF00190A302A60C5E968
:103C40000124C6E90555BDE8704000F061BB316A4A
:103C5000431AE31838BF1C469368A34202D90819D7
:103C600000F066FB73699A6894420CD85A68AC609D
:103C70002B606A6015609A685D60121B9A604FF055
:103C8000FF33F36170BDA41A1B68ECE7A84800205D
:103C900038B51B4C636998420DD08168D0E9003279
:103CA00013605A600022C2609A680A449A604FF01A
:103CB000FF33E36138BD03682246002142F8143F18
:103CC00093425A60C16003D1BDE8384000F02ABB7E
:103CD0009A688168256A0A449A6000F02FFB63693C
:103CE000411B9A688A42E5D9AB181D1A206A092D32
:103CF00098BF01F10A02BDE83840104400F018BB3B
:103D0000A84800202DE9F041184C002704F11406C2
:103D1000656900F013FB236AAA68C11A8A4215D8A4
:103D20001344D5F80C802362D5E9003213605A6041
:103D30006369EF60B34201D100F0F4FA87F31188B0
:103D40002869C047202383F31188E1E76169B14204
:103D500009D013441B1ABDE8F0410A2B2CBFC01830
:103D60000A3000F0E5BABDE8F08100BFA8480020A5
:103D700000207047FEE70000704700004FF0FF3062
:103D800070470000BFF34F8F044B1A695107FCD1F5
:103D9000D3F810215207F8D1704700BF002000521D
:103DA00008B50D4B1B78ABB9FFF7ECFF0B4BDA688E
:103DB000D10704D50A4A5A6002F188325A60D3F812
:103DC0000C21D20706D5064AC3F8042102F1883235
:103DD000C3F8042108BD00BF604A00200020005243
:103DE0002301674508B5114B1B78F3B9104B1A69CD
:103DF000510703D5DA6842F04002DA60D3F81021A7
:103E0000520705D5D3F80C2142F04002C3F80C212B
:103E1000FFF7B8FF064BDA6842F00102DA60D3F828
:103E20000C2142F00102C3F80C2108BD604A0020B9
:103E3000002000520F289ABF00F580604004002047
:103E4000704700004FF400307047000010207047AA
:103E50000F2808B50BD8FFF7EDFF00F50033026817
:103E6000013204D104308342F9D1012008BD002081
:103E7000FCE700000F2870B5054645D8FFF75AFE4D
:103E8000224CFFF77FFF0646FFF78AFF4FF0FF3314
:103E9000072D6361C4F8143120D82361FFF772FF46
:103EA0002B0243F02403E360E36843F08003E36004
:103EB00023695A07FCD42846FFF764FF4FF400310A
:103EC000FFF7B8FF00F060F93046FFF78BFFFFF710
:103ED0003BFE2846BDE87040FFF7BABFC4F810317A
:103EE000FFF750FFA5F108031B0243F02403C4F8B9
:103EF0000C31D4F80C3143F08003C4F80C31D4F801
:103F000010315B07FBD4D6E7002070BD00200052C3
:103F10002DE9F84F40EA020305460C461746D8063D
:103F200002D00020BDE8F88F27F01F07DFF8D4B0DB
:103F3000FFF736FF2744BC4203D10120FFF752FFB1
:103F4000F0E720222946204600F088FD10B92035F0
:103F50002034F0E72B4605F120021E68711CE0D1E9
:103F600004339A42F9D1FFF7E5FD05F17843234A7E
:103F7000B3F5801F224B28BF9A4603F1040338BFD4
:103F80009046A2F1080228BF9846A3F108033ABF61
:103F90009146DA469946FFF7F5FEC8F80060A5EBB2
:103FA000040CD9F8002004F11C0142F00202C9F807
:103FB0000020221FDAF8006016F00506FAD152F848
:103FC000043F8A424CF80230F4D1BFF34F8FFFF721
:103FD000D9FE4FF0FF32C8F80020D9F8002022F0B7
:103FE0000202C9F80020FFF7AFFD20222146284633
:103FF00000F034FD0028AAD030469FE7142000527C
:10400000102100521020005210B5084C237828B11E
:104010001BB9FFF7C5FE0123237010BD002BFCD098
:104020002070BDE81040FFF7DDBE00BF604A0020F1
:1040300038B5054D00240334696855F80C0B00F0C1
:10404000B5F8122CF7D138BDE84C000870B5104E09
:1040500082B0FFF76FFD054600F070F93268034645
:104060009042336037BF0B4A0A495168146836BF23
:104070000131D1E9004151600419284641F10001A4
:104080000191FFF761FD2046019902B070BD00BFAC
:10409000644A0020684A002070B5124E82B0FFF7D3
:1040A00049FD054600F04AF9326803469042336004
:1040B00037BF0D4A0C495168146836BF0131D1E948
:1040C000004151600419284641F100010191FFF7B8
:1040D0003BFD4FF47A72002320460199FCF7E8F883
:1040E00002B070BD644A0020684A00200244074BB9
:1040F000D2B210B5904200D110BD441C00B253F8AA
:10410000200041F8040BE0B2F4E700BF5040005833
:104110000E4B30B51C6F240405D41C6F1C671C6F3C
:1041200044F400441C670A4C02442368D2B243F4AE
:1041300080732360074B904200D130BD441C51F87E
:10414000045B00B243F82050E0B2F4E700440258A8
:10415000004802585040005807B5012201A900202C
:10416000FFF7C4FF019803B05DF804FB13B50446E4
:10417000FFF7F2FFA04205D0012201A9002001941F
:10418000FFF7C6FF02B010BD0144BFF34F8F064BCF
:10419000884204D3BFF34F8FBFF36F8F7047C3F8CC
:1041A0005C022030F4E700BF00ED00E00144BFF303
:1041B0004F8F064B884204D3BFF34F8FBFF36F8FEF
:1041C0007047C3F870022030F4E700BF00ED00E054
:1041D00070470000074B45F255521A6002225A60A0
:1041E00040F6FF729A604CF6CC421A600122024BF4
:1041F0001A70704700480058744A0020034B1B781F
:104200001BB1034B4AF6AA221A607047744A002079
:1042100000480058034B1A681AB9034AD2F8D02450
:104220001A607047704A002000400258024B4FF459
:104230008032C3F8D02470470040025808B5FFF719
:10424000E9FF024B1868C0F3806008BD704A002087
:1042500070B5BFF34F8FBFF36F8F1A4A0021C2F8BA
:104260005012BFF34F8FBFF36F8F536943F4003386
:104270005361BFF34F8FBFF36F8FC2F88410BFF34A
:104280004F8FD2F8803043F6E074C3F3C900C3F314
:104290004E335B0103EA0406014646EA81750139A3
:1042A000C2F86052F9D2203B13F1200FF2D1BFF3D4
:1042B0004F8F536943F480335361BFF34F8FBFF384
:1042C0006F8F70BD00ED00E0FEE700000A4B0B4869
:1042D0000B4A90420BD30B4BC11EDA1C121A22F070
:1042E00003028B4238BF00220021FDF7C7B953F803
:1042F000041B40F8041BECE7F04E0008004B0020C4
:10430000004B0020004B00207047000000F0CCB8AC
:10431000034B002258631A610222DA60704700BF23
:10432000000C0040014B0022DA607047000C004096
:10433000014B5863704700BF000C0040014B586AA6
:10434000704700BF000C00404B6843608B6883607F
:10435000CB68C3600B6943614B6903628B6943623D
:104360000B6803607047000008B5364B40F2FF71E0
:104370003548D3F888200A43C3F88820D3F888202A
:1043800022F4FF6222F00702C3F88820D3F88820C5
:10439000D3F8E0200A43C3F8E020D3F808210A4309
:1043A000C3F80821294AD3F808311146FFF7CCFF9A
:1043B00000F5806002F11C01FFF7C6FF00F5806088
:1043C00002F13801FFF7C0FF00F5806002F15401EF
:1043D000FFF7BAFF00F5806002F17001FFF7B4FF4C
:1043E00000F5806002F18C01FFF7AEFF00F5806000
:1043F00002F1A801FFF7A8FF00F5806002F1C401F7
:10440000FFF7A2FF00F5806002F1E001FFF79CFFDB
:1044100000F5806002F1FC01FFF796FF02F58C7158
:1044200000F58060FFF790FF00F0F2F8084B0522DE
:10443000C3F898204FF06052C3F89C20054AC3F897
:10444000A02008BD0044025800000258304D00086A
:1044500000ED00E01F00080308B500F0C7FAFFF701
:104460003BFB0E4BD3F8DC2042F04002C3F8DC20CB
:10447000D3F8042122F04002C3F80421D3F8043118
:10448000074B1A6842F008021A601A6842F00402E8
:104490001A60BDE80840FFF7BDBE00BF00440258E7
:1044A0000018024870470000114BD3F8E82042F092
:1044B0000802C3F8E820D3F8102142F00802C3F83C
:1044C00010210C4AD3F81031D36B43F00803D363A7
:1044D000C722094B9A624FF0FF32DA6200229A61DA
:1044E0005A63DA605A6001225A611A60704700BF4D
:1044F000004402580010005C000C0040094A08B556
:104500001169D3680B40D9B29B076FEA01011161B1
:1045100007D5202383F31188FFF70AFB002383F3D9
:10452000118808BD000C0040384B4FF0FF31D3F824
:104530008020C3F88010D3F880200022C3F88020A8
:10454000D3F88000D3F88400C3F88410D3F8840033
:10455000C3F88420D3F88400D86F40F0FF4040F4C3
:10456000FF0040F43F5040F03F00D867D86F20F084
:10457000FF4020F4FF0020F43F5020F03F00D867B8
:10458000D86FD3F888006FEA40506FEA5050C3F8F4
:104590008800D3F88800C0F30A00C3F88800D3F875
:1045A0008800D3F89000C3F89010D3F89000C3F8B7
:1045B0009020D3F89000D3F89400C3F89410D3F867
:1045C0009400C3F89420D3F89400D3F89800C3F86B
:1045D0009810D3F89800C3F89820D3F89800D3F82F
:1045E0008C00C3F88C10D3F88C00C3F88C20D3F85F
:1045F0008C00D3F89C00C3F89C10D3F89C10C3F82F
:104600009C20D3F89C3000F0C9B900BF0044025888
:10461000614B0122C3F80821604BD3F8F42042F02B
:104620000202C3F8F420D3F81C2142F00202C3F8BE
:104630001C210422D3F81C31594BDA605A689104CA
:10464000FCD5584A1A6001229A60574ADA60002263
:104650001A614FF440429A61514B9A699204FCD519
:104660001A6842F480721A604C4B1A6F12F4407F41
:1046700004D04FF480321A6700221A671A6842F099
:1046800001021A60454B1A685007FCD500221A61D6
:104690001A6912F03802FBD1012119604FF08041F4
:1046A00059605A67414ADA62414A1A611A6842F40B
:1046B00080321A60394B1A689103FCD51A6842F4AB
:1046C00080521A601A689204FCD53A4A3A499A62B2
:1046D00000225A6319633949DA6399635A64384A84
:1046E0001A64384ADA621A6842F0A8521A602B4BF0
:1046F0001A6802F02852B2F1285FF9D148229A6173
:104700004FF48862DA6140221A622F4ADA644FF06D
:1047100080521A652D4A5A652D4A9A6532232D4AD0
:104720001360136803F00F03022BFAD11B4B1A69B5
:1047300042F003021A611A6902F03802182AFAD10B
:10474000D3F8DC2042F00052C3F8DC20D3F8042177
:1047500042F00052C3F80421D3F80421D3F8DC203E
:1047600042F08042C3F8DC20D3F8042142F08042BA
:10477000C3F80421D3F80421D3F8DC2042F000422E
:10478000C3F8DC20D3F8042142F00042C3F804212E
:10479000D3F80431704700BF008000510044025834
:1047A0000048025800C000F0040000010000FF01B2
:1047B0000088900832206000630209011D02040095
:1047C00047040508FD0BFF01200000200010E00059
:1047D00000010100002000524FF0B04208B5D2F8AD
:1047E000883003F00103C2F8883023B1044A13680B
:1047F0000BB150689847BDE80840FFF773B800BF99
:10480000784A00204FF0B04208B5D2F8883003F063
:104810000203C2F8883023B1044A93680BB1D06810
:104820009847BDE80840FFF75DB800BF784A002010
:104830004FF0B04208B5D2F8883003F00403C2F854
:10484000883023B1044A13690BB150699847BDE819
:104850000840FFF747B800BF784A00204FF0B04249
:1048600008B5D2F8883003F00803C2F8883023B1C5
:10487000044A93690BB1D0699847BDE80840FFF737
:1048800031B800BF784A00204FF0B04208B5D2F8E6
:10489000883003F01003C2F8883023B1044A136A49
:1048A0000BB1506A9847BDE80840FFF71BB800BF3E
:1048B000784A00204FF0B04310B5D3F8884004F494
:1048C0007872C3F88820A30604D5124A936A0BB104
:1048D000D06A9847600604D50E4A136B0BB1506B33
:1048E0009847210604D50B4A936B0BB1D06B9847C0
:1048F000E20504D5074A136C0BB1506C9847A30529
:1049000004D5044A936C0BB1D06C9847BDE81040B5
:10491000FEF7E8BF784A00204FF0B04310B5D3F857
:10492000884004F47C42C3F88820620504D5164A06
:10493000136D0BB1506D9847230504D5124A936D42
:104940000BB1D06D9847E00404D50F4A136E0BB13C
:10495000506E9847A10404D50B4A936E0BB1D06EEC
:104960009847620404D5084A136F0BB1506F9847FB
:10497000230404D5044A936F0BB1D06F9847BDE868
:104980001040FEF7AFBF00BF784A002008B5FFF720
:10499000B5FDBDE80840FEF7A5BF0000062108B53B
:1049A0000846FEF7C9FF06210720FEF7C5FF0621CE
:1049B0000820FEF7C1FF06210920FEF7BDFF0621F2
:1049C0000A20FEF7B9FF06211720FEF7B5FF0621E2
:1049D0002820FEF7B1FF09217A20FEF7ADFF07215D
:1049E0003220BDE80840FEF7A7BF000008B5FFF77A
:1049F0009BFD00F007F8FFF755FDBDE80840FFF705
:104A000085BC00000023054A19460133102BC2E97A
:104A1000001102F10802F8D1704700BF784A002067
:104A20000B460146184600F003B8000000F00EB82F
:104A300010B5054C13462CB10A4601460220AFF3CF
:104A4000008010BD2046FCE700000000024B01463C
:104A5000186800F035B800BF1C22002010B50139DD
:104A60000244904201D1002005E0037811F8014F83
:104A7000A34201D0181B10BD0130F2E72DE9F0412F
:104A8000A3B1C91A17780144044603F1FF3C8C42D4
:104A9000204601D9002009E00578BD4204F1010457
:104AA000F5D10CEB0405D618A54201D1BDE8F08183
:104AB00015F8018D16F801EDF045F5D0E7E7000097
:104AC00037B5002944D051F8043C0190002BA1F1E6
:104AD0000404B8BFE41800F047F81E4A01981368B0
:104AE00033B96360146003B0BDE8304000F042B8F1
:104AF000A34208D9256861198B4201BF19685B6818
:104B000049192160EDE71A465B680BB1A342FAD957
:104B100011685518A5420BD1246821445418A342AA
:104B20001160E0D11C685B68536021441160DAE7D2
:104B300002D90C230360D6E7256861198B4204BFB4
:104B400019685B68636004BF491921605460CAE753
:104B500003B030BDF84A0020034611F8012B03F8DA
:104B6000012B002AF9D17047014800F009B800BFB5
:104B7000FC4A0020014800F005B800BFFC4A0020B4
:104B80007047000070470000636F6D2E63756265AB
:104B900070696C6F742E68657265332B00000000BD
:104BA0004E6F20617070207369670A004261642053
:104BB0006677206C656E6774682025750A0042610F
:104BC0006420626F6172645F696420257520736878
:104BD0006F756C642062652025750A00426164204F
:104BE00066772064657363726970746F72206C6598
:104BF0006E6774682025750A0042616420617070D8
:104C000020435243203078253038783A30782530A8
:104C10003878203078253038783A30782530387830
:104C20000A00476F6F64206669726D776172650A6A
:104C30000040A2E4F16468910600000043414E4642
:104C40004449666163653A204D6573736167652009
:104C500052414D204F766572666C6F7721000000DF
:104C60004261642043414E496661636520696E6418
:104C700065782E0000000000000000005D1E0008A6
:104C800039170008652500082D170008A917000826
:104C9000B91B0008211900087117000875170008D2
:104CA000311700084D17000835170008791B000858
:104CB0005917000841260008651700084D1B000819
:104CC0006D61696E0000000069646C6500000000A1
:104CD000C84C0008E8480020604A0020010000009D
:104CE000D53A00080000000000000020000002008B
:104CF0000200000000010030000000000000000081
:104D0000000000240000080004000000000400006F
:104D100000FC0000020000000000043000800000E1
:104D20000000000000000038000001000100000049
:104D30000000002800000000AAAAAAAA000000247F
:104D4000FFFF000000000000000000000000050060
:104D500000000000AAAAAAAA00000000FFFE0000AE
:104D60000000000000000000000000000000000043
:104D7000AAAAAAAA00000000FFFF0000000000008D
:104D8000000000005A000000000000009AAAAAAA31
:104D900000000000F3FF0000990000000000000088
:104DA0000000000000000000AAAAAAAA000000005B
:104DB000FFFF0000000000000000000000000000F5
:104DC00000000000AAAAAAAA00000000FFFF00003D
:104DD00000000000000000000000000000000000D3
:104DE000AAAAAAAA00000000FFFF0000000000001D
:104DF000000000000000000000000000AAAAAAAA0B
:104E000000000000FFFF00000000000000000000A4
:104E10000000000000000000AAAAAAAA00000000EA
:104E2000FFFF000000000000000000000000000084
:104E300000000000AAAAAAAA00000000FFFF0000CC
:104E40000000000000000000000000000000000062
:104E5000AAAAAAAA00000000FFFF000000000000AC
:104E6000000000007CB4FF7F010000000000000093
:104E70001304000000000000000018000000000003
:104E800001000000FE2A0100D204000020220020C0
:104E90000000000000000000000000000000000012
:104EA0000000000000000000000000000000000002
:104EB00000000000000000000000000000000000F2
:104EC00000000000000000000000000000000000E2
:020000040803EF
:020000040804EE
:1000000000070030610904088D020508F5020408A4
:10001000150205080D020508110205086309040808
:10002000630904086309040863090408557D050889
:1000300063090408630904086309040863090408E0
:1000400063090408630904086309040863090408D0
:10005000630904086309040899B10508C5B10508D6
:10006000F1B105081DB2050849B20508197E050859
:10007000417E05086D7E0508997E0508C57E050848
:10008000ED7E0508197F05086309040859D704089F
:100090006309040869D704086309040875B20508F0
:1000A0006309040863090408630904086309040870
:1000B000630904086309040875B3050863090408A3
:1000C00063090408E534040863090408F184050899
:1000D000630904084DB3050861B305086309040802
:1000E000D9B2050863090408630904086309040810
:1000F000630904086309040863090408457F0508C7
:10010000630904086309040889B30508058505081F
:1001100063090408630904086309040863090408FF
:10012000717F0508997F0508C57F0508F17F0508DF
:100130001D800508630904086309040863090408AD
:1001400063090408630904086309040863090408CF
:1001500045800508718005089D800508630904082D
:1001600063090408630904086309040863090408AF
:10017000630904086309040863090408630904089F
:10018000630904086309040863090408630904088F
:10019000630904086309040863090408630904087F
:1001A000630904086309040863090408630904086F
:1001B000630904086309040863090408630904085F
:1001C000630904086309040863090408630904084F
:1001D000630904086309040863090408630904083F
:1001E000630904086309040863090408630904082F
:1001F000630904086309040863090408630904081F
:10020000630904086309040863090408630904080E
:1002100063090408630904086309040863090408FE
:1002200063090408630904086309040863090408EE
:1002300063090408630904086309040863090408DE
:1002400063090408630904086309040863090408CE
:1002500063090408630904086309040863090408BE
:1002600063090408630904086309040863090408AE
:10027000630904086309040863090408630904089E
:10028000630904086309040863090408630904088E
:10029000630904086309040863090408630904087E
:1002A000291D040811640408C1A6040879D70408AC
:1002B0006DDD04087DFD0408FD030508E52B050838
:1002C0003954050819590508000000000000000015
:1002D00040A2E4F164689106F22564CE19C94DD5B7
:1002E000508E0200F683B14A00001304FFFFFFFFA7
:1002F000FFFFFFFFEFF30383EFF30982EFF30881C2
:10030000DFF814D02DE9FE4F684600F0DBFEBDE8B3
:10031000FE4F8D4670470000C4290030F1EE101AE0
:10032000A0EC200A01607047A0EC108A704700BF63
:1003300080F0004002E000BF81F0004142001FBF9A
:100340005FEA410392EA030F7FEA226C7FEA236CA3
:100350006AD04FEA1262D2EB1363C1BFD218414098
:1003600048404140B8BF5B42192B88BF704710F02E
:10037000004F40F4000020F07F4018BF404211F0D1
:10038000004F41F4000121F07F4118BF494292EA39
:10039000030F3FD0A2F1010241FA03FC10EB0C0065
:1003A000C3F1200301FA03F100F0004302D54942F2
:1003B00060EB4000B0F5000F13D3B0F1807F06D39F
:1003C00040084FEA310102F10102FE2A51D2B1F197
:1003D000004F40EBC25008BF20F0010040EA03008C
:1003E0007047490040EB0000013A28BFB0F5000F0C
:1003F000EDD2B0FA80FCACF1080CB2EB0C0200FAC2
:100400000CF0AABF00EBC25052421843BCBFD04010
:100410001843704792F0000F81F4000106BF80F48A
:1004200000000132013BB5E74FEA41037FEA226C4D
:1004300018BF7FEA236C21D092EA030F04D092F018
:10044000000F08BF0846704790EA010F1CBF00204C
:10045000704712F07F4F04D1400028BF40F00040A9
:10046000704712F100723CBF00F50000704700F0C9
:10047000004343F0FE4040F4000070477FEA2262F0
:1004800016BF08467FEA23630146420206BF5FEAC1
:10049000412390EA010F40F4800070474FF00003C1
:1004A00004E000BF10F0004348BF40425FEA000C88
:1004B00008BF704743F0964301464FF000001CE030
:1004C00050EA010208BF70474FF000030AE000BF86
:1004D00050EA010208BF704711F0004302D54042C4
:1004E00061EB41015FEA010C02BF84460146002036
:1004F00043F0B64308BFA3F18053A3F50003BCFA51
:100500008CF2083AA3EBC25310DB01FA02FC6344FD
:1005100000FA02FCC2F12002BCF1004F20FA02F204
:1005200043EB020008BF20F00100704702F12002F7
:1005300001FA02FCC2F1200250EA4C0021FA02F258
:1005400043EB020008BF20EADC7070477BB972B948
:100550000029BEBF00204FF0004106E008BF002880
:100560001CBF6FF000414FF0FF3000F0F7B9ADF164
:10057000080C6DE904CE002909DB002B1ADB00F022
:1005800085F8DDF804E0DDE9022304B0704740425D
:1005900061EB4101002B1BDB00F078F8DDF804E093
:1005A000DDE9022304B0404261EB4101524263EBBA
:1005B00043037047524263EB430300F067F8DDF8F2
:1005C00004E0DDE9022304B0404261EB41017047E1
:1005D000524263EB430300F059F8DDF804E0DDE933
:1005E000022304B0524263EB4303704753B94AB944
:1005F000002908BF00281CBF4FF0FF314FF0FF302B
:1006000000F0ACB9ADF1080C6DE904CE00F03EF895
:10061000DDF804E0DDE9022304B0704708B50246C6
:100620000B4643EC172BB5EEC07BF1EE10FA03D46A
:10063000BDE8084000F00AB8B1EE477B51EC170B5B
:1006400000F004F8404261EB410108BD9FED0B6BE7
:1006500041EC170B9FED0B5B27EE066BBCEEC66BF8
:10066000B8EE464BA4EE457BFCEEC77B16EE101AA7
:1006700017EE900A704700BFAFF300800000000043
:100680000000F03D000000000000F0412DE9F047BF
:10069000089D04468E46002B4DD18A42944669D966
:1006A000B2FA82F252B101FA02F3C2F1200120FA49
:1006B00001F10CFA02FC41EA030E94404FEA1C4897
:1006C000210CBEFBF8F61FFA8CF708FB16E341EA93
:1006D000034306FB07F199420AD91CEB030306F119
:1006E000FF3080F01F81994240F21C81023E63443A
:1006F0005B1AA4B2B3FBF8F008FB103344EA0344DE
:1007000000FB07F7A7420AD91CEB040400F1FF33F2
:1007100080F00A81A74240F207816444023840EA2F
:100720000640E41B00261DB1D4400023C5E9004368
:100730003146BDE8F0878B4209D9002D00F0EF80EB
:100740000026C5E9000130463146BDE8F087B3FA1E
:1007500083F6002E4AD18B4202D3824200F2F98006
:10076000841A61EB030301209E46002DE0D0C5E909
:10077000004EDDE702B9FFDEB2FA82F2002A40F055
:100780009280A1EB0C014FEA1C471FFA8CFE012658
:10079000200CB1FBF7F307FB131140EA01410EFBFC
:1007A00003F0884208D91CEB010103F1FF3802D2A3
:1007B000884200F2CB804346091AA4B2B1FBF7F09D
:1007C00007FB101144EA01440EFB00FEA64508D9C0
:1007D0001CEB040400F1FF3102D2A64500F2BB80FD
:1007E0000846A4EB0E0440EA03409CE7C6F120074C
:1007F000B34022FA07FC4CEA030C20FA07F401FA92
:1008000006F31C43F9404FEA1C4900FA06F3B1FB1A
:10081000F9F8200C1FFA8CFE09FB181140EA01417F
:1008200008FB0EF0884202FA06F20BD91CEB01011C
:1008300008F1FF3A80F08880884240F28580A8F174
:1008400002086144091AA4B2B1FBF9F009FB1011C6
:1008500044EA014100FB0EFE8E4508D91CEB010164
:1008600000F1FF346CD28E456AD90238614440EA07
:100870000840A0FB0294A1EB0E01A142C846A64687
:1008800056D353D05DB1B3EB080261EB0E0101FA10
:1008900007F722FA06F3F1401F43C5E9007100266D
:1008A0003146BDE8F087C2F12003D8400CFA02FCC3
:1008B00021FA03F3914001434FEA1C471FFA8CFED3
:1008C000B3FBF7F007FB10360B0C43EA064300FBC3
:1008D0000EF69E4204FA02F408D91CEB030300F161
:1008E000FF382FD29E422DD9023863449B1B89B218
:1008F000B3FBF7F607FB163341EA034106FB0EF3A1
:100900008B4208D91CEB010106F1FF3816D28B424D
:1009100014D9023E6144C91A46EA004638E72E4619
:10092000284605E70646E3E61846F8E64B45A9D211
:10093000B9EB020864EB0C0E0138A3E74646EAE780
:10094000204694E74046D1E7D0467BE7023B61442E
:1009500032E7304609E76444023842E7704700BF97
:1009600002E000F000F8FEE772B63A4880F308882B
:10097000394880F3098839484EF60851CEF2000113
:10098000086040F20000CCF200004EF63471CEF266
:1009900000010860BFF34F8FBFF36F8F40F200007C
:1009A000C0F2F0004EF68851CEF200010860BFF3AD
:1009B0004F8FBFF36F8F4FF00000E1EE100A4EF63D
:1009C0003C71CEF200010860062080F31488BFF36A
:1009D0006F8F1AF017F91AF0B9F81AF09DF94FF065
:1009E00055301F491B4A91423CBF41F8040BFAE7BE
:1009F0001C49194A91423CBF41F8040BFAE71A49D5
:100A00001A4A1B4B9A423EBF51F8040B42F8040BA2
:100A1000F8E700201749184A91423CBF41F8040BFF
:100A2000FAE71AF0D1F81AF0EFF9144C144DAC4271
:100A300003DA54F8041B8847F9E701F065F9114C13
:100A4000114DAC4203DA54F8041B8847F9E71AF059
:100A5000B9B800000007003000230030000004088F
:100A600000010030000700308089060800230030B4
:100A7000D0270030D0270030E8FD0030A002040865
:100A8000C8020408C8020408C80204082DE9F04F8F
:100A90002DED108AC1F80CD0D0F80CD0BDEC108A26
:100AA000BDE8F08F002383F311882846A04700207B
:100AB00019F08AF9FEE719F041F800DFFEE70000BF
:100AC00081F0004102E000BF83F0004330B54FEAFF
:100AD00041044FEA430594EA050F08BF90EA020F6C
:100AE0001FBF54EA000C55EA020C7FEA645C7FEAFF
:100AF000655C00F0E2804FEA5454D4EB5555B8BF22
:100B00006D420CDD2C4480EA020281EA030382EA92
:100B1000000083EA010180EA020281EA0303362D24
:100B200088BF30BD11F0004F4FEA01314FF4801CF7
:100B30004CEA113102D0404261EB410113F0004F09
:100B40004FEA03334CEA133302D0524263EB4303C0
:100B500094EA050F00F0A780A4F10104D5F1200E5E
:100B60000DDB02FA0EFC22FA05F2801841F10001B9
:100B700003FA0EF2801843FA05F359410EE0A5F18D
:100B800020050EF1200E012A03FA0EFC28BF4CF0BE
:100B9000020C43FA05F3C01851EBE37101F0004574
:100BA00007D54FF0000EDCF1000C7EEB00006EEB81
:100BB0000101B1F5801F1BD3B1F5001F0CD349080B
:100BC0005FEA30004FEA3C0C04F101044FEA445262
:100BD00012F5800F80F09A80BCF1004F08BF5FEAE9
:100BE000500C50F1000041EB045141EA050130BDC9
:100BF0005FEA4C0C404141EB0101013C28BFB1F5DB
:100C0000801FE9D291F0000F04BF01460020B1FA25
:100C100081F308BF2033A3F10B03B3F120020CDAF8
:100C20000C3208DD02F1140CC2F10C0201FA0CF0D6
:100C300021FA02F10CE002F11402D8BFC2F1200C3B
:100C400001FA02F120FA0CFCDCBF41EA0C019040F1
:100C5000E41AA2BF01EB0451294330BD6FEA04043A
:100C60001F3C1CDA0C340EDC04F11404C4F1200225
:100C700020FA04F001FA02F340EA030021FA04F337
:100C800045EA030130BDC4F10C04C4F1200220FA8E
:100C900002F001FA04F340EA0300294630BD21FACC
:100CA00004F0294630BD94F0000F83F4801306BF92
:100CB00081F480110134013D4EE77FEA645C18BF86
:100CC0007FEA655C29D094EA050F08BF90EA020F1D
:100CD00005D054EA000C04BF1946104630BD91EA15
:100CE000030F1EBF0021002030BD5FEA545C05D118
:100CF0004000494128BF41F0004130BD14F5800457
:100D00003CBF01F5801130BD01F0004545F0FE41CA
:100D100041F470014FF0000030BD7FEA645C1ABFFF
:100D2000194610467FEA655C1CBF0B46024650EA36
:100D3000013406BF52EA033591EA030F41F4002162
:100D400030BD00BF90F0000F04BF0021704730B5E8
:100D50004FF4806404F132044FF000054FF00001BD
:100D600050E700BF90F0000F04BF0021704730B57E
:100D70004FF4806404F1320410F0004548BF404253
:100D80004FF000013EE700BF42004FEAE2014FEAA8
:100D900031014FEA02701FBF12F07F4393F07F4F83
:100DA00081F06051704732F07F4208BF704793F086
:100DB0007F4F04BF41F40021704730B54FF4607499
:100DC00001F0004521F000411CE700BF50EA01029C
:100DD00008BF704730B54FF000050AE050EA010245
:100DE00008BF704730B511F0004502D5404261EBB5
:100DF00041014FF4806404F132045FEA915C3FF4F6
:100E0000D8AE4FF003025FEADC0C18BF03325FEA92
:100E1000DC0C18BF033202EBDC02C2F1200300FA43
:100E200003FC20FA02F001FA03FE40EA0E0021FA68
:100E300002F11444BDE600BF10F8012B11F8013B8C
:100E4000012A28BF9A42F7D0D01A7047034613F8F8
:100E5000012B002AFBD1181A01387047C36A13F01E
:100E6000040F01D04068704700687047704700BFAA
:100E700010B5044608462160FFF7F0FFE060FFF779
:100E8000F5FF60600023A360204610BD0368DB6AA5
:100E900013F0100F0CBF01200020704738B5044636
:100EA000C5682035C560FFF7F1FF08B14835E5603A
:100EB0006368DB69DB0903F00403E2681343E36062
:100EC00038BD00BF4FF0E023D3F8880D00F4A00038
:100ED000B0F5A00F14BF00200120704710B50446E4
:100EE000FFF7F0FF18B1A36843F00103A36010BD42
:100EF00000F47F40B0F53E4F14BF00200120704742
:100F000010B5044643689869FFF7B0FF0088FFF703
:100F1000EFFF206110BD00BF014B024A1A6070470D
:100F2000D0270030ED55CEAC4FF0E023D3F8000DC4
:100F300000F47020B0F5402F14BF0020012070474E
:100F400003691BB14268936902339361704700BF24
:100F500008B504220121024800F080FB08BD00BF53
:100F6000F4F2050808B504220121083000F076FBF0
:100F700008BD00BF08B510220121406800F06EFBDB
:100F800008BD00BF08B50068202201210C3000F028
:100F900065FB08BD08B5406804220121103000F04F
:100FA0005DFB08BD08B5042201210C3000F056FBA2
:100FB00008BD00BF08B540680C220121143000F0C4
:100FC0004DFB08BD08B50C220121006800F046FB6E
:100FD00008BD00BF38B5044610E0082201212046B4
:100FE00000F03CFB25682846FFF740FF217A626845
:100FF000521BB2FBF1F200F031FB0C341CB1236840
:10100000B3F1FF3FE9D138BD00B587B0094B00937C
:101010001433019304238DF808304FF0FF3303930A
:10102000049301238DF814306846FFF7D3FF07B00F
:101030005DF804FB28ED00E0094B1A68094B9A4261
:1010400000D1704700B583B0074B01930422012102
:101050000DEB020000F002FB03B05DF804FB00BFE3
:10106000D0270030ED55CEACACCE55ED70B5A2B06A
:101070000446FFF70BFF08B311A8FFF755F96668A0
:1010800006F1200C01AD6036AE46DCF80000DCF85D
:101090000410DCF80820DCF80C30AEE80F000CF18E
:1010A000100C7546B445EFD163681B6E2193842202
:1010B000012101A800F0D2FA22B070BD01A8FFF70B
:1010C0002DF9F4E700B587B0014601A8FFF7D0FE7F
:1010D00001A8FFF7E3FE01A8FFF700FF01A8FFF753
:1010E0000FFF08E001A8FFF7C1FF24E0FFF7A4FF0E
:1010F00000F028FA50BBFFF70FFF04A800F0ACF98E
:10110000FFF726FF01A8FFF72DFF01A8FFF732FF29
:1011100001A8FFF737FF01A8FFF73CFF01A8FFF781
:1011200041FF01A8FFF746FF01A8FFF74BFF039B14
:1011300013F0010FD6D100F07DF8FFF74BFFFFF75A
:10114000F3FE0028D2D1FFF75FFFCFE701A8FFF73A
:10115000F7FE07B05DF804FB08B5252017F086FE02
:10116000144BD3F8982042F01002C3F89820D3F81B
:10117000982022F01002C3F89820D3F89820D3F8D2
:10118000F02042F01002C3F8F020D3F8182142F00A
:101190001002C3F818216D22D3F81831064BDA601B
:1011A0004FF0FF321A620D221A600122034B1A70AF
:1011B00008BD00BF0044025800100140FC29003067
:1011C00037B50E4D2A78202A15D10D4C0D482368CD
:1011D0000D491844019219F04BF823680021019A37
:1011E00020330948297023601AF0E6FE03B0BDE8F9
:1011F000304019F075BC03B030BD00BFC4290030C9
:10120000EC290030608E0608C6290030074900220C
:10121000074B5B1A9A4201D30120704751F8040B27
:10122000013001D10432F5E700207047608E0608D6
:10123000000018085A4B2DE9F74F1F680224594B3C
:1012400007F56A57DFF880911B781837DFF87C8143
:10125000554D1F44DFF878A118F062FBA9EB080B8D
:1012600006460EB13A2C41D9A9EB0803B3EB070CA3
:1012700024D4DFF860E1661C4C4A0C21F6B2AEEBD8
:101280000200614360456FDD681801276A506244BF
:1012900007721F464260DB1B77D445490234454F35
:1012A000E4B2CA1B9A424FF00C0206FB02F266DD62
:1012B000A91801203B44AF5008724B603B2C66D804
:1012C0000C2301225C432B191A724FF0FF322A5172
:1012D0005A60394B1B782BB1384B1B682B60384B4D
:1012E0001B686B60304803B0BDE8F08FF369B069EC
:1012F00053450ABF334BF31AA3EB0A0380B10193A2
:1013000019F074F9019B58B122460C2101344A436B
:101310000121E4B2A8180172B169A9500D314160F0
:101320000C2001211F4400FB04FC5F4505EB0C026F
:1013300045F80C6006F1380C1172C2F804C004EBD9
:10134000010204F10204D2B2E4B200FB02F205EBA6
:1013500002000172F169A95019444160AED23046D1
:1013600018F0EEFA06467CE705EB010C4FF0010899
:1013700007446A508CF80880CCF804E08BE7AB187F
:101380000120AF501872596098E7344696E7012360
:1013900085F8CC324FF0FF33C5E9B13399E700BF90
:1013A000EC290030C429003004230030D02700305D
:1013B00000000430E8FD003000230030F029003048
:1013C000E82900300023003000001808608E06086D
:1013D00000070030E8FD00300C4B1B7810B50BB94E
:1013E000FFF7BAFE00230A490A48CA699206FCD5EB
:1013F0004A6A1C5CD2B2944205D10133DBB20E2B97
:10140000F3D1002010BD0023EFE700BFFC2900301E
:1014100000100140F8F2050838B5084B04461B7867
:101420000BB9FFF799FEE4B2054DAC62EB695B06C0
:1014300000D538BD19F054FBF8E700BFFC29003097
:101440000010014010B5441E14F8010F00B910BD82
:10145000FFF7E2FFF8E7000070B502680446EFF31B
:101460000581D9205369C9B20EF0D6FE294B1B78ED
:10147000A3B1294B94E8030083E803002748FFF752
:10148000E1FF6368B3B12648FFF7DCFF2548FFF7AB
:10149000D9FFFFF7A1FF2448FFF7D4FF234D2B7896
:1014A0003BB124681CB1204619F0A0F820B90023F4
:1014B0002B7070BD1E48E7E720461E4E19F0AAF8B3
:1014C00000F2145084421FD2204619F0A3F8306075
:1014D0002046194E19F0B2F804F5E053834217D9AB
:1014E000204619F0ABF830600023144A1360144A08
:1014F0001370FFF78BFE0028D9D019F0F1FA012004
:10150000BDE8704018F030BFA4F214533360DFE739
:101510003360E9E7C5290030F429003008F30508F5
:101520000DF305081EF30508F0F805080023003048
:1015300018F30508F0290030E8290030EC290030C4
:10154000C4290030284B1A7870B542B12748FFF7FC
:1015500079FF274B5868003818BF012070BD254A15
:10156000107800283CD0244E244C33682448254D64
:101570001A1D21782D1A0A44AA4205D3224A4FF097
:10158000FF31D161202222702278D2B103F12001F3
:101590008D4205D81F2A9FBF1B4AD361202222708B
:1015A00020221949184418F063FE3268237800217C
:1015B000154813442022217033601AF0FDFC19F005
:1015C0008FFA33689D4207D90F4920220F48CB611B
:1015D00018F04EFE19F084FA002018F0C5FEB8E7A6
:1015E00001221A70BAE700BFC529003064F305086C
:1015F000F429003000230030EC290030C4290030E9
:10160000608E060800001808C6290030E0FF1708A1
:101610002DE9F84307460E460024DFF83890DFF83E
:101620003880B44201D1BDE8F88324B1230702D148
:101630004846FFF707FF3D5D01342B0905F00F0514
:1016400018F80300FFF7E8FE18F80500FFF7E4FEBE
:10165000E7E700BFF0F8050874F30508474B1B786F
:101660002DE9F74F07460E4690465BB1022925D07B
:10167000042938D0012902D11146FFF7C9FF40489B
:10168000FFF7E0FE3F4B1B78002B4ED03E4A002573
:101690003E4BA2EB030938E037F81430ADF80430C4
:1016A00024B1620702D12846FFF7CCFE01340221A3
:1016B00001A8FFF7ADFFA045EED1E0E70024304DD3
:1016C000F9E757F82430019324B1A30702D1284643
:1016D000FFF7B8FE042101340DEB0100FFF798FF7E
:1016E000A045EED1CBE70024254DF9E7FFF768FDD3
:1016F000022E1DD0042E2CD0012E06D12378795D28
:101700005A1C2270224AD1540135A8450DD0214BD4
:10171000214C1B682278043313444B45E6D31C4B01
:101720004FF0FF32DA612023237003B0BDE8F08F61
:101730002378DFF85CA05A1C22703A780AF803205C
:10174000FFF73EFD23785A1C227000220AF803207E
:10175000DAE74FF0000ADFF838B022783B78511C06
:1017600023FA0AF30AF1080A21700BF80230FFF796
:1017700027FDBAF1200FF0D1C6E700BFC529003020
:10178000F0F805080023003000001808608E0608F5
:10179000C6290030EC290030C42900307047000011
:1017A00070B504461C3008F089F9182604F1400091
:1017B00004F028FF04F5D87008F0BCFB04F53E7077
:1017C00008F0BCFE04F5537008F086FF01220023E8
:1017D0001B4904F56E70C4E9E8230023194A84F814
:1017E000B03311609DB201332A4672438A5C002AED
:1017F000F8D1154B1D80154B1A6812B114480EF024
:1018000049FD186004F57E70124BC4F8EC330CF0FF
:1018100039F8114B64224FF4FA71C4F8103404F211
:10182000144304F58460C4F8143408F033FB0B4B04
:101830001A680AB10A48E2E720461C6070BD00BF82
:10184000ECF40508C43E0030C03E0030843E003059
:1018500088F3050894F8050894340608002A003037
:10186000A3F30508082906D1084B09211B68586C09
:1018700003681B6918470A2906D1044B07211B6816
:10188000586C03681B69F5E7704700BF282A0030D1
:10189000FFF7E8BF2DE9F041534D88B0044619F039
:1018A0000BF919F01DF90021286801F067FF0368A2
:1018B0004FF4E131DE6A20231A46B047032128683D
:1018C00001F05CFF036880224FF4E131DE6A4FF4DF
:1018D0008073B047204604F11C0600F049FA19F065
:1018E000FFF8204601F036FC304608F0EDF919F01B
:1018F000F7F800233D481A4619460093CDE9013315
:101900000CF030F82B68586D03685B68984710B18D
:1019100037480CF027F894F9403063B394F9183045
:101920004BBB314604F1400004F0B8FE04F57B7671
:1019300004F58261304601F003FF0121304601F0D9
:10194000D9FE204601F06AFC04F5D87008F0FCFBD3
:101950002B68D86C03681B6898472B68D86C0368A1
:101960001B6D984704F5537008F0D6FF08B0BDE82A
:10197000F0410EF0C5BC2B68002208211D4F586CA9
:10198000032603685B6A98472B6801220721586C7D
:1019900003685B6A98472B6800220A21586C036829
:1019A0005B6A98472B6801220921586C03685B6ABF
:1019B00098472B6822460821586C049403680597C1
:1019C000D3F82C803B460096C0472B680A21586C00
:1019D0000368D3F82C8008AB0096CDE9064713E9DD
:1019E0000C00C047A2E700BF282A0030C4F3050856
:1019F000EBF30508911804080148FFF74BBF00BF3F
:101A0000302A0030F0B52DED028B90F8B0338BB05A
:101A1000002B54D12C4E0EF073FC02463368C31ACF
:101A2000632B4CD9294B04AD03F118071868083310
:101A300053F8041C2C46BB4203C42546F6D10024AF
:101A4000234D9FED248A32602B780AAA2344013467
:101A500003F0070303EB4303134413F8162C07EEBC
:101A6000902A13F8172C13F8183CF8EEE77A67EE73
:101A7000887AFCEEE77ACDED017A07EE902A9DF8A0
:101A80000420F8EEE77A67EE887AFCEEE77ACDED8F
:101A9000027A07EE903A9DF808100023F8EEE77AF4
:101AA00067EE887AFCEEE77ACDED037A9DF80C00BC
:101AB00008F060FF042CC7D12B7801332B700BB0DA
:101AC000BDEC028BF0BD00BF042A0030FCF105081C
:101AD000082A00309A99993E2DE9F341144C154E8D
:101AE0002046DFF8608018F00BFF134A01461348C8
:101AF000121B134F01F004F917F012FF0446A4B1B2
:101B0000E069A169B042019114BF251AA8EB06054E
:101B100018F0F6FE019902462B46384601F0F0F81F
:101B2000204617F00DFF0446E9E702B0BDE8F0815A
:101B300000010030000700300007003008F40508FD
:101B400012F405080023003008B590F8483363B15B
:101B5000002380F8483308F015FD08F08BFD08F0ED
:101B600093FBBDE8084008F08DBD08BD10B5094CD9
:101B700003F07EFD002105222368186D0368DB69F0
:101B8000984723682821186D0368BDE810405B68FA
:101B9000184700BF282A003070B504460EF0B0FB8D
:101BA0004E4A05461368C31AB3F57A7F02D910600E
:101BB00008F044FC08F000FB494A41F28831136800
:101BC000EB1A8B4206D9016821B11560028945489C
:101BD00001F096F894F90930012B0AD1424A41F2FA
:101BE00088311368EB1A8B4203D920461560FFF742
:101BF00073FF3E4A1368EB1A132B04D904F5537094
:101C0000156008F09DFE2046394D01F0B7F894F8B4
:101C1000E833002B32D02B7843B994F91830002BDD
:101C200034D12046BDE87040FFF7ECBE314E642150
:101C30003368186D03681B69984794F918309FED55
:101C40002E7A2046013B07EE903A0123F8EEE77A20
:101C500000F8183FF0EEE77AF4EEC77AF1EE10FAEA
:101C60004CBF1946002103F0A3FC2046FFF77EFF7E
:101C700033680021186D03689B6B98472B78002B05
:101C8000CBD094F91830002BCBD070BD194E642105
:101C900000253368186D03681B69984794F918305C
:101CA0009FED157A204607EE903A00F8185FF8EE9F
:101CB000E77AF0EEE77AF4EEC77AF1EE10FA4CBF6D
:101CC0000121294603F074FC2046FFF74FFF3368DB
:101CD0002946186D03689B6B9847D2E70C2A0030A1
:101CE000142A003024F40508102A0030182A003085
:101CF000D4250030282A0030000000340148FFF7C6
:101D00004BBF00BF302A003038B5054B0A460146AC
:101D10001C68236820461D68024BA847002038BD78
:101D2000282A00301C2A003010B50A4C2046FFF744
:101D300037FD094A0949204619F074FB0CF006F8F2
:101D4000074B084A186008490848BDE8104001F0F0
:101D50000DBD00BF302A0030E4CC00309D170408D0
:101D6000282A0030FD1C0408F91904081C2A003038
:101D700010B5044604F0B4F903F0A8F948B9184BBB
:101D800018491B68186C03681B68984716480EF0C2
:101D900081FA204604F002F918B1B4F90030022BA0
:101DA0001AD004F06BFB02F041FEB4F900309FED55
:101DB0000F7A2046023B07EE903A0223F8EEE77ACC
:101DC0002380F0EEE77AF4EEC77AF1EE10FA4CBF1A
:101DD0000121002103F0ECFBBDE8104004F070B8D5
:101DE000282A003034F4050849F4050800000034BE
:101DF000BFF34F8F0549064BCA6802F4E0621343F4
:101E0000CB60BFF34F8F00BFFDE700BF00ED00E0E8
:101E10000400FA05102213B5002104468DF80720AE
:101E20001AF0CAF8054B0DF1070221461B68586DE0
:101E300003685B6B984702B010BD00BF282A0030D2
:101E40002DE9F041ADF54A7D0D46002140F27512B5
:101E500068AC06460AA809911AF0AEF84FF4C472AD
:101E6000002120461AF0A8F8DFF808810EF048FAA1
:101E70004FF47A72384B09AFB0FBF2F0186093E878
:101E8000070084E8070001F091FB037C237401F054
:101E90008DFB437C0DF5E17063740323A3742F4B1A
:101EA0005A6962619A68DB68A261E361FFF7B2FF79
:101EB00041F20433D8F80C202384002A284B1868F8
:101EC000284B3ADD0DF2D321CDE90032264B5022CA
:101ED000406D01F043FD50210DF2D3201AF0F4FBC8
:101EE00098F91020394684F83201013A204618BF8B
:101EF000012215F023FC98F9103080B2E97E5A1EB9
:101F000053425341069300230393AB7E029305F1A2
:101F1000190301930123CDE90470009330460CA30B
:101F2000D3E9002314F0DAFC011E02DC0F480BF0A9
:101F300019FD0DF54A7DBDE8F081009350220C4B50
:101F40000DF2D321406D01F009FDC4E7AFF300802D
:101F50009E6AC421818A46EE742E0030D0020408A5
:101F6000282A00305BF6050854F6050870F60508C7
:101F7000F1200608302A00302DE9F043274D95B0B6
:101F8000D5F8D83F002B3CD02F1D0026DFF89480D9
:101F9000384614F0EDFC044698B34022002103A813
:101FA0000296ADF84C601AF007F894F8440001F07E
:101FB0005DFB211D8DF84C0003A894F8442019F016
:101FC000EDFF236843F00043029394F845308DF809
:101FD0004D300EF097F9D5F8D84F10EB0802236872
:101FE00020460096D3F8109041F1000302A9C8479B
:101FF00000280DDC95F8D53F072B05D9084814F0CB
:10200000BBFC15B0BDE8F083013385F8D53FF8E798
:10201000384614F0B1FC85F8D56FB9E7802E003052
:10202000842E003040420F002DE9F041DC220C46A6
:10203000CAB005460021444819F0BEFF4FF0405396
:10204000424A1A60A38A013B9BB2C92B73D8404B0A
:1020500000260822204600930023194614F0D0FCE5
:10206000721CF3B2D1001646A28A013A934209DAF1
:1020700003F140530822204616330093002314F046
:10208000BFFCEDE74FF040531A7D0AB9E27E1A75A6
:102090002846002614F0CAFB4FF0405331467D22FB
:1020A000587509A8DFF8B08008AF089619F084FFCA
:1020B0003146812229A819F07FFF98F9102039466E
:1020C00029A8013A18BF012215F092FC98F91030A6
:1020D00080B203965A1E1F4E53425341CDE90470FD
:1020E00006932846A37E029304F119030193282343
:1020F0000093E17E332412A3D3E9002314F0EEFB16
:10210000013C14F0FF0408D0FFF736FF33680121CB
:10211000186D03685B689847F2E70F48FFF726FDE4
:10212000284614F083FB40F0304040F4002018F0C3
:1021300073FBFFF75DFE4AB0BDE8F081AFF30080AE
:1021400026417272DF25D7B7040000309AAD44C52E
:1021500014000030282A0030302A003070B50D46B7
:1021600014461E4614F062FB50B9022E07D1012C12
:1021700005D12AA3D3E900230120C5E9002370BDBE
:10218000282C29D00DD8601E83B20A2B16D80A2815
:1021900014D8DFE800F01D13133925131313132D82
:1021A000290040F24C439C4226D009D840F22643F5
:1021B0009C422DD040F239439C4221D00020DEE7E2
:1021C00044F627639C42F9D116A3D3E90023D3E751
:1021D00016A3D3E90023CFE716A3D3E90023CBE767
:1021E00016A3D3E90023C7E716A3D3E90023C3E767
:1021F00016A3D3E90023BFE716A3D3E90023BBE767
:1022000016A3D3E90023B7E716A3D3E90023B3E766
:1022100016A3D3E90023AFE7AFF30080401DA12050
:1022200026812A0BECFD51169C2A1F639E6AC4214D
:10223000818A46EE26417272DF25D7B7F017304A01
:1022400039059E56D5A4D139F922B6A7CDD269EB6E
:10225000C51A133B03806A5575F30087C41EDD8BD6
:102260003CD93120DBC293A716112720011517CBCB
:102270000E03561F2DE9F047DFF89CA086B00546F7
:102280000F460AF104001646984614F0CFFA70B3D0
:10229000DAF8CC4F45EA064964B32368994511D072
:1022A000A246A468002CF8D10C21012018F03AF9BC
:1022B000CAF80800D8B1C0F80090DAF808309C607D
:1022C000DAF808400434124B124893F910300096A3
:1022D0005A1E534253412A460593BDF83830CDE982
:1022E00003831823CDE901433B4614F0A1FA06B05D
:1022F000BDE8F0870C21012018F014F9CAF8CC0FC2
:102300000028F4D08460041DC0F80090DBE700BF13
:10231000302A0030842E0030802E003010B5C4B03A
:10232000694614F061FFE8B9BDF800300E4CB3F512
:10233000007F0FD1BDF802309FED0C7A07EE903A86
:10234000F8EE677A67EE877A9FED097A67EE877A0B
:10235000C4EDEA7ADDE94223C4E9E8230DF0CCFFBD
:10236000C4F8AC0344B010BD302A00300AD7233C77
:1023700035FA8E3C2DE9F0410D46ADF5876D0646E8
:1023800018F0AEFB0AA9284615F08CFB044600287D
:1023900040F0B2804FF4D0720146A6A819F00CFEAE
:1023A0009DF8C020102A7BD8531E0F2B1FD80DF18B
:1023B000C1010DF2D93019F0F1FD22460DF12701CE
:1023C0000DF2D93003F068F80446002C68D09DF86F
:1023D000C03063B39DF8301049B39DF82730013BFE
:1023E000032B00F28980DFE803F0162B353D49AA64
:1023F0000DF12701BDF82800499403F083FB044642
:1024000000284DD001230DF2D93249A900931123A0
:1024100002F082FFD9E701296ED19DF9383094F995
:1024200000209A422DD02370204603F0C1F89DF879
:102430002730013B032B5FD8DFE803F02362686D90
:10244000012959D1BDF93830B4F900209A4257D04A
:102450002380E9E701294FD10E9B2268934255D092
:102460002360E1E7022947D1DDED0E7A94ED007A91
:10247000F4EE477AF1EE10FA4DD00121C4ED007A66
:10248000D2E701238DF8983294F90030DA17CDE9BC
:10249000A8325C210DF2D9301AF016F98DF8D80364
:1024A0000024DFF8888040F26F124AA82146499440
:1024B00019F082FD98F9102049AFA6A8013A3946D3
:1024C00018BF012215F0F8FB98F9103080B2E97EB0
:1024D0005A1E0394534253410693AB7E029305F177
:1024E000190301930B23CDE90470009330460DA32B
:1024F000D3E9002314F0F2F90DF5876DBDE8F08102
:1025000001238DF89832B4F90030BFE701238DF82C
:1025100098322368BAE702238DF898322368A8938B
:10252000B7E700BFD5A4D139F922B6A7302A0030C9
:102530002DE9F0432DED028BB1B005460C4614F0A9
:1025400075F98046002858D1237E022B1FD1E38ADB
:10255000012B1CD1BE4E331D9D4218D10DF0D0FE73
:10256000074601F0B7FE03464FF4C87007F516772B
:10257000B3FBF0F202FB103317FA83F3C6F8D03F37
:10258000E77E4FB9B3480BF0EDF986F8D47F31B050
:10259000BDEC028BBDE8F0830EA9204615F0ECF9E6
:1025A0000AA8FFF737FC9DF83A400AA90DF13B0055
:1025B000224619F0E3FC28B1A7480BF0D3F986F8BE
:1025C000D48FE4E70F2C0CD8D6F8D03F214686F8FC
:1025D000D44FA3F51673A148C6F8D03F0BF0C2F94B
:1025E000D5E79DF83810284614F018F99DF83820E2
:1025F00031789B480BF0B6F9C9E7E38A282B00F045
:10260000B3801FD8013B9AB20A2AC0D80A2BBED881
:1026100001A252F823F000BF572704088F250408B1
:102620008F250408CD2804087B2704088F2504087B
:102630008F2504088F2504088F250408AB2704087C
:102640009927040840F24C42934200F01B8175D850
:1026500040F22642934200F0298140F239429342EF
:1026600095D1DFF80C8201230EA9204688F8B033FB
:1026700015F01AF800288AD1074608F55379DFEDDE
:10268000798A9DF83820FBB29A4280D930AA484610
:1026900002EB830313F8864C13F8855C13F8846C03
:1026A000E400AD00F60008F08BF96428E4B205F010
:1026B000F805F6B237D0002835DB07EE900AFF2286
:1026C0000021B8EEE78A07EE904AF8EEE77A28EEA6
:1026D000288A67EE887AFDEEE77A17EE903A18B20C
:1026E00001F0F0FD07EE905AFF220021F8EEE77AA4
:1026F000C4B267EE887AFDEEE77A17EE903A18B228
:1027000001F0E0FD07EE906AC5B2FF22F8EEE77A2D
:10271000002127EE888ABDEEC88A18EE103A18B25A
:1027200001F0D0FDC6B2002332462946204608F00B
:1027300021F901231F4488F84833A2E744F62762B1
:1027400093427FF424AF204631B0BDEC028BBDE84C
:10275000F043FFF7E3BD2146284631B0BDEC028BC4
:10276000BDE8F043FFF76CBB2146284631B0BDEC15
:10277000028BBDE8F043FFF757BC3B480BF0F2F883
:102780003A4B0A211B68186D03685B689847384804
:10279000FFF7ECF9FFF72CFB2146284631B0BDECE2
:1027A000028BBDE8F043FFF7E5BD0AA9204615F00E
:1027B0004BF900287FF4EBAE9DF82830012B0FD1A8
:1027C00003F05CFE02F032F903F07AFB03F088FCC0
:1027D0002849294803F068FC2849294803F064FC8B
:1027E000DFF88C80102200210EA819F0E5FB0123F0
:1027F00098F9102008AF00260EA8D21A39468DF895
:10280000403018BF01220896ADF824608DF826608C
:1028100015F032F998F9103080B20396591E4B42E8
:102820004B41CDE9047006932846A37E029304F140
:10283000190301930A230093E17E03A3D3E9002344
:1028400014F04CF8A3E600BFCDD269EBC51A133BD8
:10285000802E003098F60508C3F60508E4F6050852
:1028600006F705080AD7233C22F70508282A003076
:10287000302A0030A81A0608702A0030C42506083D
:10288000E02B00300EA9204614F04AFF00287FF408
:102890007EAE1C4B9DF838101B68A1F1FF02586DED
:1028A0005142036851411B68984770E60EA92046C3
:1028B00014F096FE014600287FF469AE9DF8393089
:1028C0000DF13A02104804F0C1FA60E60EA9204664
:1028D00014F0D8FF00287FF45AAE0C4DD5E9F4234C
:1028E00052EA030109D0DDE90E01CDE9000105F549
:1028F000846007F0D3FAC5E9F601D4E90023C5E9FD
:10290000F42344E6282A0030702A0030302A0030B0
:10291000F0B500F140050446ADF5277D284604F0EA
:102920003DFA94F84861D4F8C02304EB0613D3F8B9
:102930008C309A4200F03481C4F8C0334FF4D07226
:1029400000213EA819F038FB94F8AA3133B9A82326
:1029500003FB064393F89930012B0CD894F81874B4
:102960004FB90DF0CBFC00220023CDE93E01CDE9AB
:102970004023002313E001233146284684F818340D
:1029800003F01EFFCDE93E0194F84811284603F0FC
:1029900087FF50EA0103CDE94001EAD002238DF818
:1029A0000831A8230A2203FB064103FB0656D1F88F
:1029B000B0008C3680FB0207CDE94407D1F8AC00AB
:1029C00080FB0207CDE94607D1F8A8004243CDE9D4
:1029D0004822D1F8CC2094F848114A92726803FB3F
:1029E00001434B92B2684C9293F8CA208DF834217F
:1029F00093F8992094F8AA3153B9062A0DD8DFE844
:102A000012F007000700D200D600D800DE00E30075
:102A100000238DF83531ADF83631062303AA284658
:102A20008DF8383103F0B0FE38B1DDED037A67EE92
:102A3000A77ACDED507ACDED4F7A04AA94F84811DB
:102A4000284603F0AFFE28B1DDED047A67EEA77AE1
:102A5000CDED517A05AA94F84811284603F086FE78
:102A600048B1DDED057A67EEA77ACDED547ACDED6C
:102A7000537ACDED527A00265D4FDA2207A831460F
:102A8000069619F099FA97F9102006A93EA8013A7E
:102A900018BF012214F09AFC06AB80B240F2274224
:102AA00000904DA1D1E90001FFF7E4FB202231465F
:102AB0003EA819F081FA94F84831A822DFED4D6A5A
:102AC00006A93EA802FB0343B3F8C620B3F8C830FA
:102AD00007EE102A97F9102007EE903AB8EEC77A61
:102AE000013AF8EEE77A18BF012227EE267A67EE60
:102AF000A67A8DED407ACDED417ACDE90666CDE935
:102B0000086614F0EDFB06AB80B240F2254200905F
:102B100033A1D1E90001FFF7ADFB94F84811284635
:102B20004096CDE93E6604F04DFA94F94E308DF8AA
:102B3000FC003BB1284604F073FA18B9409B43F0FF
:102B4000010340939DF8FC3043B104A9284604F0EA
:102B500069F918B9409B43F00203409305AA94F821
:102B60004811284604F06CFA08B1059B3E9397F98A
:102B70001020002306A93EA8013A0693ADF81C30A8
:102B800018BF01228DF81E3014F012FB06AB80B284
:102B900044F62362009014A1D1E90001FFF76AFB1B
:102BA0000DF5277DF0BD02228DF8352133E7032294
:102BB000FAE703238DF8353140F201132BE70323A5
:102BC0008DF83531022326E703238DF835314FF494
:102BD000817320E7AFF300805F43370F00E741CAFE
:102BE000D2BFDBC3C4BDE89B697F00BBABB43CBABA
:102BF000302A00300AD7233C10B590F8441104461F
:102C000007F0F2F97C23C0B203FB0044D4F8900033
:102C100010BD000070B590F9C53196B00446002B88
:102C20005CD090F8F332002B58D000F5D8752846C8
:102C300007F0ECF9D4F8BC632846FFF7DDFF8642C5
:102C40004CD094F8F412284607F0CEF97C26C0B296
:102C500006FB004090F8E131002B3FD02846FFF7FB
:102C6000CBFF94F8F412C4F8BC03284607F0BCF973
:102C70002822C5B200210CA819F09EF906FB0543D5
:102C80009FED1A7A0021D3ED8D7A152203A80291C7
:102C900067EE877ACDED097AD3ED8E7A67EE877A83
:102CA000CDED0A7AD3ED8F7A67EE877ACDED0B7A88
:102CB00019F082F90E4B02A909A893F91020013AE4
:102CC00018BF012214F0C8FA02AB80B240F2E93218
:102CD000009004A1D1E90001FFF7CCFA16B070BD55
:102CE000AFF30080F2C20B46A9D4A7E26F12833A79
:102CF000302A003090F940300BB1FFF709BE704721
:102D00000FB430B5C3B07C22002146AC23A854F8E0
:102D1000045B19F051F90021772205A8049119F0FC
:102D20004BF923462A465A210DF1AE0003940AF0CE
:102D3000D5FD114B5A2804A993F9102028BF5A2019
:102D4000013A8DF8AD0023A818BF012214F0D0FD80
:102D500004AB80B243F6FF72009005A1D1E90001F7
:102D6000FFF788FA43B0BDE8304004B0704700BFB9
:102D7000759D040C8EA454D6302A00302DE9F047FE
:102D80002DED028BAEB005460DF0BAFA8B4A074620
:102D90001368C31A322B09D9894B1B7833B189497F
:102DA00010600B78013303F01F030B70864C0DF09D
:102DB000A3FAD4F8D03F984255D9201DDFF80092ED
:102DC00013F034FD8046002840F0CD800DF098FAD5
:102DD00099F8003006468DF82080002B40F0AF8037
:102DE00001F078FA4FF4C87306F51676B0FBF3F2EB
:102DF00002FB130394F8D42F16FA83F3C4F8D03FE0
:102E0000724B1B785B00DBB28DF82830002A00F093
:102E100091801CA8FEF7FEFF94F8D41F1CAB0DF1A7
:102E20002900C1F110061944F6B2062E28BF062665
:102E30003246013619F0B2F80023F6B26448059321
:102E40000AAB049603931823029308AB0193012362
:102E5000009356A3D3E9002313F0EAFC011E64DBC0
:102E6000002384F8D43F5B4A1368FB1AB3F57A7FDA
:102E7000C0F0D78017600DF045FA02460B46544863
:102E800013F084FD52491CA814F05CF96422BDF8CB
:102E900074305343BDF87020B3FBF2F39BB2462B62
:102EA00003D921784C480AF05DFD0DF025FA4FF466
:102EB0007A734A4FDFF84491B0FBF3F0484B386027
:102EC000D3F80080D8F8540003685B6E984799F9EE
:102ED00010201CA93881013A384618BF012214F08D
:102EE000DFFC1CAB80B240F25512009031A1D1E959
:102EF0000001FFF7BFF999F90860002E00F0868005
:102F000048460023F6B2012100F8083F02F050FBCA
:102F10002A2E2CD1334C2046FFF7F2FED8F8500071
:102F2000642103685B689847F5E722782E480AF029
:102F300019FD95E743F001038DF8283069E7214634
:102F40001CA811F8048B14F0FDF8BDF8742064235C
:102F5000414626485A43BDF87030B2FBF3F292B2B4
:102F60000AF000FD3CE7002389F800307BE72B2EB8
:102F700004D11F48FFF7C4FE1E4B98474FF4FA6177
:102F80001CA800F031FCD8F850004FF47A710368A7
:102F90005B689847D8F854000368DB6A984778B3B1
:102FA000012800F0AB8014482BE000BF401DA12099
:102FB00026812A0BF1C6A7C1D068080F643E0030F5
:102FC000D4250030683E0030802E0030702E003056
:102FD000842E0030603E0030A4F70508742E0030C7
:102FE000282A0030CEF7050830F7050867F70508EE
:102FF000DFF7050838ED00E01AF80508302A003040
:103000004E48FFF77DFE1CA800F0FAFB00237B7101
:103010000DF076F947F23053984202D9484817F03C
:10302000FBFB95F91830002B6AD12846FFF762FEAA
:103030002846DFF81C81FFF7EDFD2846FEF784FDEA
:10304000404F0DF04DF906469FED3A8B0DF048F9D3
:10305000801BB0F57A7F67D2D8F800304021186D18
:1030600003689B689847FEF787FF002140220BA862
:103070000A91ADF86C1018F09FFFD4F8D83F002BE0
:10308000E4D04FF00109D4F8D80F00258DF81C903A
:103090000DF11D028DF81D5007A903688DED008B01
:1030A000D3F808A02B46D0479DF81C30002BCDD07C
:1030B000294648221CA818F07FFFD4F8D80F08AA88
:1030C0000AA903685D690DF11E03A8479DF86C000D
:1030D00000F0E8FA9DF86D3002460BA98DF8B400B7
:1030E0001DA88DF8B53018F059FF0A9B1CA9384669
:1030F0001C93DDE9082313F00FFEC4E7124880E7B4
:1031000095F8E433002B93D0002395F8E22395F84B
:10311000E11385F8E43395F8E00307F02BFC0B4B43
:10312000012283F8482383E72EB0BDEC028BBDE873
:10313000F08700BF0000000000000000EFF7050866
:10314000263A09B0842E003004F80508302A0030F1
:10315000282A003073B54FF48073264D0446264E5E
:10316000AB800DF0CDF84FF47A73B0FBF3F028602C
:103170006288B4F902307F2A204898BF337090F9F2
:1031800008302BB10023012100F8083F02F010FAAB
:103190001B4B082243F2B0709A6100F00BFA05460F
:1031A00009F03CFE174B00221D60174BC3F8D85F97
:1031B0001A7094F91030012B18D1626961682846A1
:1031C00009F0D8FE002311494FF47A620193104BA5
:1031D000A1F1280000930F4B13F0FAFA317839B1BE
:1031E0000D4802B0BDE8704013F018BB0123E5E7BD
:1031F00002B070BD742E0030702E0030302A0030C6
:10320000000C02585C3E0030802E0030AC2E0030A6
:103210005D21040831250408842E003037B50546A9
:1032200040F206223948012115F028F840F2062222
:103230000221364815F022F8354B364C0321D3F8DD
:10324000E820212042F48002C3F8E820D3F81021BE
:1032500022F48002C3F81021D3F81021D3F8902073
:1032600042F48002C3F89020D3F8902022F4800228
:10327000C3F89020D3F89030236823F00103236033
:10328000236823F480532360236823F4706323604E
:10329000214B2361236823F400332360636823F404
:1032A000006363604023A360A36843F40043A3600A
:1032B000AA23E360E36843F40043E36015F0C0FD34
:1032C0002368164943F002032360236843F0040394
:1032D0002360236843F008032360236843F020033E
:1032E0002360236843F0010323600D4B00951B68A6
:1032F000186B0368DC680B4BA446019302AB13E91F
:103300000C0003B0BDE83040604700BF0014025815
:103310000044025800580040380F300034F80508C7
:10332000282A00308D34040890F9183010B513B9EC
:10333000012380F8E83311B153B2002B04DA02F014
:103340007F0380F8E33310BD90F8E343022C10D0E4
:10335000032C15D0012C05D103F00F0141EA021313
:1033600080F8E2330134012380F8E34380F8E4334A
:10337000E9E703F00F0141EA021380F8E133F1E7D6
:1033800003F00F0141EA021380F8E033EAE700009E
:10339000092B2DE9FF410C46054611461E465BD818
:1033A0001A4601A818F0FAFD242C3AD1092E38D17A
:1033B0009DF805309DF804201B029DF8081043EA93
:1033C00002439DF80620090213435B421A0C8DF854
:1033D00006308DF804201A0A9DF807308DF8052074
:1033E00041EA03419DF80930194349420B0C8DF81D
:1033F00009108DF807300B0A9DF80B108DF8083076
:1034000009029DF80A3041EA03419DF80C30194346
:1034100049420B0C8DF80C108DF80A300B0A8DF810
:103420000B30D5F8B47367B1013E01AD4FF0010820
:10343000731C11D03B79A34211D03B68D3B11F4616
:10344000F8E7082000F0B6F89DF80430C5F8B4039A
:10345000437101230471837104B0BDE8F08101342C
:103460002B78384687F80680E4B27B71013E01353F
:103470000746DDE7082000F09DF82B7838600471DE
:1034800001344371E4B280F80680EFE710B49DF890
:10349000044001945DF8044BFFF77ABF3629D0F859
:1034A000B40310D0E0B103798B4213D00068F9E780
:1034B0000379242B09D000680028F9D17047002334
:1034C000837180207047222070478379002BF6D1CA
:1034D000184670473429EED0002383714079704735
:1034E000704700002F4B10B59C69200715D52E4A58
:1034F000C4F34641002082F8E613C4F3004182F889
:10350000E50382F8E71319B19A6942F001029A6162
:10351000244AD36943F00803D361610718D5214BCE
:1035200021485A6A90F8E633D2B290F8E513232B7B
:1035300005D81F2B07D931B980F8B12303E0552BEB
:1035400001D1FFF7F1FE90F8E533013380F8E53360
:10355000A2071CD5144A92F8E633232B0DD81F2B53
:1035600010D992F8E533104692F8B1131944C9B254
:10357000FFF794FF0B4B986204E0552B02D1094BE7
:103580000021996292F8E533013382F8E533A3060E
:1035900004D5044AD36943F02003D361BDE8104049
:1035A00014F010BC00580040302A0030004870472A
:1035B00050F805080121884238BF084616F0B2BF0E
:1035C00008B116F0B3BF7047FFF7F4BFFFF7F8BFBD
:1035D0007047000013B56C46031D84E8060094E8AC
:1035E000030083E80500012002B010BD73B58568B3
:1035F000019155B11B885B0707D4D0E90036DB6B1E
:103600009847019AC1B23046A847012002B070BD68
:1036100070B598B08568044601915DB1BDF8703011
:103620005B070AD4D0E90036DB6B9847019AC1B238
:103630003046A847012018B070BD0022002305A81D
:10364000CDE9022300234622ADF8103018F0A6FC85
:103650000CF058FE0423ADF810302368CDE90201C8
:103660001B6C02A920469847E4E70000082817D9F8
:103670000C280CD910280CD914280CD918280CD9CE
:1036800020280CD930288CBF0F200E20704709202D
:1036900070470A2070470B2070470C2070470D20A0
:1036A00070470000082817D909280CD00A280CD028
:1036B0000B280CD00C280CD00D280CD00E2814BFD1
:1036C0004020302070470C20704710207047142095
:1036D00070471820704720207047000040687047EE
:1036E00013B50146806818B104680091A168884745
:1036F00002B010BD37B504460D46072200F10C019B
:1037000001A800F08BF8636801A82B43636000F008
:10371000A7F8012003B030BD37B504460D460E2290
:1037200000F10C0101A800F079F8636801A823EA10
:103730000503636000F094F8012003B030BD000081
:1037400037B504460D461D2200F10C0101A800F01A
:1037500065F8002301A8A560636000F081F80120EE
:1037600003B030BD436818478368184710B5024C52
:103770008260C0E9004110BDB0F8050830B50B4DBE
:1037800085B00B46041D696801AA2868092B03C28D
:10379000298988BF002011809FBF04AA9B1813F8B5
:1037A0000C3C54F8230005B030BD00BF14F20508EE
:1037B000007B00F00100704770470000816082804C
:1037C00070470000826838B504465AB1037B13F095
:1037D000010507D143F0010303739047237B65F391
:1037E0000003237338BD0000044B1B6810B504466A
:1037F000186D03681B699847204610BD282A0030C1
:10380000054B00211B6810B50446186D03681B6941
:103810009847204610BD00BF282A0030F8B50C4B51
:103820000446016017461E68306D03681B6C98479C
:10383000054610B1736DA3F84270206803689B6859
:1038400098471DB1736D0022A3F842202046F8BDB1
:10385000282A003010B50446FFF7E0FF204610BDCF
:1038600010B5044600680368DB689847204610BD21
:1038700000207047002070470020704700207047EC
:103880007047000000230B70704700000020704755
:10389000704700007047000000207047002070470C
:1038A0004368C26893423CBF8268D1544368013385
:1038B0004360012070470000F8B505460C468F189C
:1038C0000026BC4207D02B68284614F8011B9B68D1
:1038D00098470644F5E73046F8BD000000207047E1
:1038E0004FF0FF3070470000002070470020704705
:1038F00038B590F89C3004460D468B420CD080F8C9
:103900009C100CF0F9FC2368C4F8A00020465B680A
:10391000984708B984F84D5038BD00007FB50D4672
:103920001446194600267AB1531E0B4A6846CDE963
:103930000026089ACDE9025300F042F8019884422B
:1039400004D92E5404B070BD1346EEE7002CF9D014
:103950002C4404F8016CF5E7C0F8050808B410B56C
:1039600085B007AC54F8043B00940394FFF7D6FFEE
:1039700005B0BDE8104001B070470000F8B505463D
:103980000E4617460024BC4208D02B6828465B69C7
:103990009847431C02D030550134F4E72046F8BD67
:1039A0000EB403B503AA036852F8041B5B680192C6
:1039B000984702B05DF804EB03B0704700F000B820
:1039C0002DE9F04F0B46064690462DED028B8DB04B
:1039D0001978002900F0C182252907D0013303930B
:1039E000336830469B689847039BF1E759789A1CE7
:1039F00025290392F4D00025AA462C461F2C35D841
:103A00002B2928D01AD8202927D023292BD0A1F15F
:103A10003003DBB2092B32D861064DBF05EB8505BB
:103A200044F020040AEB8A0A03EB450556BF03EB7A
:103A30004A0A05F0FF050AF0FF0A05E02D290FD01C
:103A40003029E4D144F00104039B13F8011B0393D4
:103A50000029D3D122E044F0020444F00404F3E747
:103A600044F00804F0E744F01004EDE77F2CCED9D1
:103A7000230613D56C2911D144F48074E4E72E2970
:103A800005D1620600F1698244F04004DCE76C294C
:103A900002D144F08004D7E76829D5D0A1F14503CD
:103AA000022B5DD8203144F01004C9B208F1070898
:103AB00014F0400F24F0C00428F0070808BF0625C2
:103AC0006529A4B2B8EC028BB7EEC88B51D144F093
:103AD000400427060DD5F0EEC87A9FEDA17AF4EEEA
:103AE000C77AF1EE10FAC2BF4FF63F73234043F09E
:103AF000400414F0800346D03B2DA9464FF0070741
:103B000028BF4FF03B0909F101095FFA89F9172233
:103B1000002106A8029318F04FFA4A46B0EE480A70
:103B2000394606A80CF0B0FF9DF81830834603F024
:103B300009020193029B012A2ED0A0072ED414F073
:103B4000040F0CBF00222022019911F00C0757D05E
:103B5000002A40F0A082BAF1030F4FD8174636E092
:103B6000A1F16503022B00F25A8124F01004A4B2E3
:103B70009CE7662902D144F08004AAE7002DA8D072
:103B8000013DEDB2A5E70A2D87BF0A2599462F46CC
:103B9000994688BF2F46BAE72D22D5E72B22D3E7D7
:103BA0000427AAEB07072107FFB20AD43368013FB5
:103BB000029220219B683046984717F0FF07029A2F
:103BC000F4D122B13368114630469B689847019B77
:103BD00004F01004634D13F0080F634B08BF1D463B
:103BE000013D15F8011F002900F0AE800CB120390D
:103BF000C9B2336830469B689847F2E70327D0E79D
:103C0000CDF808B0002B36D0019BD944DB065FFA13
:103C100089F907D59DF81930312B04BF09F1FF3917
:103C20005FFA89F94FFA89F3002B44DDB9F1080FE7
:103C300028BF4FF0080914F08003049316BF2BEA45
:103C4000EB730523013302B101330DB1691C0B4441
:103C50009A45C4BFAAEB0303DFB214F0090F2FD1BA
:103C600077B33368013F059220219B68304698471F
:103C7000059AFFB2F4E76006DDD45D4504DB1BF175
:103C8000040FA8BF44F080046B1C06A90B4435B197
:103C900013F80119302902D1013DEDB2F7E72106F1
:103CA000C9D505F101095D455FFA89F906DDA5EB86
:103CB0000B05EDB2BFE74FF00109BCE70025BAE7FD
:103CC00022B13368114630469B689847220708D4D2
:103CD0003FB13368013F302130469B68FFB29847BF
:103CE000F6E7049B002B47D02BEAEB7406ABABEB5B
:103CF00009096D42ABEB040A9A44A34517DBA145C1
:103D000015DA9AF80110013CA54212DC002900F0F6
:103D1000C881336830469B689847631C04D1336878
:103D20002E2130469B6898470AF1010AE5E73021C9
:103D3000E9E7A34507D19DF81930352B16D802D1F4
:103D4000019BDD0612D591B9002F3FF44DAE3368CB
:103D5000013F202130469B68FFB29847F4E700BF3F
:103D60007F96184BE8F80508E4F805083121336818
:103D70009B6830469847E7E79DF81910304631298F
:103D80001EBF019B03F0EF03019333689B689847C4
:103D9000E5B914F0100F3368304614BF4521652192
:103DA0009B689847BBF1000F29DACBF100032D2166
:103DB0000293336830469B6898473021029B092B59
:103DC00023DD01310A3BC9B20293F7E702353368BC
:103DD0004FF002092E21EDB29B68304698474B46C2
:103DE0000CAA09F1010930461A4433685FFA89F9CF
:103DF0009B6812F8181C9847A945F0D1C9E702D171
:103E0000019BDC06D1D42B21D3E7336830469B6875
:103E100098470299336830319B68C9B2A9E7632992
:103E200035D073294ED0642963D124F0900714F45F
:103E3000807F0DF11809BFB279D008F1070222F096
:103E4000070251689046002958F8080B04DA4042EE
:103E500047F0800761EB41010A234A4600F074F9FC
:103E6000A0EB0900C4B27B0640F1978027F001095E
:103E7000AC421FFA89F980F0CB8007F01403102BB5
:103E800003D127F011071FFA87F9AB4687E058F8EE
:103E9000043B01250DF118098DF81830200701D4D5
:103EA000AA451CD84D445746A9453FF44DAF336849
:103EB000304619F8011B9B689847002FF4D0013F4A
:103EC000FFB2F1E714F0400F58F8049B14BF2946E5
:103ED0004FF0FF31484618F0F7FB0546DEE7336840
:103EE0000AF1FF3A202130469B685FFA8AFA984728
:103EF000D6E7692999D0752925D124F010040A2321
:103F0000A7B217F4807FDBB20DF118093ED008F19B
:103F100007084A4628F00708F8E8020100F014F9FB
:103F2000A0EB090027F08007C4B2BFB29BE758F8A6
:103F3000040B0A2249460028BCBF404247F08007D4
:103F400000F0B4F88CE724F006077029BFB211D056
:103F500008D8582911D06F2916D00DB0BDEC028BAE
:103F6000BDE8F08F7829F8D1F90601D547F00407AC
:103F70001023C6E747F01007F6E7E20601D547F041
:103F800006074FF40473BCE70823BAE71A4649460C
:103F900058F8040B00F08AF8C2E7A346B94619F0B6
:103FA000100F42D00CAB234413F8193C302B31D105
:103FB00029F016091FFA89F919F0080745D119F0F7
:103FC000010F36D0DA4546D904EB0A05A5EB0B05FF
:103FD000EDB2336819F0100F9B6840D030213046A5
:103FE000984719F0040F09D019F0020F336818BF71
:103FF00058219B6808BF7821304698473368AC4207
:104000009B6839D2013D30213046EDB29847F5E743
:10401000A346C4E719F0040F02D10BF1010B01E034
:104020000BF1020B5FFA8BFBC6E719F0860FC3D0CA
:10403000F3E73368DA459B680FD90BF1010B2021B8
:1040400030465FFA8BFB9847F3E7DA4505D9AAEBD0
:104050000B07FFB2BDE72546BBE70027B9E719F01C
:10406000860FCBD019F0020F14BF2B21202119F09D
:10407000800F18BF2D21BFE7651E06AB53FA85F5EB
:10408000013C336815F801193046E4B29B68984743
:10409000002CF5D158E6BAF1040F3FF681AD0027A8
:1040A00090E5A3457FF450AE45E600BF082A30B541
:1040B00005D10346C008FCD130330B700DE0102A47
:1040C0000DD100F00F0202F13003392B88BF02F14D
:1040D0003703000901F8013BF3D1084630BD034620
:1040E0000022DCB223F00103023304F1300442F178
:1040F0000002580840EAC270C31842EB5202180985
:1041000040EA0270C01842EB1212030A43EA02634B
:10411000181842EB1222030C43EA02431B1842EB2D
:104120001242D31842F100001B0943EA007302094E
:10413000C3EB431553EA1010C3EB850504EB4504AC
:1041400001F8014BCDD1C8E7082B30B50AD10346A1
:10415000C00840EA4170C90850EA0104F7D1303381
:10416000137012E0102B12D100F00F04000904F1BB
:10417000300340EA01700909392B88BF04F1370385
:1041800002F8013B50EA0103EED1104630BD20F0A9
:104190000104C5B2023405F1300541F100036108A4
:1041A00041EAC3710C1943EB5303210941EA03713E
:1041B0000C1943EB1313210A41EA03610C1943EB79
:1041C0001323210C41EA0341091943EB1343591806
:1041D00043F10003080940EA03701909C0EB4014D9
:1041E00050EA1313C0EB840405EB440502F8015BAD
:1041F000CDD1CAE770EE600ADFED057AF0EEE00A95
:10420000F4EEE70AF1EE10FA4CBF012000207047EF
:104210000000003408B517F041FCB4EE400ADFEDB1
:10422000037AF1EE10FA17FE800A08BD00000000C4
:1042300008B52DED028B9FED088AF0EE480A17F0C5
:1042400003FCB5EEC00AF1EE10FA48BF30EE080AE2
:10425000BDEC028B08BD00BF0000B443B4EE400AC1
:1042600010B5F1EE10FA04462DED028BB0EE608A27
:10427000F0EE418A0FD705F09FFF4FF48061A2B2A4
:1042800005F086FF38EE288AB6EE000A28EE000A0E
:10429000BDEC028B10BDB4EEE00AF1EE10FA06D4CC
:1042A000B4EE410AF1EE10FA31FE000AF0E7B0EE8A
:1042B000600AEDE7884203D39042014628BF1146C9
:1042C00008467047884203DB90420146A8BF11466A
:1042D00008467047094A49F26900136899B21B0CF5
:1042E00000FB013344F250611360054B186882B241
:1042F000000C01FB0200186080B27047DC25003022
:10430000D825003091ED011A88B0D0ED077A90EDF4
:10431000010AD0ED040A21EE000A91ED007A61EE67
:10432000200A90ED036A21EE271AD0ED066AD0ED3F
:10433000005AE7EE060AD1ED027AA5EE870A90ED63
:10434000056AA7EE261AD0ED026A90ED087AE7EE2C
:10435000860AA6EEA70AA7EE871A08B0704700BF24
:1043600091ED005AD1ED015A91ED026AD0ED006A4B
:1043700090ED017AD0ED027A76EE856A37EE257AF5
:1043800077EE867AC0ED006A80ED017AC0ED027AA0
:10439000704700BFD0ED006A90ED017AD0ED027A4F
:1043A00066EE806A27EE007A27EE800AC0ED006A8A
:1043B00080ED017A80ED020A704700BF90ED007A2F
:1043C000D0ED017A90ED026AC7EE006A87EE807A3E
:1043D000C6EE007AC0ED006A80ED017AC0ED027A87
:1043E000704700BFD0ED007AF4EE677AF1EE10FA74
:1043F00010D6D0ED017AF4EE677AF1EE10FA09D614
:10440000D0ED027AF4EE677AF1EE10FA6CBF01207B
:104410000020704701207047D0ED007A9FED0F7AA1
:10442000F0EEE77AF4EE477AF1EE10FA14DCD0ED14
:10443000017AF0EEE77AF4EE477AF1EE10FA0BDC4F
:10444000D0ED027AF0EEE77AF4EE477AF1EE10FA68
:10445000CCBF01200020704701207047FFFF7F7F05
:1044600008B52B2900F27E82DFE811F044004402F7
:104470003E02310228021702650156014D016C010E
:1044800058003C01790184014500D4000001EB0093
:10449000350122011B01060193010402FE01D8012E
:1044A00045005800CD01BE01B401A7019E01C7001F
:1044B000BE00B700AA009B00700061002C006902DA
:1044C0005E024F02D0ED015AD0ED007A9FEDD76A1F
:1044D00035EEA77AD0ED026A77EEE57AF1EE666AFC
:1044E00027EE067A67EE867AC0ED016A80ED027AE1
:1044F000C0ED007A08BD90ED007AD0ED016AD0EDF4
:10450000027AB1EE477AF1EE666AF1EE677AC0EDB3
:10451000006A80ED017AC0ED027A08BDD0ED027A22
:104520000268F1EE677A436842600360F3E7D0ED1A
:10453000007A90ED026ADFEDBD6A37EE867A77EE9B
:10454000C67A27EE267A67EEA67ACFE7D0ED017A13
:104550009FEDB76ADFEDB76A9FEDB77A67EEA66A9F
:10456000D0ED005A27EE877ADFEDB44A67EE867AFF
:104570009FEDB35A9FEDB34AA5EEA47A90ED026A7F
:10458000E5EE857ADFEDB04AE5EE846A9FEDAF5A3D
:10459000DFEDAF5AA6EE057AE6EE257AE6EE246A5E
:1045A000B5E790ED027AD0ED007AB1EE477A436834
:1045B000F1EE677A836080ED007AC0ED017A08BD84
:1045C000D0ED007A90ED017AF1EE677A8368B1EE72
:1045D000477A036080ED027AEFE7426881680368FA
:1045E00041600260836008BDD0ED017A8268F1EE1F
:1045F000677A036802608360DFE790ED027AD0EDAE
:10460000017AB1EE477A0368F1EE677A836080ED54
:10461000017A6DE790ED016AD0ED007AD0ED026A83
:1046200037EE867ADFED8B5A77EEC67A9FED7F6A9A
:10463000F1EE666A27EE257A67EE867AC0ED026AA9
:10464000E5E790ED026AD0ED007ADFED786A37EEAB
:10465000867A436877EEC67A836027EE267A67EE1D
:10466000A67AC0ED017A80ED007A08BDD0ED027A1D
:104670004368F1EE677ABEE7D0ED025AD0ED007ADA
:10468000D0ED016A37EEE57A9FED686A77EEA57A9C
:10469000F1EE666A67EE867A27EE067AC0ED026A68
:1046A000DFE7D0ED017A8368F1EE677A436032E7A5
:1046B000D0ED026AD0ED007ADFED5C5A37EEE67A93
:1046C0009FED646A77EEA67A436827EE067A8360E8
:1046D00067EEA57AC5E78268416803688160026079
:1046E000436008BDD0ED017AD0ED005A9FED4F6ACE
:1046F00037EEA57AD0ED026A77EEE57AF1EE666ADA
:1047000027EE067A98E790ED017AD0ED027AB1EEC5
:10471000477AF1EE677AFCE6D0ED007A90ED016A17
:10472000DFED426A36EE677A77EE867A27EE267AF2
:1047300067EEA67A6BE7D0ED007A4368F1EE677A10
:1047400003603AE7D0ED007AD0ED015A9FED376A69
:1047500037EEE57AD0ED026A77EEA57ACEE790EDF6
:10476000007AD0ED027AB1EE477AF1EE677A80ED09
:10477000007AD0E690ED016AD0ED007AD0ED026AC1
:1047800036EE677ADFED295A77EE867A9FED316A49
:104790004EE7D0ED027A90ED017AF1EE677A036888
:1047A000B1EE477A4360A1E6D0ED007A4268F1EEBF
:1047B000677A8368826043609AE690ED017AD0ED73
:1047C000026AD0ED007AB1EE477AF1EE666AF1EE58
:1047D000677A89E6D0ED017A90ED007AF1EE677A9A
:1047E0008368B1EE477ADDE7D0ED016A90ED027A99
:1047F000F1EE666AD0ED007AB1EE477AF1EE677AB3
:10480000C0ED016AB3E7D0ED007A90ED027A43681B
:10481000F1EE677AB1EE477A03607AE6D0ED027A7C
:104820000368F1EE677A836062E600BFF304353F08
:10483000DB26B93E46D0BC3EC9355BBF4F0DAABE94
:10484000C6AC6EBFCF78123E4D1F6BBFF184CABE9F
:10485000F63BCC23F30435BFF304353F81177E3F8D
:10486000A296F93DA296F9BDD0ED007A8368F1EEEB
:10487000677A5AE690ED026AD0ED007AD0ED016ACF
:1048800037EE867A5FED0C5A77EEC67A1FED0F6A27
:10489000F1EE666A67EEA57AFEE6D0ED017AD0ED1C
:1048A000006A5FED145A37EEA67A1FED156A77EEAF
:1048B000E67A27EE257A67EE867AA8E690ED007A0A
:1048C000D0ED017AB1EE477AF1EE677A73E6D0ED7A
:1048D000007AD0ED016A5FED205A37EEE67A1FEDDF
:1048E000236A77EEA67AE4E7D0ED017A0368F1EE69
:1048F000677A60E7D0ED007A90ED016A5FED2A6A91
:1049000037EE867A77EEC67A10E7D0ED017A90ED31
:10491000026A5FED2F6A36EE677A77EE867A27EEC7
:10492000267A67EEA67A55E6D0ED017A90ED026A16
:104930005FED376A37EE867A77EEC67AEFE7D0ED2D
:10494000027A5FED3A6A1FED3A5A27EEA67A90EDA9
:10495000006A67EE857A5FED3D5AA6EE257AE6EEAF
:10496000267AC3E505F028FC40F211124FF48001CD
:10497000BDE8084005F00CBC90ED020AD0ED017ACC
:1049800020EE000A90ED007A27EE077AA7EEA70A3C
:10499000B7EEC77AB7EEC00A37EE007BB5EE407BC4
:1049A000F1EE10FA04D4B1EEC70BB7EEC00B7047AE
:1049B000B0EE470B08B517F01BF8B7EEC00B08BDFB
:1049C0007047000038B5056804462DB128460BF045
:1049D000D1FE2846FEF7F4FD204638BD37B5044623
:1049E0000D46134601920246054801F0A7FD019BC2
:1049F00022462946034803B0BDE8304001F09EBD81
:104A0000BC3E0030A43E00300422064B13B50446E1
:104A100001460DEB02000193FFF7E0FF024B1C8003
:104A200002B010BDFFFF3F00B03E0030502307B57D
:104A30008DF804304123042200218DF8053006232F
:104A40000DEB02008DF807108DF80630FFF7C6FF5A
:104A50000420FFF7D9FF03B05DF804FB02EB8202EC
:104A600000EB820042783AB933B1008A000703D4E0
:104A70003F2098400844704702FA03F0FAE700002C
:104A8000430608D4C00908D0054B1B88184214BF40
:104A9000012000207047002070470120704700BFB0
:104AA000B43E00300B4B013010B51A8880B20A4B6F
:104AB00018241B6804FB0033824206D91C89183372
:104AC0008C4204D0013080B2F6E7002010BD0120F6
:104AD000FCE700BFC03E0030C43E0030028AC3681D
:104AE000D20648BF1B68184670470000828A0369D7
:104AF000D20648BF1B6818467047000013B5002453
:104B0000042369461D482246CDE9004401F0DCFC3F
:104B1000042322461A480DEB030101F0D5FC9DF851
:104B20000030502B07D19DF80130412B03D19DF867
:104B30000230062B1DD09DF80430502B17D19DF864
:104B40000530412B13D19DF80630062B0FD10C49AF
:104B50000A4801F02DFD50B105F02EFB4FF4B37261
:104B60004FF0805105F014FB012002B010BDFFF79B
:104B70005DFF0249024801F01BFDF5E7BC3E003035
:104B8000A43E0030828AC368920705D51B68181EB0
:104B900018BF01200B6070470120FBE737B50B8A77
:104BA00014460D46DA0705D523688A681344236046
:104BB000012012E09B07FBD50A4B182201A91B68B4
:104BC00002FB0030FFF7DEFF48B101992268AB68B5
:104BD0000A44D3581BB15B1A236003B030BD0020D8
:104BE000FBE700BFC43E00302DE9F04F1D468BB0FF
:104BF000182306469DF85480174653434FF0000B88
:104C00000691059308F10603DBB207935FFA8BFA6E
:104C1000142303FB0AF3EC5C05EB0309002C4CD0D6
:104C2000062C28D1B8F10B0F21D84846FFF756FFC4
:104C30000446C8B1169B09AA494638460993FFF7AE
:104C4000ADFF88B14346524614992846FFF706FF48
:104C5000099B3A4606990293079BCDE90003234638
:104C60003046FFF7C1FF18B90BF1010BCEE700206A
:104C70000BB0BDE8F08F4346524614992846FFF723
:104C8000EDFEB0EB963FEFD1C6F30423A342EBD188
:104C90000B4C09A9059B20681844FFF773FF0028F7
:104CA000E2D0D9F80830099A1344169A1344069AA8
:104CB0001360059B20681844DAE72046D8E700BF58
:104CC000C43E0030204B2DE9F04F5FFA80F8B3F876
:104CD00000A0C0F340330F4687B0054648EA0328DA
:104CE0001A4BC0F3042B00211E681FFA81F9CA4534
:104CF00027D933893446434520D13378062B0FD149
:104D00003046FFF7F3FEC8B100234A463946009308
:104D1000CDE9013303462846FFF766FF044609E064
:104D20009B450BD105A93046FFF72CFF0028F5D095
:104D3000059B3B60204607B0BDE8F08F0131183677
:104D4000D3E70024F6E700BFC03E0030C43E003089
:104D50002DE9F04F984618238DB0044653430D4675
:104D60000AA917460693474B9DF858901868069B6A
:104D7000DDF868B01844FFF705FF00287FD0002356
:104D8000079309F10603DBB209939DF81CA01423D5
:104D900003FB0AF3EE18EB5C002B70D0062B3BD123
:104DA0003046FFF79BFE0890002831D0B9F10B0F79
:104DB00065D8179B0BAA314638460B93FFF7EEFEDA
:104DC00030B39BF80030012B59D85A1C0BEB8303EE
:104DD000414628468BF8002052465E604B46FFF75E
:104DE0003DFE1B9A034608992046CDE904B2199A64
:104DF0000392189A02920B9A0192099A00923A46EB
:104E0000FFF7A6FF00BB9BF80030013B8BF800309A
:104E1000079B01330793B8E7179AB06810440A9AC2
:104E20001044A04213D14B46524641462846FFF754
:104E300015FE189B1B9A1860199B1E6000231370A7
:104E4000104B1868069B18440DB0BDE8F08F052B79
:104E5000DED1031D9C4203D000F108039C42D7D150
:104E6000201A1B9B52464146800818704B46284624
:104E7000FFF7F4FD189B1860199B1E60E0E7002007
:104E8000E2E700BFC43E00302DE9F04F00258BB0B3
:104E900006460F469046DFF8A0A007931560254B05
:104EA0001FFA85FB1B885B4542D95B461822DAF85E
:104EB00000105343CC1811F8039009A92046FFF7BE
:104EC00061FE98B3B9F1060F17D12046FFF70EFE29
:104ED000014658B3149B5A46304602970593079BE8
:104EE000CDE903830023CDE90033FFF731FF04460A
:104EF000E0B120460BB0BDE8F08F0998B04204D174
:104F00000023149A3B601370F3E7B9F1050F0DD13C
:104F1000031D9E4203D000F108039E4206D1301AC1
:104F2000149B8008187000233B60E2E70135B6E768
:104F30000024DEE7C03E0030C43E00302DE9F047DB
:104F400009889846234B88B0C1F3080904461B68BA
:104F5000174609EB4901119E03EBC10513F831A077
:104F600007A92846FFF70EFE20B90025284608B0FD
:104F7000BDE8F0870021BAF1060FC8F8001013D180
:104F80002846FFF7B3FD0028EFD0109B4A4600915A
:104F90000596CDE90383CDE901170B46014620466E
:104FA000FFF7D6FE0546E1E70798A04202D1396037
:104FB0003170DBE7BAF1050FD7D1031D9C4203D056
:104FC00000F108039C42D0D1241A0023A4083470B5
:104FD0003B60CBE7C43E00300138C0B204289ABF22
:104FE000014B185C0020704710F905082DE9F84FB7
:104FF0009846931D00240746DBB20D461646A3468D
:10500000A1462DED028B08EE103AE3B21422534371
:10501000F85CF918002857D04B783F2B04D90020B2
:10502000BDEC028BBDE8F88F16B1002B08BF3F2303
:10503000C3F1200EA3F1200C2BFA03F209FA0EFEA5
:1050400029FA0CFC42EA0E02C3F1200E42EA0C02DD
:1050500012F0010FA3F12002E1D14FF0010C06285C
:105060000CFA02F22CFA0EFE0CFA03F342EA0E02DC
:1050700043EA0B0B42EA090915D10B2ECFD808469B
:10508000FFF72CFD824660B14868FBF7DFFE404425
:1050900018EE102A2946C3B25046FFF7A7FF002892
:1050A000BDD00134B1E7FFF797FF82460028B6D0A4
:1050B0004868FBF7CBFE40441028B0D82B88043357
:1050C00003EB0A002880ECE70120A9E72DE9F74F60
:1050D00004230025DFF894904FF0180AADF806304D
:1050E000214B1FFA85F81B8843453BD90AFB08F37F
:1050F000D9F80020D75CD418062FB4F808B025D111
:10510000B8F1000F03D1002003B0BDE8F08F2046B6
:10511000FFF7ECFC064608B90135E1E76068FBF7EC
:1051200095FE0022C3B20DF106013046FFF75EFF87
:105130000028E8D059464046FFF7B4FC0028E2D1E9
:10514000062FE9D0A38A9B07E6D5DCE73846FFF7B0
:1051500043FF0028D7D0BDF8063004331844ADF81B
:105160000600E7E70120CFE7C03E0030C43E003034
:10517000437803F01F021F2A0FD00278C3F34013B5
:1051800042EA032340F2FF12934206D0006801383E
:10519000C31C94BF0020012070470120704700000D
:1051A0002DE9F34106460D460424214FDFF888809F
:1051B0007B88A34237D90423224638460DEB0301EE
:1051C00001F082F99DF80510737881EA0302D20696
:1051D00018D1C3F3401396F800C0C1F340129DF8F4
:1051E00004004CEA032340EA022293420AD13268C7
:1051F000019B534013EA080F04D101202C8002B018
:10520000BDE8F08101A8FFF7B3FF20B1094B2C8066
:105210001C800020F3E701F01F00FFF7DDFE031DF7
:105220001C44A4B2C4E74FF6FF732B80F1E700BF24
:10523000BC3E0030B03E003000C0FFFF70B50C46F1
:10524000114615461E46204617F03EFA831CAB4217
:1052500009D85F2258362254221803305670A842CB
:105260009CBF0022E25470BD2DE9F74FDDE90D54DB
:105270009B464FF000099DF83C3007468A4616468B
:105280004968224628469DF83080009317F008FAB6
:105290005FFA89F29BF800109142019212D92146DF
:1052A000284617F011FA019AC0B2844207D90BEBD5
:1052B00082025168221A2844496817F0F1F909F16D
:1052C0000109E5E7E6B12146284617F0FDF9C3B22A
:1052D0009C4204D9E21A7168E81817F0E1F9009BC2
:1052E00013B9B8F1000F13D03378052B10D1434612
:1052F00022462946384603B0BDE8F04FFFF79EBF6F
:10530000009B13B9B8F1000F02D09AF80030ECE717
:1053100003B0BDE8F08F0000F0B58BB01F4600234E
:10532000154607AC05AA07930646C4E901330DF1FB
:105330001303CDE9004306ABFFF700FE014610B9A9
:1053400028700BB0F0BD9DF840303046069A0195AC
:10535000CDE902739DF8133000932346FFF784FFD5
:10536000EFE700002DE9F04F4FF0180887B0044632
:105370000E4608FB01F84FF0000ADFF818B1CDE93E
:10538000022314225FFA8AF35343039A12F803901C
:10539000D518B9F1000F7AD0B9F1060F6F6828D18E
:1053A0003846FBF753FD39460246204617F042F9CE
:1053B000002865D12846FFF791FB074600285FD0FB
:1053C000029B05AA294630460593FFF7E7FB002814
:1053D00056D06868FBF73AFD109B059A314600935A
:1053E00020443B46FFF7BEFF002849D007B0BDE888
:1053F000F08F3946204617F003F980B9DBF800003A
:1054000005A94044FFF7BEFB002839D0109B83F864
:105410000090059BA8681844029B1844E6E7B9F180
:10542000050F2DD11021384617F04EF939465FFA95
:1054300080F920464A4617F01FF908BB14F90930D5
:105440005F2B1DD109F1010914F80930583B022BDB
:1054500016D8DBF8000005A94044FFF793FB78B1AC
:10546000A868059B109A1844029B184404231370E3
:1054700014F90930592B06D05A2B06D0582BB5D029
:105480000AF1010A7DE70430B0E70830AEE748468C
:10549000ACE700BFC43E00302DE9F04F04468BB0AE
:1054A00017460025DFF8C0B002912E4B1FFA85FA8F
:1054B0001B88534553D9182253465343DBF8002029
:1054C00012F8038002EB0309B8F1060FD9F8043093
:1054D00033D110211846039317F0F6F8039B5FFAB7
:1054E00080F820464246194617F0C6F806460028BE
:1054F00033D14846FFF7FAFA034670B3029A04EB39
:105500000800514600923246FFF72CFF804620B338
:105510007FB10DF1130306AA05A90596009307AB09
:105520000996CDE90766FFF7AFFC069B0BB11B8A16
:105530003B8040460BB0BDE8F08F1946204617F07F
:105540005FF850B9029B07A9484683F80080FFF72F
:1055500019FB20B1DDF81C80EBE70135A5E74FF022
:105560000008E6E7C03E0030C43E003010B500231E
:1055700090B00446069306A90A9307AACDE908331A
:105580000DF11703009308ABFFF77EFC014668B1ED
:10559000112301222046CDE902320BAB079A019379
:1055A0009DF81730009308ABFFF75EFE10B010BDFA
:1055B000F0B52C4D87B04FF4CE72064602900C46E3
:1055C0008DF80C1001A8291DFEF728F9052204A961
:1055D00028680BF007FA074601A8FEF741F9052FE6
:1055E00006D1049BB34203D19DF81430A34236D0B8
:1055F0001D4E1E4F40F25712314601A8FEF70EF91C
:1056000028680BF011F9042821D9052202A928687D
:105610000BF080F9431F5C425C4101A8FEF720F9C2
:10562000ECB93C68636D93F89C3093B9206D01210F
:1056300003681B699847206D4FF4FA7103689B68F3
:105640009847206D002103681B699847D2E7002422
:10565000E3E7206D03681B6C98470028E6D007B08D
:10566000F0BD00BF883E00308C3E0030282A00305C
:105670002DE9F341154EC924154F06F10408013CEC
:10568000A4B2FCB14FF4A172414601A8FEF7C6F8DE
:1056900030680BF0AFF8054601A8FEF7E1F8042DDD
:1056A00010D93D680A21286D03681B699847286D49
:1056B0000A2103685B689847286D002103681B690D
:1056C0009847DCE702B0BDE8F08100BF883E0030BB
:1056D000282A003000B500238BB0049305AA099353
:1056E00004A9CDE907330DF10D03009307ABFFF7D4
:1056F000CBFB10B3059B23B31B78028903F01F0378
:105700000DF10E0106A88DF818201B02C2F300222D
:1057100043EA4233049A43EA82339DF81820134344
:105720000693FFF73DFD40B19DF8193003F01F03CC
:10573000052B03D09DF80D3003B100200BB05DF8B0
:1057400004FB0378D9E70000F0B5134F89B0064693
:105750000D463B88F3B10DF10B03002404AA03A905
:10576000009305AB03940794CDE90544FFF78CFB48
:1057700080B10A4B38881B68A2B290420AD91A46F7
:1057800001340C3311688E42F6D1137A01202B704C
:1057900009B0F0BD0020FBE7B83E0030AC3E003061
:1057A00013B50DF107010446FFF7CEFF10B92046EF
:1057B000FFF790FF02B010BD0138032816D8DFE8CC
:1057C00000F002080E13FDEEC07A17EE903A0B704F
:1057D0007047BDEEC00A10EE103A0B807047BDEE68
:1057E000C00A81ED000A704781ED000A7047000091
:1057F00007B5036803F0004303600A4B1B881BB91D
:10580000002003B05DF804FB074B11B11A68127851
:105810000A7001A91868FFF7B5F90028F0D00198BF
:10582000EFE700BFC03E0030C43E00302DE9F04F2E
:105830008FB09B4680460E469DF870309DF8609074
:105840000B9318231A9D434308920A93002307934E
:1058500014239DF81CA003FB0AF3F45CF718002C3A
:1058600000F0BA80388AFFF70BF9002800F0B18009
:10587000062C2DD13846FFF731F90446002800F0F8
:10588000A880199B0DAA394640460D93FFF786F96B
:10589000002800F09E804B46524659463046FFF79E
:1058A000DDF80B9A03462146049240461B9ACDE947
:1058B00002520D9A019209F10602D2B20092089AA0
:1058C000FFF7B4FF002800F084800FB0BDE8F08F30
:1058D000089B1B780993002B3CD02B8852465946D5
:1058E000304668F308032B804B46FFF7B7F83B4B75
:1058F00003EA40302B6823F0FF4323F4FF0323F433
:10590000FC4318431B9B286003B11C70344B0DA94A
:1059100018680A9B1844FFF735F9002859D00D9AEA
:10592000BB681344199A98180B9A002ACDD02D4AB7
:105930001278002AC9D03A78012AC6D13A8A520789
:10594000C3D5199A9B56002BBFD1EB7843F0800347
:10595000EB70BAE74B46524659463046FFF77EF8A1
:105960002B68C3F35133984233D10123089A137043
:1059700095F90330002B06DAEB78099A62F3C71326
:105980001046EB70A1E7052C23D16B78C3F34302DB
:10599000022A1ED8013262F344036B701B9B13B1C1
:1059A00004231B9A13700E4B0DA918680A9B184408
:1059B000FFF7E8F868B1B8680D9C95F801B020448D
:1059C000199BCBF3430B18440BF1FF3B00EB8B000F
:1059D0007BE7079B01333AE7204676E700E0FF7F4D
:1059E000C43E0030E02500302DE9F04F1746048812
:1059F00000228BB0DFF8E090C4F308038DF8272075
:105A00000546B9F800200E461C469A4262D91BB2E0
:105A1000DFF8C88003EB4303D8F80020D90012F860
:105A20003330052B18D14378C3F34302022A15D82B
:105A3000013262F3440343700EB10423337068787B
:105A4000D8F80020C0F343001144431EC86800EB9F
:105A500083000BB0BDE8F08F062B04D00134012386
:105A6000A4B28DF827304FF0180B4FF0000AB9F8A8
:105A70000030A3422ED9D8F800300BFB04F15A189D
:105A80000793908AFEF7FCFFB0B1079B595C06298B
:105A900015D11046FFF72AF8014668B100230DF131
:105AA00027022046CDF800A0CDE90367CDE901A586
:105AB000FFF7BCFE0028CCD10134A4B2D7E72B6895
:105AC000C4F3080403F0004323432B6006B1317094
:105AD000D068BEE70020BCE7C03E0030C43E0030C6
:105AE00037B505460C4601220DF107012846FFF7A0
:105AF0007BFF28B19DF80730042BF4D804B1237044
:105B000003B030BDF8B50025074610460E461446D2
:105B1000FFF76EFE38B1BD4205D031462046013553
:105B2000FFF7DEFFF6E7F8BD0139032913D8DFE8F8
:105B300001F002090C0F90F9003000EE103AB8EEB7
:105B4000C00A7047B0F90030F7E790ED000AF6E7B9
:105B500090ED000A70479FED010A70470000C07F7A
:105B6000B4EE400A10B5F1EE10FA04460CD6F0EE91
:105B7000C07A9FED317AF4EE477AF1EE10FA03DC49
:105B8000042902D180ED000A10BD032919D1B5EE18
:105B9000C00A9FED2A7ADFED2A7A4FF400609FED6C
:105BA000291AF1EE10FADFED280A58BFF0EE477A15
:105BB00030EE270AFEF752FBBDEEC00A84ED000A64
:105BC000E2E702291AD1B5EEC00A9FED1C7ADFED9B
:105BD0001C7A40F605009FED1D1AF1EE10FADFED7C
:105BE0001C0A58BFF0EE477A30EE270AFEF736FB64
:105BF000BDEEC00A10EE103A2380C5E70129C3D1DB
:105C0000B5EEC00A9FED0D7ADFED0D7A40F60A0081
:105C10009FED101AF1EE10FADFED0F0A58BFF0EE0B
:105C2000477A30EE270AFEF719FBFDEEC07A17EE31
:105C3000903A2370A8E700BFFFFF7F7F0AD7233C7D
:105C40000AD723BC0000004F000000CF00FEFF4633
:105C5000000000C70000FE42000000C32DE9F34130
:105C60001D4690F900300F469046232B4FF000045C
:105C70002CD001AA1649019417F06EFB064618B9FC
:105C8000002002B0BDE8F081FBF7E0F81028F7D85B
:105C900001AA0F49204617F05FFB0028F0D02146EB
:105CA00017F0EEFA01AA88ED000A204608493E6086
:105CB00017F052FB30B10749FBF7BEF810B90120CD
:105CC0002870DEE7002301202B70DAE72046D8E7B2
:105CD000ECF80508F3F805082DE9F041254D4FF0E3
:105CE00000089CB007466E8A1435A0F80080002E8C
:105CF0003CD0632E31464FF0000328BF63219CB295
:105D0000E85C621C0A2892B206D0013398B2814244
:105D1000F5D891422AD014462246294603A816F007
:105D20003DF91CAB234403F8648CE34301341E4467
:105D30009DF90C3015FA84F5232BB6B2D7D0002B81
:105D4000D5D00DF1020302AA01A903A8FFF786FF2F
:105D50000028CCD000220DF103010198FFF79CFB35
:105D60000028C4D03B8801333B80C0E701201CB031
:105D7000BDE8F08118F905082DE9F04FDFF824811E
:105D80009DB0D8F8000008B1FDF720FC0024DFF832
:105D900018A1DFF818910DF10200C8F80040AAF828
:105DA0000040A9F80040ADF80240FFF795FF002839
:105DB00072D0BDF802300C20394EA3465843FDF78F
:105DC00003FC143636F8027CC8F80000BDF8021057
:105DD000A1425FD9002F5DD0632F38464FF00003FA
:105DE00028BF63209DB216F803C06A1CBCF10A0FDD
:105DF00092B206D001339DB2A842F3D8904249D066
:105E000015462A46314603A816F0C8F81CAB2B44A9
:105E100003F864BCEB4301351F449DF90C3016FABE
:105E200085F6232BBFB2D1D0002BCFD06B4602AA70
:105E300001A903A8FFF712FF0028C7D000220DF127
:105E400001010198FFF728FB05460028BED00C236E
:105E500003FB04F2D8F800309850D8F8003013440F
:105E6000029A5A609DF800201A7222B1B9F80030E7
:105E70000133A9F8003001342846A4B2FFF72AFC08
:105E80000028A3D19DF8011028469DED020AFFF7D6
:105E900067FE9BE7AAF800101DB0BDE8F08F00BFB9
:105EA00018F90508AC3E0030B83E0030AA3E00307C
:105EB000024B5B8A0BB1FFF75FBF704718F905080B
:105EC00030B5002085B0FFF7F3FF214B1A7872B987
:105ED00001221A701F4B204A1B680292186D1F4A3C
:105EE0000368039204AA9B6A12E9060098470424F7
:105EF0001B4D6B88A34229D90423224669462846B4
:105F000000F0E2FA6846FFF733F918B1154B1C8030
:105F100005B030BD01A90098FEF7D4FE60B19DF830
:105F20000100221D00F01F0092B2FFF755F8019901
:105F30000346284600F0C8FA9DF8010000F01F0053
:105F4000FFF74AF804300444A4B2D2E70020DFE7A8
:105F5000BA3E0030282A0030693E0030016404084F
:105F6000BC3E0030B03E00300A4B002270B51E88A7
:105F7000094B1B6894B2A64208D91C4601320C3367
:105F800025688542F6D194ED010A70BD91ED000AB5
:105F9000FBE700BFB83E0030AC3E00302DE9F043D7
:105FA00000238BB00446039304AA099303A9CDE907
:105FB00007330DF10903009307ABFEF765FF0546B4
:105FC00020B9002630460BB0BDE8F083049B002BBF
:105FD00040D01B782A8903F01F030DF10A0105A8A0
:105FE0008DF814201B02C2F3002243EA4233039AC5
:105FF00043EA82339DF8142013430593FFF7D0F84A
:10600000064690BB06A92846FEF7BCFD0028D9D05D
:106010009DF81570DDF8108007F01F07DDF8189067
:10602000B8F1000F1AD09DF81C30ABB1089A012BC3
:10603000956802D0099B9B681D4408F10C0120461D
:10604000FFF792FFD8F80810494429443846FFF773
:10605000B3FBB7E70378BDE73546EEE705F110017E
:106060002046FFF781FF4946F0E79DF815009DF8AF
:10607000093000F01F02052A0FD0002BA1D100F03B
:106080001F002146FEF7A8FFBDF80A200346054879
:10609000043292B200F018FA94E7002BEFD0A4EB90
:1060A0008304ECE7BC3E00302DE9F04106460C4687
:1060B00000254FF01408EBB208FB03F3E75CE1188E
:1060C00067B1042F08D888680C313044FFF74CFFC3
:1060D00001463846FFF770FB0135ECE7BDE8F0817B
:1060E0002DE9F7430024134FDFF84C804FF01809D7
:1060F000FEF704FD3A88A3B29A4217D909FB03F3CD
:10610000D8F80020D55CD618042D0DD801A930464A
:10611000FEF738FD40B1019806F11001FFF724FFAA
:1061200001462846FFF748FB0134E3E703B0BDE82A
:10613000F08300BFC03E0030C43E00302DE9F3477D
:10614000DFF888904FF419621D496846FDF766FB39
:10615000B9F800502DB11B4B1A881B4B1B889A4273
:1061600026D00524174F184E4FF00008B9F80050FC
:106170001DB13A8833889A421AD0013C14F0FF04CA
:1061800016D04FF0000A002101A83D88CDF8048008
:10619000FFF72EFB1FFA8AF30AF1010A20B1002152
:1061A00001A8FFF79DFCF5E7A9F800303580DDE791
:1061B0006846FDF755FB284602B0BDE8F08700BFF2
:1061C0006C3E0030A83E0030B63E0030B23E00309B
:1061D000024A138801331380704700BFA83E003085
:1061E000F0B500230E4604462DED028B91B00593C9
:1061F00006AA0A9305A9CDE908330DF1110300930E
:1062000008ABFEF741FE0546D0B10699E1B10A7828
:106210002B8902F01F029DF811708DF81C30C3F31A
:1062200000201302059A43EA403343EA82339DF883
:106230001C201A43C3F30423052B07927BD02FB1F4
:1062400011B0BDEC028BF0BD0278E1E7012B05D166
:1062500021B10B8A590701D5FFF7BAFF27466EE037
:10626000BDF812204FF6FF739A42E9D09DF81D1039
:1062700001F01F01042925D99DF81D00BDF8122049
:1062800000F01F004149FEF7A7FE131849880833A4
:106290008B4248D20432104480B2FEF7B5FB9DF821
:1062A0001D0000F01F00FEF797FEBDF81210024619
:1062B0003846043189B2FEF791FB0422BDF8121072
:1062C00007A85FE02046FFF72FFC0699F0EE408A12
:1062D00071B10C31FFF748FEB0EE408AF0EE400A93
:1062E000B0EE680AFDF786FF28B1002EC4D1A7E7FB
:1062F00005F11001EEE7002EBED19DF81D3003F030
:106300001F03032BB8D038EEC88A9FED210AF0EEA8
:10631000E88AB0EEC88A68EE808AB4EEE88AF1EEC8
:1063200010FAA9D58CE71B4B1B491B68186C036836
:106330001B68984784E7002F90D0A4EB87071123B0
:10634000012229462046CDE902320BAB069A019381
:106350009DF81130009308ABFEF786FF0DF1120196
:1063600007A8FEF71DFF00283FF47AAF9DF81D0037
:1063700000F01F00FEF730FEBDF81210024638464E
:10638000043189B2FEF72AFB5AE700BFBC3E003059
:1063900017B7D138282A003000F905087FB5164D07
:1063A0002E1D4FF4BB72314601A8FDF737FA28685D
:1063B0000AF020FA042812D9052202A928680AF056
:1063C0002DFB431F5C425C4101A8FDF749FA44B133
:1063D00001229DF80C100298FFF702FFE1E700246C
:1063E000F2E7064B1B68186D03685B6B984708B1B2
:1063F000FFF7A4FE04B070BD883E0030282A0030AC
:10640000FFF7CCBF10B50446FDF7DAF8204610BD03
:1064100070B5134C0026204607F034FA2046114C84
:10642000114A124914F0FEFF204640F8046B07F0B1
:1064300029FA1420FDF7BEF805469B210AF088F9D9
:10644000094A0B492046256014F0ECFF3146094803
:1064500000F026F807210848BDE8704000F020B899
:106460006C3E0030883E0030E4CC0030C149040866
:10647000C5490408BC3E0030A43E003008B5064BB8
:106480001B68D86B03685B68984720B90348BDE870
:10649000084007F067BA08BD282A00302C19060802
:1064A0000023084A0170438030B514780333063264
:1064B0008C4201BF448832F8025C64194480362B58
:1064C000F3D130BD4C1906082DE9F84F194E074697
:1064D0008A461C4606F16C08DFF85C9031783B7800
:1064E000994204D1B588954209D8521B92B206361A
:1064F000B045F3D1B4FA84F04009BDE8F88F52FA00
:1065000084F1E3B2A9425146D8BF1D46D9F8003004
:10651000C8BFAD1AD86B7388C8BFEDB21A44036800
:1065200092B2D3F808B02B46D847641BE2D0AA44F5
:106530000022DCE74C190608282A00302DE9F84F24
:10654000194E074692461C4606F16C08DFF85C902F
:1065500032783B789A4204D1B5888D4209D8491BDC
:1065600089B20636B045F3D1B4FA84F04009BDE8EB
:10657000F88F51FA84F2E3B2AA425246D8BF1D46C0
:10658000D9F80030C8BF6D1AD86B7388C8BFEDB298
:106590001944036889B2D3F80CB02B46D847641B62
:1065A000E2D0AA440021DCE74C190608282A003072
:1065B0002DE9F041448888B04B880746884600257D
:1065C0009C4228BF1C46DCB1202C26462A46694640
:1065D00028BF202640463346FFF776FF18B9002033
:1065E00008B0BDE8F08133466A4629463846FFF7D1
:1065F000A5FF0028F3D0A41B3544A4B2ADB2E2E756
:106600000120EDE738B500254FF0FF330446303068
:1066100040F8043C40F81C5C40F8185C40F8145CFE
:1066200007F030F904F1640009F0E2FE0C4920465D
:10663000C4F88C50C4F89050C4F89450C4F8505129
:10664000C4F85451C4F85851FFF72EFD054B1A6891
:1066500012B1054809F01EFE20461C6038BD00BF7F
:10666000A81A0608C83E0030B8190608084699B1AD
:10667000C81FC3B2102B0ED810280CD8DFE800F0CA
:10668000090B090B0B0B0B090B0B0B0B090B090966
:10669000090000207047012070470000F8B52DED7B
:1066A000028B90F9023004460E46032B32D100F1E2
:1066B0002A073846FFF774F8054658BB94F92A3084
:1066C00038469FED298A013B07EE903A0123F8EE08
:1066D000E77A84F82A30F0EEE77AF4EEC87AF1EE41
:1066E00010FA4CBF19460021FEF762FF94F9023000
:1066F000204607EE903A00F8025FF8EEE77AF0EEF7
:10670000E77AF4EEC87AF1EE10FA4CBF01210021CD
:10671000FEF74EFF21782046FFF7A8FF30B1002298
:106720000521304603F098FAC4F804010025B3EEC1
:106730000E1AF1EE040A4FF4E17094ED090AA56017
:10674000FDF78CFDB7EE007A238A84F85850C7EE27
:10675000007A013B9BB2C72BBDEC028B84BFC823E0
:106760002382C4ED597AF8BD00000034A82310B587
:1067700001FB03340444647824B103FB0101D1F824
:1067800098301360204610BDA82310B501FB0334D8
:106790000444A47824B103FB0101D1F89C301360B8
:1067A000204610BDA82310B501FB03340444E4784F
:1067B00024B103FB0101D1F8A0301360204610BDC5
:1067C000A82303FB01032DE9F047D3F8B0200646C8
:1067D0000F4622B9D3E92E0150EA010335D04FF01C
:1067E000A80909FB0769B9F86040002C50D02A4875
:1067F0002A4DA4FB0048D9E92E23134330D007F1DA
:10680000400356F82310D1F848A0BAF1000F1ED16A
:10681000D1F838A009F072FD65194FF0A8024FF4C5
:106820007A7448F1490815EB0A0502FB0766A5FBD7
:10683000043548F1000804FB0855D6E92E24801AD7
:1068400061EB0401181845EB0101BDE8F0874FF436
:106850007A720023D1E91001F9F7C8FE8244D9E722
:10686000D9F85C004923401943F10003051948EBAE
:10687000030409F041FDD9F8B0104FF47A73401ABF
:10688000401944F10004A0FB030103FB0411DCE701
:1068900020462146D9E700BF00840C24B0F5F790CC
:1068A00038B5A82303FB0103B3F86040FCB14031C5
:1068B00050F821108D6C8DB9886B0E490E4BA4FBDE
:1068C0000114C9184FF47A7344F14904091844F1CA
:1068D0000004A1FB030103FB041138BD4FF47A72DD
:1068E0000023D1E91001F9F781FE2844E5E72046AD
:1068F0002146F2E700840C24B0F5F79000EBC101CB
:10690000C1F84421A1F8483170470000435609B24C
:10691000022B0BD1038D5B0708D500EBC100054BA3
:10692000C0F844312E23A0F84831704700EBC10075
:10693000014BF5E7D41B0608781A060838B500EBBA
:106940008105D5F80431FBB100EBC104B4F848214E
:10695000D2B11A681846126A9047D5F80431B4F8D3
:10696000482119688242CD6828BF0246D4F84411F4
:106970001846A847D4F844310344C4F84431B4F865
:106980004831181AA4F8480138BD00002DE9F04F2D
:1069900004460E4685B04FF0A80809F0ADFC4FF64E
:1069A000FF7208FB064302900020A3F8862083F8BC
:1069B0005900A3F88820A357092B00F01E81A3F1EA
:1069C0001602D2B2012A40F2188104EB8607D7F8EA
:1069D0000421002A00F011813822012108FB064819
:1069E0000B2B02FB064208F1580882F8111100F047
:1069F000C7800F2B00F0D0800A2B40F0D9804FF4D5
:106A0000CC70FCF7D7FDD7F8043142462146054645
:106A100001F090F83823029903FB0643D3F80C21C8
:106A20008A1AB2F5966F28D993F810214FF03809D9
:106A3000013209FB0649D2B2082A08BF002283F8B6
:106A40001021D7F804016E4A036899F810115B6AA7
:106A500052F821109847D7F8040100210368DB6D34
:106A60009847029BC9F80C3194F91330002B0DDDC7
:106A700065B931462046FFF749FF94F91330002BE2
:106A800004DD1DB931462046FFF758FF4FF0380BA3
:106A900006F128030BFB064904EBC30309F58979CA
:106AA0000393039B1B89002B40F0A580D7F80401BA
:106AB00003681B699847002800F09D80002D48D18D
:106AC000D7F8040103685B699847A35D5FFA80FA11
:106AD000013B012B0DD80BFB0643494A93F81031BB
:106AE00052F8233094F91320002A63D1B3F5164FDE
:106AF00069D2238D13F0010FA35DA3F1110314BF1D
:106B00004FF461324FF4E122012B70D80BFB0643A6
:106B10003B4993F8103151F82330934267D15146E5
:106B2000484601F0C5FE002861D0A3574FF49B6092
:106B3000112B0CBF4FF001094FF00209FCF73AFD91
:106B40004246CDF800902146D7F80431054601F0C1
:106B5000D1FFA8230122284603FB064383F85920CE
:106B600004EB0613029A1C46C7F80051DA644FF48E
:106B70007A63A4F8503005B0BDE8F04F02F0D2BE01
:106B80004FF4BC70FCF716FDD7F80431424621469D
:106B9000054600F0C7FA3DE74FF4C870FCF70AFD60
:106BA000D7F8043142462146054600F01FFD31E783
:106BB00005462FE7B3F5E13F9BD3228D510702D461
:106BC000B3F5613F95D15146484601F071FE00286A
:106BD0008FD04FF49B60FCF7EDFC0023424621462A
:106BE00000930546D7F8043101F084FF81E7002DBA
:106BF0003FF457AFADE7002DABD105B0BDE8F08F46
:106C0000581A06082DE9F84F435604460D46072B3F
:106C10000BD063B9A82101FB050484F859304FF665
:106C2000FF73A4F88630A4F88830BDE8F88F90F898
:106C30000A31CB40DA07F8D400EB81070FFA81F86C
:106C4000D7F800311BB9BDE8F84FFFF79FBE90F9A8
:106C50001330002B01DDFFF771FED7F800014FEA7A
:106C6000051A03689B689847834609F045FB06466A
:106C7000BBF1000F61D1A244DAF84C30C31AB3F56E
:106C80007A6FD2D94FF0A809594609FB05404A4608
:106C9000583015F091F909FB05424FF6FF734FF498
:106CA0007A6182F85850A2F88630A2F88830CAF883
:106CB0004C60AAF85010615D172903D8344BCB40C3
:106CC000DB070BD4D7F8000198BBA821002301FBF8
:106CD0000545C7F8003185F8593002E0012382F8F4
:106CE000593004EB0814B4F85030F52B4CD994F813
:106CF0005220B3F5FA6F02F1010284F8522094D2C7
:106D000094ED157A07EE903AB5EEC07AF1EE10FAEE
:106D100085BFF8EEE77ADFED1F6AF8EE677A67EE77
:106D2000A67A84BFDFED1C6AE7EE267AC4ED157AF9
:106D30007BE703685B689847C7E7A82707FB054719
:106D400097F8C03053B100234FF47A72D7E92E017F
:106D5000F9F74CFC0023064687F8C03004EB0A0321
:106D600004EB0511DA6CB21AA1F85020A821DE64F8
:106D700001FB054595F85920012AB2D994F86A21FA
:106D8000002AAED19E64ACE7002284F85220B7E717
:106D90000042C0000AD7A33C48E17A3F13B504463D
:106DA00000F1300140F2064201A8FCF737FD002156
:106DB0002046FFF727FFD4F8003113B1012384F8F0
:106DC000093101A8FCF74CFD02B010BD10B40C460F
:106DD00011461A463CB9D0F8000120B103685DF8AD
:106DE000044B5B6918475DF8044B704770B490F929
:106DF0000660044613467F2E0DD00A46F1B270BCE1
:106E0000FFF7E4BF172B0AD0D4F8000138B10368AC
:106E100070BC5B69184790F90030122BF2D170BC3E
:106E20007047000010B590F900300C460BB90020F7
:106E300010BDD0F8000118B9002301202370F7E736
:106E400003681B6998470028F1D1F5E72DE9F04167
:106E50009046CA0704460F461E4605D441461A46C8
:106E6000BDE8F041FFF7C2BFD0F84C31002B43D052
:106E7000D4F84C21C7F34105FF081378002B46D105
:106E8000D4F84C3106205F700123D4F84C1103FA7A
:106E900005F20B78134332460B70B423414613FBC3
:106EA0000503D4F84C01184415F078F8B32ED4F843
:106EB0004C3138D86A1C05EB4505C5EB05159A70B1
:106EC000D4F84C3106EB85059D80D4F84C118A78B6
:106ED000DAB1012308789340013B984215D18A88A2
:106EE00020460631FFF782FFD4F84C21002393702F
:106EF000D4F84C21137008E040F2D621012013F0A1
:106F000011FBC4F84C010028B2D1BDE8F0815178E2
:106F1000B94202D1EB40DB07B2D500239370D4F81D
:106F20004C211370ACE71A780F2ACED104229A7044
:106F30004FF43472D4F84C319A80C6E7174B10B432
:106F4000136049BBB0F92030002B0DDD07EE903AFD
:106F50009FED137AF8EEE77A67EE877AC2ED007A52
:106F600001205DF8044B7047D0F8003113B190F860
:106F7000591049B990F9000010B900231360EFE7E8
:106F8000431E58425841ECE7196818468C6A11466E
:106F900023465DF8044B18470020E2E7CDCCCC3DFA
:106FA0006F12833A90F809318B4209D9083130F9D0
:106FB0001100002804DDC828A8BFC82080B270478F
:106FC000C820704731BB90F92A301BBB90F90030C4
:106FD00003B3122B1BD0172BDFED0F7A9FED0F7A27
:106FE00047FE877A90F85230012B13D890ED157A2E
:106FF000B4EEE77AF1EE10FA0CD5D0F8C430042BD9
:1070000008D8D0F8000128B10368DB6A1847DFED23
:10701000027AE7E7002070470000754300005743FD
:1070200008B5034690F90E0040B1D3F8000128B12D
:1070300003681B6B984780F00100C0B208BD0000D8
:1070400031B9D0F8000118B1036811469B6C18479C
:1070500000207047012070470020704770470000F3
:1070600070470000014B01200B607047CDCC4C3EB7
:1070700001207047012070470120704700207047B1
:1070800070470000002070477047000006207047DE
:1070900000487047041C06087047000010B50446FD
:1070A000FCF78EFA204610BD70B586B004460E4639
:1070B000122201AD0021284614F07EFF0221642334
:1070C00003228DF804108DF806300D238DF80F1073
:1070D00004218DF8073001238DF80B208DF8101056
:1070E00007218DF8162094F866218DF812108DF87E
:1070F0000820D11800228DF80D308DF8116084F829
:107100006611E95C01330A44122BD2B2F9D16068EE
:1071100029468DF8152013220368DB68984706B0CE
:1071200070BD000010B5044602F078FB0F4B002143
:10713000204623600E4B84F866111A681B79C4F848
:107140006D2184F87131C4F8681184F86C1184F8E9
:107150005A10FFF7A9FF03212046FFF7A5FF09F00A
:10716000CBF86E30C4F86801204610BD141C060828
:1071700020F2050870B586B004460D46164600217B
:107180001422684614F018FF0223072103228DF809
:10719000003064238DF80B1006218DF802300F2388
:1071A0008DF807208DF8033001238DF80C100A218B
:1071B0008DF8142094F866218DF80D108DF80420B8
:1071C000D11800228DF809308DF80F308DF80E603F
:1071D00084F866118DF811501DF8031001330A442C
:1071E000142BD2B2F8D1606869468DF813201522AD
:1071F0000368DB68984706B070BD00008B1800205C
:1072000030B5DD790C46002165F307009D7965F303
:107210000F205D7965F317401D7965F31F60DD78F8
:1072200065F307019D785B7865F30F2163F31741E0
:10723000A35C63F31F6141EC100B30BD8818002381
:107240008A5C10B5C47864F307038478407864F3EB
:107250000F2360F3174362F31F6300EE103A10BD73
:107260008B18002010B5DC7864F307009C785B78FD
:1072700064F30F2063F317408B5C63F31F6010BD52
:107280008B184FF000005B7863F307008B5C63F3AF
:107290000F2080B2704700002DE9F04F2DED068BD6
:1072A00090F85D3083B00446402B40F0F080032519
:1072B00000269FED7B8B9FED7C9B9FED7DAB94F833
:1072C0005E30AB4240F2DD8004EB050A05F10208B6
:1072D0009AF85F709AF86090012F33D1D4F80CB00F
:1072E000424604F15F012046FFF7BAFFCBF80400E5
:1072F000D4F80CB0AA1D2046FFF7C2FFABF8080077
:10730000E3689AF8672083F832209AF86830E268D8
:1073100013F0010F14D09AF869300321DD07517082
:107320000AD5E26804219807517005D55907E2682B
:107330004CBF062305235370013609EB0805BEE751
:107340005770F9E7022F30D104F15F014246204621
:107350000191FFF753FF20EE080BE36805F10A02E5
:107360000199204620EE090BBDEEC00B83ED050A06
:10737000FFF744FF20EE080BE36805F112020199C4
:10738000204620EE090BBDEEC00B83ED060AFFF789
:1073900035FF20EE0A0BE368BDEEC00B83ED040A57
:1073A000E56808F0A9FFA865C6E7082F2DD104EB12
:1073B000080393F85F30DB07BED504F15F01E7688F
:1073C000EA1C2046DFED3C7A0191FFF737FFEA1D0A
:1073D000204687ED070AFFF731FF20EE270AE36812
:1073E000204683ED080A02F035FA05F10B020199F7
:1073F0002046FFF723FFB1EE400AE368012283ED48
:107400000F0AE36883F8502096E7092F10D1DFEDCB
:107410002B7AAA1D04F15F012046FFF70FFF20EE33
:10742000270AE368BCEEC00A10EE102ADA8583E76B
:107430000C2F82D104F15F01AA1D2046FFF7FEFE4A
:10744000F0EE407A05F10A022046FFF7F7FEE36806
:1074500037EE800A05F11202F6EE007A204620EEA1
:10746000270A83ED110AE768FFF7E8FE012387ED9D
:10747000120AE2681E4482F85230E26882F8533001
:107480005BE7052E4FF0010002D0E3685870002042
:1074900003B0BDEC068BBDE8F08F00BFAFF30080FA
:1074A000F8C1631ADCA54C4000000000D012634113
:1074B0000000000000005940E02E65420000C84274
:1074C00090F85A30013B052B04D8DFE803F0101B7D
:1074D0001F233944022908D140F20123A0F85A3071
:1074E0000023A0F8623180F8643100207047022345
:1074F00080F85C1080F85A3090F86431194480F8B4
:107500006411F2E7032380F85D10F3E7042380F8A9
:107510005E10EFE7B0F86231C218013382F85F10F5
:107520009BB290F86421A0F86231114490F85E207B
:107530009A4280F86411D8D8052380F85A30D4E7ED
:10754000062380F85F1180F85A3090F864318B423E
:10755000CBD1FFF7A1BE002380F86011EDE700005A
:1075600038B5044608F0C8FE054694F86C31042B83
:107570001BD8D4F86821824217D223440022204627
:107580006E3593F86D11FFF7F5FD94F86C31032219
:107590002046234493F86D11FFF7ECFD94F86C310D
:1075A000C4F86851013384F86C31002560680368C1
:1075B0001B69984750B1606803685B699847C1B21E
:1075C0002046FFF77DFF2843C5B2EFE7284638BDC8
:1075D0000620704700487047641C0608704700008A
:1075E00010B50446FBF7ECFF204610BD10B504466D
:1075F00002F014F9104B2360002384F8603084F803
:107600006C30C4E91933AA2384F8713141F2442360
:10761000A4F87231A36893F913305BB160680E224D
:1076200006490368DB6898476068222204490368BA
:10763000DB689847204610BD241D06086C1C060810
:107640007B1C060838B5B0F87921044690F87431EF
:10765000B0F875511A44D0F8811102F073F92A2D4F
:1076600040F0A780E368B4F87F211A81E368D4F87A
:1076700081215A60E56808F03FFE9FED7A7BA8659E
:10768000D4F87520D4F87930E16843EC162B26EE57
:10769000076BBDEEC66B81ED056AD4F87D20D4F88A
:1076A0008130E16843EC162B26EE077BBDEEC77BED
:1076B00081ED067AD4F88520D4F88930E1689FED11
:1076C0006B7B43EC162B26EE077BBDEEC77B81ED73
:1076D000047AE36894F8AE2083F83220D4F8952039
:1076E000E36807EE902AD4F8992007EE102A77EE87
:1076F000877AB6EE007A67EE877A9FED5E7AC3ED01
:10770000117AE368D4F89D209A640123E26882F834
:107710005230E26882F85330D4F8A510E26807EEE0
:10772000901A67EE877AFCEEE77AC2ED1E7AE2687D
:1077300094F8AE1082F87C10D4F86D10E268F9B9B4
:10774000D4F87130222B0FD81F2B30D8102B16D025
:107750000F2B07D9122B03D8102B03D004230FE0D3
:10776000142BFBD001230BE0322B02D003D8302B9B
:10777000F8D1062304E0443B012BEFD9F2E70323C1
:10778000537094F85A3043F0010384F85A3094F857
:107790005A309A07C3F3400063D5E268E16D52683E
:1077A000914224D123F0030384F85A3059E0052391
:1077B000E6E7632D1DD0AE2D4ED1D4F87520DFED58
:1077C0002E6A07EE102AE36827EE267ABCEEC77A07
:1077D00017EE102ADA85D4F87920E36807EE902AAC
:1077E00067EEA67AFCEEE77A17EE902A1A8600205A
:1077F00037E0D4F87D2004F16D05D4F881302046BF
:10780000E16843EC172BF7EEC77BC1ED077AD4F89C
:107810008520D4F88930E16843EC172BF7EEC77B5D
:10782000C1ED087A02F016F82A6A6B6AE06843EC48
:10783000172BF7EEC77B0122F1EE677AC0ED0F7AC6
:10784000E36883F85020D4F88131E36594F85A3026
:1078500043F0020384F85A3094F85A0010F0010003
:1078600095D138BD00000000D01263410000000037
:107870000000594000007A440000C8420823054A2D
:1078800001F00100490800B15140013BF8D1084620
:10789000704700BF2083B8EDF8B50546144656186A
:1078A000A6420AD014F8010B1F0A5840C1B228465C
:1078B000FFF7E4FF87EA0003F2E71846F8BD00008F
:1078C00038B590F86C300446013B082B06D8DFE849
:1078D00003F010191D26374C50586000AA2904BF28
:1078E000012380F86C30002380F88D3184F88E31CC
:1078F00004E0442904D1022384F86C30002038BD10
:107900000023F9E71229FBD10323F5E7042380F8CC
:10791000741180F86C3080F88D310023E6E7B0F800
:107920008D311B2BECD8C218013382F871119AB239
:10793000A0F88D3190F874319342DFD80523DBE74E
:10794000B0F88D31FF2BDBD890F874011A1A01338F
:10795000224482F86D109AB2A4F88D31B4F87931CE
:1079600003449A42CADB0623C6E70723C0F86D1119
:10797000C2E7D0F86D3103EB01210823C0F86D1187
:10798000BAE7D0F86D3103EB01410923C0F86D115E
:10799000B2E7D0F86D51002300F2711205EB0165DA
:1079A00080F86C3090F87411C0F86D51FFF774FFD7
:1079B00004F16D020346B4F879112046FFF76CFF1D
:1079C000854204D12046BDE83840FFF73BBEA36E98
:1079D0000133A36692E7000073B58368044693F908
:1079E0001330F3B108F088FC94F860300546052B9D
:1079F00017D8626E824214D2144AC835666852F8AB
:107A0000231008460191F9F721FA336802460199DB
:107A1000DB683046984794F860306566013384F837
:107A200060300025606803681B69984750B1606842
:107A300003685B699847C1B22046FFF741FF2843BE
:107A4000C5B2EFE7284602B070BD00BF041D0608AE
:107A50000620704700487047741D060801207047D3
:107A6000014B01200B6070470AD7A33D836F0120B3
:107A70000B607047836893F9133023B1006E031FC6
:107A8000584258417047012070470000836F13F43B
:107A9000746F0CBF012000207047000010B5044631
:107AA000406E12F043FD204610BD000010B50446A4
:107AB000FFF7F4FF2046FBF783FD204610BD0000D2
:107AC0008268436F92F90E2003F42073022A04D0D7
:107AD000A3F52073584258417047B3F5207F08D072
:107AE000064B1B685B6D93F89C3023B990F87C00C3
:107AF0007047012070470020704700BF282A0030DF
:107B000007B5836893F913307BB1026E042A0CD059
:107B1000C3684FF0030C197804230131CDE9003C10
:107B200090F85A300248FBF7EBF803B05DF804FB1D
:107B3000781D060810B5044601F070FE0B4B23605B
:107B40000B4BE3660023236784F87E3008F0D4FBF8
:107B5000E2680123A066204682F87D30A268128D7B
:107B6000920744BFE26882F82C3010BD3C20060822
:107B7000AC1D060870B5B0F8843040F6AE7204460D
:107B8000C3F30C03934200F043810AD840F6A1727C
:107B9000934200F02E8140F6A77293423AD0002023
:107BA00014E140F6BC72934200F0558141F2147228
:107BB0009342F4D1B0F88620D0F8881001F0C2FECC
:107BC000D4F8903007EE903AD4F8943007EE103A9B
:107BD000D4F8983000EE103AE368B4EE407AF1EE53
:107BE00010FA37FE000AF4EE407AF1EE10FA37FE92
:107BF000800ADFEDAC7AB4EEE70AF1EE10FAC0F2DB
:107C00002681012283F85120E46813F047FF84EDB8
:107C1000100AC4E7B0F88C304FF6FF7299B2914267
:107C200005D0C2681381C368D0F888205A60B4F8C0
:107C300086202046D4F8881001F084FEE56808F01C
:107C40005BFBDFED997AA865D4F8AC3007EE103A0B
:107C5000B4EEE77AF1EE10FA57DDE26801255363DE
:107C6000E368D4F8B0209A63D4F8B430E26807EE41
:107C7000903AF1EE677AC2ED0F7AE36883F85050DC
:107C8000E66896ED0E0AD6ED0D7A20EE000AA7EE14
:107C9000A70AFCF7BFFA86ED070AE368D3ED0D0AE1
:107CA00093ED0E0A13F0CEFEB7EEC00AE6689FED24
:107CB000777B20EE070BB7EEC00BFCF7B9FA0A2171
:107CC00086ED080AB4F8CE30E2684B43DFED776A00
:107CD0009367B4F8DA20E36807EE102AB8EE477A23
:107CE00027EE267A83ED117AB4F8DC20E36807EEFC
:107CF000902AF8EE677A67EEA67AC3ED127AE36807
:107D000083F85250E36883F85350D4F89020D4F8A5
:107D100094309FED607B43EC162BB4EEC76BF1EE15
:107D200010FA34DDE1689FED595B43EC172B9FEDB2
:107D30005B6B27EE057B27EE067BBDEEC77B81EDF7
:107D4000057AD4F89820D4F89C30E16843EC172BDE
:107D500027EE057B27EE067BBDEEC77B81ED067A1D
:107D6000D4F8A430D4F8A020E16843EC172BD4F861
:107D7000A830B7EEC77B07EE903A77EE677A9FEDB3
:107D80004C7A67EE877AFDEEE77AC1ED047A94F8D3
:107D9000CA30FF2B1CBFE26882F8323094F88E3074
:107DA00003F00F03082B09D8DFE803F005111411C5
:107DB000171A14171A00E36801225A7094F88E30CB
:107DC000012013F0400F0ED0E368587070BDE368D7
:107DD0000322F2E7E3680422EFE7E3680622ECE718
:107DE000E3680522E9E71B06F0D5E36802225A7032
:107DF000ECE7B0F88620D0F8881001F0A3FDE36826
:107E0000B4F89420DA85E368B4F896201A86C6E6BA
:107E1000B0F88620D0F8881001F094FDD4F89430A2
:107E2000A26F6367D4F8983082EA030111F4746F8B
:107E300009D0E16803F4746302F474621D480978A0
:107E40000131FAF75DFFD4F89830A367A7E6002068
:107E500083F85100BAE7B0F88620D0F8881001F016
:107E600071FD94F88E00E36830BB83F87C00E36812
:107E70009867E368C3F88400E368C3F88000E368A8
:107E8000C3F88800A2E700BFAFF30080F8C1631A0F
:107E9000DCA54C4000000000006A08C100000000A2
:107EA000D012634100000034005043C80AD7A33BFE
:107EB0000000C842BC1D060894F8902083F87C207E
:107EC0004FF6FF72B4F8BD30934216BF0A2200236A
:107ED0005343E2689FED2F7B9367D4F89420D4F846
:107EE0009830E56843EC162BB4EE476BF1EE10FAD0
:107EF00042D0D4F89C00D4F8A01041EC160BB4EE9C
:107F0000476BF1EE10FA37D0D4F8A400D4F8A810DB
:107F100041EC160BB4EE476BF1EE10FA2CD0B4F82E
:107F2000B8004FF6FF71884226D09FED1C6B43ECE2
:107F3000172B27EE067BBDEEC77B85ED217AD4F8A3
:107F40009C20D4F8A030E16843EC172B27EE067B89
:107F5000BDEEC77B81ED207AD4F8A420D4F8A830F8
:107F6000E1689FED107B43EC162B26EE077BBDEE00
:107F7000C77B81ED227A12E60020C5F88400E36811
:107F8000C3F88000E368C3F88800E36883F854000E
:107F90001CE700BFBBBDD7D9DF7CEBBD00000000F4
:107FA00000408F400000000000408FC02DE9F84FD6
:107FB00090F87E3004460D46013B082B06D8DFE8DA
:107FC00003F0404B4F575B63677DB200242908D113
:107FD000012380F87E300023A0F888310020BDE81E
:107FE000F88F90F88F314FB2DFF8F0914FF006081C
:107FF0005E1C00F5C57B0344F6B2032EB24680F842
:108000008F61A8BF4FF0030A83F88A715246594620
:1080100059F8040B14F030FB78B9042E06D1303F28
:10802000092FDBD9002384F88F31D7E7D6D93E2D2D
:10803000F8D1012384F89031F4E7B8F10108E5D1D3
:10804000F0E7402903D1022384F87E30C6E75229A5
:1080500040F09A800923F7E70323A0F88210F3E7A2
:10806000B0F88210042301EB0525A0F88250EBE75D
:108070000523A0F88410E7E7B0F88410062301EB8D
:108080000525A0F88450DFE70723A0F88610DBE77A
:10809000B0F8861001EB0525ADB2AB07A0F886500D
:1080A0000CBF08230023072D80F87E3096D80023CC
:1080B00080F87E30236F013323678FE7B0F8883173
:1080C000FF2B98BFC21803F1010398BF82F88810F4
:1080D0009BB2B0F88620A0F88831083A9342FFF6A8
:1080E0007DAFB3F5807F4FD800220221843008F0A5
:1080F00055FE0221024604F1860008F04FFEB4F856
:108100008610024604F18800083908F047FE002373
:1081100084F87E30B4F882308342CBD12046BDE86B
:10812000F84FFFF727BDB0F88821FE2A2CD8831816
:1081300001320A2992B283F88810A0F888217FF4CE
:108140004DAF8318002183F8881090F888303A2BBF
:108150001AD1466EC6B100F18A01053A304614F0D4
:108160008BFA054680B9304612F0E0F9236E656659
:10817000042B06D8DFE803F0030A0C1A28000123B9
:10818000236608F0B9F8A06600235DE70223F7E74D
:1081900094F85A300133DBB2032B84F85A30F0D90B
:1081A00003232366002384F85A30EAE794F85A3010
:1081B000A2680133DBB284F85A3092F90C200AB17C
:1081C000022BDED90423DBE701F0F6FF4FF4AF7298
:1081D0004FF4801101F0DCFFD3E700BF0C2006084C
:1081E0004068112201490368DB681847E81D06084A
:1081F00038B58368054693F90E303BB3406F10F4F1
:10820000007412D1EB68124819780131FAF778FD41
:10821000EB68104819780131FAF772FD2846FFF72C
:10822000DFFF85F87C40002038BDC30506D5EB682C
:10823000094819780131FAF763FDF4E710F080047A
:1082400004D1EB68054819780131F4E70120EBE728
:10825000FC1D06081C1E06083D1E0608561E0608C4
:1082600010B504460548FAF74BFD1322606804492F
:108270000368BDE81040DB68184700BF7C1E060895
:10828000901E0608F0B504464068002585B00368D6
:108290002E461B6998470746BD420BD060680135E2
:1082A00003685B699847C1B22046FFF77FFE06432B
:1082B000F6B2F1E7A36893F91320FAB1226E042A0B
:1082C00000F0938008F018F8E36D0546834215D25C
:1082D000A36E03F5FA63834213D2E06EF8F7B6FD9E
:1082E0000746606803681B6A9847B84206D360680F
:1082F0003A46E16E0368DB689847A566304605B0EC
:10830000F0BD94F89031002BF8D0636E2BBB236E38
:10831000042B22D8DFE803F00337444A6100D4E994
:108320000232606804F164051278134493F9222044
:10833000036803921B6E98473E493F4B039A0128FE
:1083400008BF0B463D49284600934FF4613305F0C2
:10835000F9FA013001D100236366606E0028CDD0A8
:10836000F8F774FD0546606803681B6A9847A842E1
:10837000C4D360682A46616E0368DB6898470023AF
:1083800084F89031BAE7D4E902322D4904F164004F
:1083900012781344012293F9223005F0D3FAD8E77A
:1083A00094F85A20274B53F8222009E0A36893F948
:1083B0000C30012B0AD0022B0CD0002BCDD1224A3D
:1083C000224904F1640005F0BDFAC2E794F85A208E
:1083D0001F4BE8E704232366BFE701F0EDFE93227D
:1083E0004FF4801101F0D4FEB7E793F90E30022B61
:1083F00084D1184B1B685B6D93F89C301BB1012333
:1084000084F87C307AE794F87C30002B3FF476AF28
:10841000636F9B057FF572AF07F06EFFE36D054656
:108420008342BFF46BAF05F57A752046FFF718FF5E
:10843000E56563E7A91E0608A41E0608B11E060826
:10844000D41E0608242006082D1F0608124106081F
:1084500000200608282A003006207047836893F918
:1084600013302BB1D0F8B804B0FA80F0400970474F
:1084700001207047004870478C20060870470000B4
:1084800090F8BC34812B08D81A0611D4033B012B79
:108490000ED9084B01200B607047FF2BF9D1054B1B
:1084A0000B60836893F91300B0FA80F040097047BD
:1084B000014BEFE7AE47613E8FC2F53D70470000CC
:1084C000002070470120704710B50446FBF778F88C
:1084D000204610BD10B40022D0F8B834012101FAB2
:1084E00002F41C420AD0C1680748097850F82220DB
:1084F000013106485DF8044BFAF702BC0132132A39
:10850000EDD15DF8044B70474C2206089420060814
:10851000C1F302710139C9B204299ABF014B585CF9
:10852000002070474422060830B5039C0A4491425B
:1085300009D011F8015B18782844C0B2187025786A
:1085400028442070F3E730BD2DE9F041044640682F
:1085500086B01D4603688846BDF8306017461B6A22
:10856000984706F1080398424FF000003AD3B5232C
:108570008DF813700DF10F0704228DF8103062236F
:108580000DF112018DF80E008DF80F0020468DF8C8
:1085900011300DF10E0300978DF81280ADF81460C4
:1085A000FFF7C2FF3246294620460097FFF7BCFF7F
:1085B0006068062204A90368DB6898476068324651
:1085C00029460368DB689847606801220DF10E01B7
:1085D0000368DB6898476068012239460368DB68F6
:1085E0009847012006B0BDE8F081000013B50446AD
:1085F000406803681B6A9847072806D900230621AC
:1086000020461A460093FFF79FFF02B010BD0000FE
:108610001FB590F88B34052B05D9FFF7E7FF002035
:1086200005B05DF804FB02238DF80C108DF80D20C9
:1086300006210093012203ABFFF786FFF0E700005D
:10864000F0B5044640681D4685B003680F461646DF
:108650001B6A98470A280FD90323012206212046C6
:10866000009303AB8DF80C708DF80D608DF80E50F3
:10867000FFF76AFF05B0F0BD0020FBE790F8CE34AD
:108680000133DBB280F8CE342BB990F86D2490F82A
:108690007214FFF7D5BF70470A2938B5054618464A
:1086A00063D004D801290AD0022964D038BD0D292D
:1086B000FCD1032AFAD14FF4802401232EE0122AA0
:1086C00035D8012AF2D9931E102BEFD801A454F803
:1086D00023F000BF3B870408478704081987040874
:1086E000AD8604085387040889870408AD8604080A
:1086F000AD860408AD860408AD860408AD8604087E
:10870000AD860408AD860408AD860408AD8604086D
:10871000AD8604085F87040801232024834239D1F1
:10872000D5F8B83423EA0403C5F8B834BEE7202AE4
:10873000BCD14FF400440523F0E795F8D24484F00F
:1087400001030224EAE795F8D24484F001030424EB
:10875000E4E795F8D24484F001030824DEE795F8B5
:10876000D24484F001031024D8E7092A10D00B2A40
:108770009CD18024DFE7102A01D0152A96D1AB685E
:108780004FF480749B7BC9E701234FF40054C5E785
:108790004024D0E72846FFF753FFD5F8B8342343E9
:1087A000C5F8B834012385F8D0347FE72DE9F047C8
:1087B00084B006460C46924690F8BC3402AF802B3B
:1087C00004D000200837BD46BDE8F087FFF7A0FEC3
:1087D00000238046C7E9003300F10F0370681FFAD9
:1087E00088F523F00703ADEB030D03681B6A0DF159
:1087F0000809984705F110039BB29842E1D3012381
:108800007C603C4608353B700723ADB242467B7026
:1088100003CC029004A80391514613F0BFFB4B46D2
:108820008A22062130460095FFF78EFECAE7000037
:108830007FB590F8BC3405460E460024802B14D139
:108840004068CDE9024403681B6A98470F280CD999
:1088500008238B220621284600936B44ADF808407C
:108860000396FFF771FE04B070BD2046FBE70000E1
:108870000C23092213B50446062100930A4BFFF787
:1088800063FE07F039FD94F88034C4F87C040133AA
:10889000064884F88034E3681978013102B0BDE8F5
:1088A0001040FAF72DBA00BFF0220608BC200608D7
:1088B00010B5002308248278082A0ED8DFE802F0D9
:1088C0000B051217202B37474D00622902D10223D6
:1088D000837002E08370B52901D0002042E08378E4
:1088E0000133F5E70323C17083700171F5E70423B9
:1088F0008370C37819440379C9B2C1701944F4E78D
:108900000523027901708370C3780B44DBB2C37016
:1089100013440371E1E706238370C3781944037994
:10892000C9B2C1701944002301714370D5E7C378FF
:10893000027819440379C9B2C170194443780171AE
:108940000133DBB29A424370C7D10723C0E7C27834
:1089500084708A42C1D08370ADE7027983708A4205
:10896000A9D1012010BD0000002307B504220A216F
:108970000093FFF7E9FD03B05DF804FB13B58368CE
:10898000044693F91330002B4AD0406803681B6AF1
:1089900098470D2844D9D4F8B834082B05D194F859
:1089A000D23413B10023C4F8B83494F88A345A1C72
:1089B00084F88A24152B00F29680DFE803F00B433D
:1089C0004B1349474D1119253A3F317D4F515456AC
:1089D00062693191072201212046FFF719FE73E0F9
:1089E0002022F8E7204602B0BDE81040FFF7FEBDA8
:1089F00094F8BC34FF2B13D10023302201210093C3
:108A00002046FFF7A1FD5FE0A36893F90C30022B2D
:108A100008D000231622062120460093FFF794FD7C
:108A200002B010BDD4F8B83423F48053C4F8B8347D
:108A3000F6E70023242200930621E1E700233E22EB
:108A40000093F9E7002308220093F5E70222C2E72A
:108A50000322C0E70622BEE71222BCE70422BAE7DF
:108A600009220A21B8E70B22FBE7A36893F90E302D
:108A700023B9D4F8B83423F48073D7E71022022145
:108A8000AAE7A36893F90E30002BF2D01522F6E77F
:108A900094F88C345BB9154B1B685B6D93F89C3074
:108AA0002BB9204602B0BDE81040FFF75DBFD4F8F7
:108AB000B83423F40073B9E794F8BC34802B0BD19D
:108AC0000B492046FFF7B4FE0028A9D194F88A3458
:108AD000013B84F88A34A3E7002371220093ABE7BB
:108AE00003220D2178E70023F3E700BF282A003096
:108AF0000100032010B5044600F090FE114BE16820
:108B000023604FF47F43A068A4F88A3441F6FF73D2
:108B1000C4F8B834FF2384F8BC349DF8083084F8D6
:108B2000CC34012384F8CF3484F8D13484F8D3349E
:108B3000002309781A46FDF7E1FE2046FFF71EFFE5
:108B4000204610BDA02206081FB5C36804468068F1
:108B50001978FEF727FA012306210822ADF80A301A
:108B60000023ADF808002046ADF80C3002AB0091B0
:108B7000FFF7EAFC04B010BDB0F86E24083200F034
:108B8000E1BE00002DE9F04F2DED028B90F872143C
:108B900095B00446052944D190F86D24012A01D0EE
:108BA000002023E090F85A30062B0CD00A2BF7D186
:108BB00090F85B30092B2FD00B2BF1D1D0F8B834C3
:108BC00023F0800325E090F85B30312B1DD012D8C4
:108BD000162B00F07281242B4FF0000000F038813A
:108BE000092BDDD184F8732484F8D00415B0BDECD2
:108BF000028BBDE8F08F3E2B00F05A81712BCFD154
:108C0000D0F8B83423F4803303E0D0F8B83423F438
:108C10008043C4F8B834C3E7D0F8B83423F0400335
:108C2000F7E706290FD190F86D24242A00F0DA80A6
:108C300072D8082A00F0678155D8002A00F05E81BA
:108C4000012A00F03F8194F872540A2D40F0CD8142
:108C500094F86D3403F0FD02092AA1D0042B40F0F2
:108C6000D181012304F2AB4604F28D472A4684F8F1
:108C70008C3404F17801304613F012FD1E2204F109
:108C80005A01384613F00CFDE3683246B8481978AB
:108C90003B460131FAF734F80822B649304613F062
:108CA000EBFCD8B92A46B449384613F0E5FC60B964
:108CB00094F8BC34802B1EBFD4F8B83443F480330E
:108CC000C4F8B834802384F8BC340A22AB4938464F
:108CD00013F0D2FC10B9812384F8BC34D4F8B83432
:108CE00023F0080395E7162AADD1836893F90C5059
:108CF000022D00F0E28090F85A30AB4200F0DD80A7
:108D0000034603F85A5F08250095FFF71DFCD4F8C9
:108D1000B83443F4805393E0712A00F00E818B2A1B
:108D200000F02E813E2A8ED1D0E902CE9EF800308E
:108D3000634493F90F20002A00F0BA8000F15A052D
:108D400005AE00F192092B46B0462868083555F863
:108D5000041C37464D4503C73E46F6D1286800211E
:108D60003860084642FA01F5ED0703D501291CBF1A
:108D70000130C0B201310729F4D1420094F85D50AE
:108D800000264FF0080A03922246B5427BDD9EF88A
:108D9000001092F85E70614491F90F00F1003841C3
:108DA00010F0010065D0012F59D094F85B90039822
:108DB000A9F1030B9BFBF0F094F8BCB4C0B2BBF17B
:108DC000040F82F85F0001D8022F4FD082F8609024
:108DD0002144D1F8620040F0010001360832C1F8A8
:108DE0006200D2E700238268A0F85A3092F901307D
:108DF0005E1C08D090F85C1099421EBF80F85C3071
:108E00000123A0F85A3092F90D30B4F85A0013F14A
:108E1000640F1BD094F966209A4217D040F00200EC
:108E200084F86630A4F85A00242204F15A0306217B
:108E300020460092FFF788FBD4F8B83443F48063EF
:108E4000C4F8B834012384F8D034A9E60028EBD163
:108E5000D4F8B83423F48063C4F8B834C6E64FF0CD
:108E6000030082F85F7082F86000B1E782F860A0CA
:108E7000AEE7214482F85F0082F86000D1F862001A
:108E800020F00100A9E719463C224046039313F065
:108E900075F8039B60B1ED003E22062120460435A3
:108EA0000095FFF751FBD4F8B83443F40063C7E7EB
:108EB000D4F8B83423F40063ABE6D4F8B83423F420
:108EC0008053A6E6B0F86E34082B10D190F88B349E
:108ED000052B02D9FFF78AFB62E6034490F85B207A
:108EE00090F85A1093F85C30FFF7D6FB58E690F8EC
:108EF0005C3090F85B2090F85A10F5E790F85A3003
:108F000080F88B344CE6D0E90213B0F85A201B7875
:108F1000083331F913309A4207D1C36D012B04D1C4
:108F2000D0F8B83423F0010373E62046FFF70CFEB7
:108F3000D4F8B83443F0010382E7B0F85C30002580
:108F400013F001030CD02823A0F85C50009300F12B
:108F50005A03FFF7F9FAD4F8B83443F480336FE7D3
:108F6000D0F8B82422F48032C0F8B82418E600BF44
:108F7000DC200608F4200608FD2006080821060863
:108F8000B0F86E5400F15E06B24F4FF00008043D99
:108F9000EDB2042D7FF657AED6F80090B94511D149
:108FA0003379EBB105AA394620468DF81480FFF7D6
:108FB000FDFB012384F8D034D4F8B83443F4803373
:108FC000C4F8B83449462046FFF7A2FA00283FF417
:108FD000E7ADC0F1FC0304301D440644EDB2D8E710
:108FE000D4F8B83423F48033EAE7022D0ED194F894
:108FF0006D34102B04D1A36893F90E3013B1CFE573
:10900000152BF8D02046FFF739FBC9E50D2D07D108
:10901000D4F86C34904A23F0FF039342F2D1BFE5B9
:10902000012DEFD194F86D24122A17D8012A1BD9EB
:10903000931E102B18D8DFE813F026009800BC0010
:109040001700CD00150117001700170017001700B3
:10905000170017001700170017000502202A00F05C
:10906000E681302A00F06C8294F8CE040130C5B25B
:1090700084F8CE54002D7FF493AD2B460121204679
:10908000FFF7DEFA8CE594F8D23433B1D4F8B83473
:1090900043F00203C4F8B83440E0D4F85A10204634
:1090A000FFF76AFDD4F85A30D4F85E200A21C4F8DC
:1090B0007834E368DFED696A9A61E368D4F8622086
:1090C0005A61D4F86A30E26893FBF1F31361E36804
:1090D00094F8CF245A70D4F86E2094F8CD3407EE6B
:1090E000102A43F00103B8EE477A84F8CD34E368E0
:1090F00027EE267A83ED117AD4F87220E36807EE22
:10910000902AF8EE677A67EEA67AC3ED127A012309
:10911000E26882F85230E26882F85330E36893F8EC
:10912000543063B107F0E8F8D4F8C834C01AB0F589
:10913000C87F40F23182E368002283F8542094F81B
:10914000CD34D9077FF52CAD9A07C3F340007FF5E6
:1091500027ADD4F87414D4F8782491427FF420AD6C
:1091600023F0030384F8CD3440E5D4F85A102046A8
:10917000FFF702FD94F8D23423B1D4F8B83443F0A9
:10918000040387E794F85F10E26811F0010F0BD039
:1091900094F85E30032B05D18A0700D5042384F8A8
:1091A000CF34BBE7022BFAD0012384F8CF345370BD
:1091B000B4E70023D4F85A10204684F8D134FFF7DE
:1091C000DBFCE368B4F86620DA85E368B4F8642071
:1091D0001A86A3E7D4F85A102046FFF7CDFC94F87E
:1091E000D234E2681BB1B4F86230138196E794F888
:1091F0006510CB0728D594F86430032B22D18F0754
:1092000000D5042384F8CF3494F8D1341BB1E3683B
:10921000B4F88620DA85E36894F8892083F8322050
:1092200094F8CF34012B7FF679AFE56807F064F846
:10923000A865E368D4F85A205A60E368B4F862205D
:109240001A816BE7022BDDD0012384F8CF345370F1
:10925000DAE700BF0100032000031C006F12833A0D
:10926000ACC527370125D4F85A10204684F8D254CB
:10927000FFF782FCD4F85A30D4F872200A21C4F8DF
:10928000C034C4F87834E3689A61E368D4F876208F
:109290005A61D4F87E30E26893FBF1F3136194F8DD
:1092A0006E30052B00F2C080DFE803F0BEBE039DE8
:1092B000B6BEE36802225A70E26801251FED198AE2
:1092C00053781FED190A84F8CF3494F8CD3443F065
:1092D000010384F8CD34D4F8823007EE903AF8EEEA
:1092E000677A67EE887AC2ED117AD4F88620E3684F
:1092F00007EE902AF8EE677A67EE887AC3ED127A65
:10930000E36883F85250E36883F85350E36894F8B5
:10931000712083F83220D4F89620D4F85A3007EE22
:10932000902AC4F87434F8EEE77AE36867EE887A36
:10933000C3ED077AD4F89A30E66807EE903AF8EE73
:10934000E77A27EE800AFAF773FF86ED080AE368EA
:1093500083F85050D4F88A20E36807EE902AF8EE9C
:10936000E77A67EE887AC3ED0D7AD4F88E20E36849
:1093700007EE902AF8EEE77A67EE887AC3ED0E7A68
:10938000D4F89220E36807EE902AF8EEE77A67EEC9
:10939000887AC3ED0F7AE36883F85150D4F89E20A1
:1093A000E36807EE902AF8EE677A27EE888A83ED65
:1093B000108A94F8CD3443F0020384F8CD3494F845
:1093C000D1343BB1E368B4F8A620DA85E368B4F899
:1093D000A6201A86E56806F08FFFA865E368D4F832
:1093E0005A205A609AE60322E3685A7094F86F3064
:1093F0009E0742BFE36804225A7094F86F305D06FE
:1094000042BFE36805225A7094F96F30002BBFF613
:1094100053AFE36806224EE794F86F106248F9F7FD
:109420006FFCE368032246E7E3685D7044E720468B
:10943000D4F85A10FFF7A0FB94F8653098077FF531
:109440006DAEFAE694F8D23423B1D4F8B83443F0D0
:1094500010031FE6D4F85A102046FFF78DFBD4F80E
:109460006E209FED528A07EE902AD4F85A309FED75
:10947000500AF8EE677AC4F87434E36867EE887AC5
:10948000C3ED077AD4F87230E56807EE903AF8EE4B
:10949000E77A27EE800AFAF7CBFE85ED080A012568
:1094A000E36883F85050D4F85E20E36807EE902A12
:1094B000F8EEE77A67EE887AC3ED0D7AD4F8622089
:1094C000E36807EE902AF8EEE77A67EE887AC3ED54
:1094D0000E7AD4F86620E36807EE902AF8EEE77A71
:1094E00067EE887AC3ED0F7AE368D3ED0D0A93ED4A
:1094F0000E0A12F0A7FADFED2F7AE66820EE270AAF
:10950000FAF796FE86ED080AE66806F1340007F0E1
:1095100059FC86ED070AE36883F85150D4F87620A9
:10952000E36807EE902AF8EE677A67EE887AC3ED73
:10953000107A94F8CD3443F0020384F8CD34EDE58D
:10954000D4F85A102046FFF717FB94F85F2002F07A
:109550000702022A84F8BC2413D8AAB1D4F8B8347C
:1095600023F40063C4F8B834D4F8B83430220121AD
:10957000204623F40073C4F8B8340023FFF760F8E2
:10958000CCE5D31E012BEFD90B4B0C491B68186C93
:1095900003681B689847E7E7D4F8C424D4F8C034BC
:1095A0009A427FF4FDAACAE5132106080AD7233C94
:1095B000ACC52737E02E6542282A0030272106084F
:1095C0002DE9F843044606F097FE0546D4F88434A6
:1095D000B4F88824C31A93426AD32046FFF7CEF921
:1095E000D4F8B834C4F88454002B36D094F8D2247C
:1095F00082BB13F0170F2DD04FF49673A4F8883464
:1096000060684FF0000808260368C14647461B699A
:109610009847B0F5005F28BF4FF4005085B21FFA9D
:1096200088F39D4240F2D880606803685B69984780
:109630000028C0F2D180C3B20621000280B294F8A3
:109640006C24082A3ED8DFE802F04238485263749E
:1096500095B2B90040F2EE23D0E74FF4FA63A4F8D4
:109660008834A36893F91230002BC9D094F873247E
:10967000002AC5D194F88024042AC1D8D4F87C04E7
:1096800041F288322D1A9542BAD9554A1268526D64
:1096900092F89C20002AB3D1012B05D0022BAFD128
:1096A00094F8D034002BABD02046FFF7E1F8A7E7C1
:1096B000D4F8B834002BA3D1D3E7622B05D1022311
:1096C00084F86C3408F10108A9E784F86C74B52BB0
:1096D000F8D194F86C340133F2E7032284F8723441
:1096E00084F86A3484F86C2484F86B34EAE7042242
:1096F00094F86B1484F86D3484F86C2494F86A241C
:109700001A44D2B284F86A240A4484F86B24D9E754
:10971000052294F86B14A4F86E3484F86C2494F841
:109720006A241A44D2B284F86A240A4484F86B2466
:10973000C8E794F86A2494F86BC41A4484F86C144B
:10974000D2B284F86A24624484F86B24B4F86E249C
:10975000024492B2B2F5826FA4F86E2404D9A4F840
:109760006E7484F86C746AE7A4F87074002AA9D146
:109770000723A5E794F86A2494F86B141A44D2B22C
:1097800084F86A240A4484F86B24B4F87024B2F58F
:10979000826F3CBF121982F85A30B4F87034B4F8B2
:1097A0006E2401339BB29A42A4F8703490E794F887
:1097B0006A2484F86C649A42D3D183E794F86B24CA
:1097C00084F86C749A427FF47DAF2046FFF7DAF993
:1097D000002818BF814675E74846BDE8F88300BFFA
:1097E000282A00300320704737B5054640681446E4
:1097F000019168B103681B6A9847A04208D968685C
:10980000224601990368DB6803B0BDE83040184781
:1098100003B030BD704700007047000010B504462B
:109820000B48C4E90212C4E9000364224FF4FA7140
:1098300004F1180000F02EFBE2680023204682F8B5
:109840005130E26882F85230E26882F8533010BD3D
:109850004023060838B5C5680446DFED137A2DEDC0
:10986000028B95ED088A28EE278AB0EE480A11F09F
:10987000DFFDD5ED077A27EE800A85ED0D0AB0EE03
:10988000480AE56811F0AEFF0022D5ED077A27EE11
:10989000800A85ED0E0AE368DA630022E36883F844
:1098A0005020BDEC028B38BD35FA8E3CF0B5C46853
:1098B0004FF0380C174E87B02578846836686F1CD7
:1098C0000CFB054E0368766D9EF811E15B6BCDE9EC
:1098D0000412BEF1000F12D00CFB054494F81041A5
:1098E00098470D4B53F824300097CDE90103DDE98B
:1098F00004120A4B3046FAF731F807B0F0BD98472A
:10990000074BCDE90070DDE904123046FAF726F87E
:10991000F3E700BF282A0030581A0608FC22060880
:109920001E23060800B58FB0332201A9FFF7BEFF42
:1099300001A90348F9F7E4F90FB05DF804FB00BF93
:10994000F12006082DE9F0432DED028B836B85B0E5
:10995000044689468B4200F09D808163D0E90487EC
:1099600058EA070321D0C3685B78012B1DD9002278
:109970000023C0E9042306F0BFFCE56C3223064651
:10998000C5F11905226DE0640544B5FBF3F55D43AF
:10999000636DAB4219D1B4F85830042B11D80133A0
:1099A000A4F85830236D0BBB15E0606830B1036834
:1099B00091B29B6F984780460F46DCE706F09EFC0D
:1099C000F9E79542EED02565ECE700236565A4F83C
:1099D0005830002A63D1E368A0681978FDF7E2FAED
:1099E000C822322100B2FAF76DFC2065236D04F124
:1099F000180005EB53024FF47A75B2FBF3F25A43A9
:109A0000D4E910136A43521843F10003CDE90087EB
:109A1000C4E9102300F042FAE3680122C3E9180107
:109A2000E36883F8682003AAE368A0681978FDF763
:109A300085FA08B3E5680023DFED1E7A4FF47A72E9
:109A40009DED038AD5E9180138EE278AF6F7CEFD99
:109A5000301A61EB4101F6F733FDDFED177A07EEBF
:109A6000100A67EE277AB4EEE78AF1EE10FA4ABFE1
:109A7000EB6E00230133EB66E3685B78012B09D9B9
:109A80004FF47A720023D4E91001F6F7AFFDA9EB89
:109A90000000A06405B0BDEC028BBDE8F0834FF47C
:109AA0007A7123682046DB6CB1FBF2F1C9B29847AA
:109AB00078E700BFCDCC4C3D6F12833A10B5044B14
:109AC000044604491860FCF7EFFA204610BD00BFB9
:109AD000CC3E00303824060810B590F8231089B920
:109AE000012380F82330084B1868F9F747FE036814
:109AF00080224FF4E131DC6A4FF40073A446BDE8E4
:109B00001040604710BD00BF282A0030002849DD02
:109B10006F283FD01BDC13283ED00EDC431E082BE1
:109B200011D8082B2CD8DFE803F03A052B2F2B2B6C
:109B30002B2B32004FF416607047392832D064283E
:109B400033D0262833D04FF47A7358437047B0F59A
:109B5000E67F2FD009DCE6282FD0B0F5807F2FD00C
:109B60007328F0D14FF4E130704740F299339842B6
:109B700029D040F2DC53984228D0B0F5FA7F27D0A4
:109B8000B0F5FA6FDFDD70474FF4965070474FF431
:109B9000165070470F4870474FF4964070474FF487
:109BA000966070474FF4614070470B4870474FF420
:109BB000164070474FF4E12070474FF46130704712
:109BC0004FF47A3070474FF4612070470348704774
:109BD0000348D8E7FCB10100A086010060E316004D
:109BE00020A10700914215D0CBB2581E012801D9FF
:109BF0002B2905D1511EC9B201290BD92B2A09D015
:109C0000053B012B08D8501FC0B201288CBF002093
:109C10000120704701207047002070472DE9F8436C
:109C200000250446894617462E4600F1060818F915
:109C3000352049462046FFF7D5FF38B1B74203D15A
:109C400004EBC500BDE8F8830136F6B20135042DFA
:109C5000EDD10020F6E7000038B50446FFF7DEFF3F
:109C6000054670B1011B084BC1F3C7011868F9F72D
:109C700085FD044618B10368A9885B6D98472046A6
:109C800038BD0446FBE700BF282A00300C4B70B5F6
:109C90001E6805460C46C9B23046F9F76FFD0368E9
:109CA00005EBC4055B6DA988984738B9306C22462E
:109CB00004490368BDE870401B68184770BD00BFC9
:109CC000282A0030902306082DE9F74390F9213027
:109CD0000646013305D0FF23012100F8213FFBF7A1
:109CE00067FC30463546FFF7F7FE684B0127DFF883
:109CF000A0911B680193F9B20198F9F73FFD05F1B6
:109D00000808044668B3B9B23046FFF7BFFF95F9BB
:109D10000E3001332C2B00F2B080DFE803F0221765
:109D20001717292C2E2E3838AE2CAE41AE4954725E
:109D3000AEAE7DAEAE86AE8EAEAEAEAEAE22AE9E58
:109D40009EAEAEAEAEAEAEAEAE9E1700A868FFF74A
:109D5000DDFE23680146DD6A4FF4807380222046D1
:109D6000A84701374546042FC5D103B0BDE8F083AD
:109D70000923AB60F5E73923FBE7A868FFF7C6FEC8
:109D8000236801464FF48072DD6A1023E7E77323EE
:109D90004FF4E131AB602368DD6A80231A46DEE7C9
:109DA00028460923002100F80E3FFBF701FCD8E705
:109DB00073234FF4E131AB602368DD6A80231A46D8
:109DC0002046A84712E06423102249462046AB6093
:109DD0002368DD6A2023A8472368022120465B6EA2
:109DE00098472368022120469B6E984723680121EB
:109DF0002046DB6E9847236800212046DB6D98479C
:109E0000AFE773234FF4E131AB602368DD6A1E23B3
:109E10001A462046A847EEE7A868FFF777FE2368B2
:109E20000146DD6A80231A46CAE7A868FFF76EFE7E
:109E300023680146DD6A802390E74046FBF7B0FCCB
:109E400008B97323AB60A868FFF760FE236801467A
:109E50004FF40072DD6A1023DBE74046FBF7A0FCFD
:109E600008B97323AB60A868FFF750FE236801466A
:109E70008022DD6A4FF48073CBE7A868FFF746FEC7
:109E80002368014620465B6A98476AE7282A003023
:109E9000A086010001804280704700002DE9F04358
:109EA000DDE9074C017EA71A6CEB030629B1D0E966
:109EB0000251AF4276EB010103DA0121C0E90276DB
:109EC00001764FF47A78B0F800E0D0E9025108FB4F
:109ED0000EFE551943EB01011EEB050941F1000887
:109EE000A14578EB0C0809DAB4EB0E046CF1000123
:109EF000A21A254661EB0303C0E90223438B0BB989
:109F0000C0E90476D0E904420133A7429BB276EB64
:109F1000020242884383B8BFC0E904769A4201BF77
:109F2000D0E90423C0E90223002343832846BDE887
:109F3000F083000000214FF0FF33002210B5436290
:109F4000044600F1300301600171C0F80510417250
:109F5000417600F59470D9707C3343F8742C43F843
:109F6000702C43F86C2C43F8682C43F8642C43F8AD
:109F7000602C43F85C2C43F8582C43F8542C43F8DD
:109F8000402C43F83C2C43F8382C43F8342C43F84D
:109F9000302C43F82C2C43F8282C43F8242C43F87D
:109FA000202C43F8102C43F80C2C43F8082C984232
:109FB000D1D1054B1A6822B9044920461C60FCF730
:109FC00073F8204610BD00BFD03E0030C4250608FF
:109FD00090F8321029B90123438611708375184611
:109FE00070470020704700004FF0000070470000ED
:109FF00049B1037D012B06D05A1C0433027540F889
:10A0000023100120704700207047000038B5044637
:10A0100090F9150008B394F84301F0B10025227DB2
:10A02000EBB29A4207D90433013554F82300036890
:10A030009B689847F3E706F05FF9D4F89030C31AAD
:10A04000B3F5FA7F94F928312CBF0020012084F861
:10A05000310013B1002384F8443138BD024690F931
:10A060001500B0B192F8430198B1D2ED177A9FED87
:10A07000097AF4EEC77AF1EE10FA09D4B7EE087A4D
:10A08000F4EEC77AF1EE10FAD4BF01200020704739
:10A0900000207047ABAA2A3F014B1868704700BFE9
:10A0A000D03E003010B50446006810B103685B680C
:10A0B0009847204610BD000010B50446006810B156
:10A0C00003685B689847204610BD000030B5D0F8A3
:10A0D000345185B0044615F480351FD1174B01A8C3
:10A0E000174A1B68196B0B681B689847019B042271
:10A0F000294603A80393CDE9015507F003FD014666
:10A100002046FFF775FF03A8FFF7D6FF02A8FFF769
:10A11000D3FF019810B103685B689847237D0BB1AA
:10A12000A37D4BB9054B07491B68186C03681B6876
:10A1300005B0BDE83040184705B030BD282A0030D2
:10A1400034F805086425060810B590F91530044662
:10A15000A3B1036E8366837D8BB10C4B64211B68B6
:10A16000186D03685B6898472046FFF74FFF94F827
:10A17000323003B92366012384F8433110BDFFF761
:10A18000A5FFA37D002BF2D0E7E700BF282A00300F
:10A1900010B50368028119434368013301604360CD
:10A1A000044B1B685C6DA162596D406888855B6DCE
:10A1B000DA8510BD282A003000487047D43E0030B0
:10A1C00070B5732204464FF400010E48FFF7E0FF1C
:10A1D0000D4E0E4B1D6833783BB9686D0422214645
:10A1E000483006F091F8012333706B6D2A2283F812
:10A1F00046206B6D93F89C301BB92146044806F04D
:10A2000049F870BDD43E0030E03E0030282A0030CE
:10A21000B426060810B5832204464FF08061094831
:10A22000FFF7B6FF084B1B685B6D93F89C303BB99A
:10A230002146064803F096FB2146054806F02AF819
:10A2400010BD00BFD43E0030282A0030C8260608C2
:10A25000E426060810B40123417B094A8B401268AA
:10A2600013420AD1074B1B68DB6C1A685469428998
:10A27000184623465DF8044B18475DF8044B7047B9
:10A28000F03E0030282A003010B5054C2068FFF75A
:10A29000E1FF2068BDE810401430FFF7DBBF00BFCE
:10A2A000183F003001289FBF054B00EB80001B6862
:10A2B00003EB800094BFB0F908000020704700BF96
:10A2C000183F0030037B9B0735D4B0F90830572B7B
:10A2D00032DC452B07DC0B2B3ED015DC032B10DCCE
:10A2E000012B39DC7047463B112B24D8DFE803F003
:10A2F0003423233434141414141414372323232341
:10A300001414042B17D107E0202B0EDC1E2B26DCA7
:10A31000152B05DC0F2B0EDD41F2941107F0C6BCA6
:10A32000183B9BB2022BF7D97047292B17D02D3B36
:10A330009BB2022BF0D970476E2B0DD003DC5E3B35
:10A340009BB20F2BF6E77E2B09D003DC7C3B9BB244
:10A35000012BEFE77F2BD5E7642107F0AFBC4FF46B
:10A360007A71FAE708B503888B4208D8FFF724FF13
:10A370002E224FF40031BDE80840FFF709BF4B091A
:10A3800001F01F0100EB8300012303FA01F1436890
:10A390000B43436008BD00002DE9F041DFF89880D1
:10A3A000D8F80070AFB320480021204C4288043018
:10A3B000920011F001FE00231A4644F833200133C5
:10A3C0008C2BFAD13E891A4D8B2E2A6023D8384621
:10A3D000FFF778FF31461448FFF7C4FF54F83630D2
:10A3E00043F0010344F83630D8F80000868B8B2EFA
:10A3F00014D81430FFF766FF31460B48FFF7B2FF61
:10A4000054F8363043F0020344F83630094B012249
:10A410001A70BDE8F08101232B60E5E72B6843F05B
:10A4200002032B60F2E700BFF43E00301C3F003017
:10A43000EC3E0030E83E0030183F0030234B2DE961
:10A44000F0471E680025224B4FF00108F06C1A6897
:10A450000368204FDFF88090D3F88C30D18D984777
:10A46000FFF79AFF3C68F06C2C44D0F800C02389B9
:10A47000617B8B2B1DD808FA01F2D9F800301A4203
:10A4800017D1DCF80C309847B4F90830862B13D17B
:10A4900000222188204607F0FBFB2046FFF7DAFE6A
:10A4A0001435282DDED1F06C0368BDE8F0475B6AF7
:10A4B0001847DCF81030E6E7872B02D10022A1888C
:10A4C000E8E7882BECD100226188E3E7282A0030F6
:10A4D000E43E0030183F0030F03E0030074B10B52E
:10A4E0001B7804460BB9FFF757FFA3B28B2B95BF20
:10A4F000034B044B53F83400186810BDE83E00309D
:10A500001C3F0030EC3E00300A4B10B51B7804466F
:10A510000BB9FFF741FFC4F34A12074B012004F0C7
:10A520001F0403EB820300FA04F45B681C4208BFBB
:10A53000002010BDE83E0030F43E003070B5061D2E
:10A5400004460D4D304607F015FB04F1180007F0E6
:10A5500011FB04F1380003F095F9084B2046084937
:10A560001C602E60FBF7A0FD2B68002220465A736A
:10A57000012283F8212070BD183F0030E43E0030F6
:10A5800024270608354B70B5354E2DED028B9FED17
:10A59000358A82B01C6804B3D4ED027AF4EEC87A2E
:10A5A000F1EE10FA11DBB4F9005040F2B710D4ED1F
:10A5B000010A06EBC50537EEA01A95ED010A70EE0B
:10A5C000E70AF9F74BFE85ED010AB4F9003006EB16
:10A5D000C3035B686360E468DDE7234B4FF4DE721E
:10A5E000224D01A81968224E3831F9F717F92B8846
:10A5F0006BB332680121013BD1742B803068038931
:10A60000B0F908208B2B06D8154B03EBC20393ED52
:10A61000010A07F073FB6B883068DBB10122013B54
:10A6200080F827206B80838BB0F91C208B2B07D8F8
:10A630000B4B143003EBC20393ED010A07F05EFBF2
:10A6400001A8F9F70DF902B0BDEC028B70BD3368BB
:10A65000DC74D3E780F82730E5E700BF143F003013
:10A660001C3F003000000034E43E00300E3F00305C
:10A67000183F0030024B1B68D86C03681B6B1847EF
:10A68000282A0030024B1B68D86C03685B6B1847A4
:10A69000282A003010B50446FFF704FE01300BD025
:10A6A000064B186838B1012202FA04F3426B1342D8
:10A6B00014BF0120002010BD0120FCE7E43E003063
:10A6C00003481422034B002140F8043B11F074BCF2
:10A6D000F43E00308C00050010B506490446FBF737
:10A6E000E3FC054B1A6812B1044805F0D3FD20467F
:10A6F0001C6010BD342806087C430030B0270608D3
:10A7000038B50D4C0D4D237845F82310486055F8A9
:10A71000230003689B689847237850B955F82300B5
:10A7200010B103685B6898472378002245F823201E
:10A7300038BD01332370FBE780430030A443003071
:10A740002DE9F74F6F4D04462B78002B00F0D48095
:10A7500003B0BDE8F08FA3683B40802B00F09180F0
:10A7600058D8082B00F0B2803FD8022B62D0042BBF
:10A770006FD0013E4FEA4707EDD11420F8F71AFFDA
:10A7800014223146074611F017FC5F4B394620462C
:10A790003B6044F620633B82FFF7B2FF2B78052B2A
:10A7A000D6D81C20F8F706FF584B0146036040F648
:10A7B000E44303832046FFF7A3FF2B78052BC7D87C
:10A7C000B420F8F7F7FE05463146B42211F0F4FB49
:10A7D00028464F4B40F8143B03F054F829462046D6
:10A7E00003B0BDE8F04FFFF78BBF402BC1D1D8F8C5
:10A7F00000304FF0000AD86A0368DB6898470346C8
:10A8000009FA0AF21A422AD10AF1010ABAF1200F12
:10A81000F6D1AEE7B3F5007F60D0B3F5805F64D0CA
:10A82000B3F5807FA5D16820F8F7C4FE019000F051
:10A830000DFF51E05820F8F7BDFE0021824601F0DF
:10A8400047FE51462046FFF75BFF2B78052B90D93A
:10A850007EE75820F8F7AEFE01218246EFE7582048
:10A860000193F8F7A7FE83465FFA8AF100F0E0FD56
:10A8700059462046FFF744FF2A78019B052AC3D991
:10A8800066E7D8F800304FF0000AD86A03681B6901
:10A890009847034609FA0AF21A4205D10AF1010A59
:10A8A000BAF1200FF6D164E758200193F8F782FE41
:10A8B00083465FFA8AF100F0BBFD59462046FFF758
:10A8C0001FFF2A78019B052AE8D941E75420F8F7B1
:10A8D00071FE019000F0D6FE0199B3E76820F8F709
:10A8E00069FE019000F0F6FFF6E75C20F8F762FEE3
:10A8F000019000F0FFFFEFE701270D26DFF814803D
:10A90000B94636E780430030E02B060804290608E4
:10A9100094310608282A003010B51C220446002174
:10A92000054811F049FB054B002220461A60BDE89E
:10A930001040FFF705BF00BF81430030A043003047
:10A9400070B50024084D094E2A78E3B29A4207D91F
:10A9500056F8230010B10368DB6898470134F3E729
:10A96000034B00221A6070BD80430030A4430030C6
:10A97000A04300302DE9F74F05460E46174698468E
:10A980000024DFF83490DFF834A099F80020E3B217
:10A990009A420DD95AF8230040B103683246CDF8E7
:10A9A00000802946D3F81CB03B46D8470134ECE779
:10A9B00003B0BDE8F08F00BF80430030A4430030F7
:10A9C0000378013BDBB2022B9ABF024AD05600202B
:10A9D000704700BF30280608014B1868704700BF59
:10A9E0007C43003070470000704700007047000053
:10A9F00070470000704700007047000010B5044623
:10AA0000F8F7DEFD204610BD1B4B10B51B78044641
:10AA1000D90702D54FF0004314E005F06DFC6369DF
:10AA2000C01A238B984226D3144A237A1179C3F390
:10AA3000800088420BD061F382035A072372E9D564
:10AA40006FF00303E36005F057FC606113E0D17B16
:10AA5000C3F30010884206D061F304132372DB06AF
:10AA600009D5074BEEE7D37D13B14FF02043E9E75B
:10AA7000D37A002BCED110BDA043003081430030EB
:10AA8000000040ED10B4037A03F001028A4215D0B1
:10AA900061F30003037243681A7B0A4B1B685B6C0B
:10AAA00019680C69017C007AC007184623465DF8D6
:10AAB000044B5CBFB2FA82F2520918475DF8044BAE
:10AAC000704700BF282A003010B54368044693F948
:10AAD00002200AB9002010BD597901740029F9D06B
:10AAE0000B4B01221B68586C03685B689847002178
:10AAF0002046FFF7C7FF074B227A0120197961F33F
:10AB000082022272DA7A237A62F3C3032372E2E7C3
:10AB1000282A00308143003010B5C368044663B171
:10AB200005F0EAFB6369C01AB0F5486F06D300214F
:10AB30002046FFF7A7FF0023E36010BD6423B0FBAE
:10AB4000F3F04FF0004323FA00F0E3681842204688
:10AB500014BF01210021BDE81040FFF793BF0000A2
:10AB600010B50446FFF750FF2046BDE81040FFF740
:10AB7000D3BF00007047000010B50446F8F720FD71
:10AB8000204610BD2DE9F84F924603EB8303144A8B
:10AB900080468946002402EB030B052C09EB0407D1
:10ABA0004FF0000514BF1BF804600026BFB2D8F8B0
:10ABB0000800F1070AEB050205F1010503683946B3
:10ABC00092B248BF5B684FEA560658BF9B689847E9
:10ABD000082DECD10134062CDFD1BDE8F88F00BF81
:10ABE000FC290608F8B506460C4617465D1E15F901
:10ABF000011F79B120393A463046C9B25E2998BF63
:10AC00004BB2214604F1070488BF0023FFF7BAFFC7
:10AC1000A4B2ECE7F8BD000001EB8101054B4A004E
:10AC20001979063219B1044B0021FFF7DBBF034B42
:10AC3000FBE700BF81430030282906083B290608AE
:10AC400001EB8101054B4A009979063219B1044B99
:10AC50000021FFF7C7BF034BFBE700BF8143003074
:10AC60005029060863290608174A30B5537889B079
:10AC700005460C46062B22D8DFE803F023041719FB
:10AC80001B1D1F00114B927804EB8404132103A8B1
:10AC900000920F4A02F00CFE03AB6200002128462E
:10ACA0000632FFF79FFF09B030BD0A4BEBE70A4BB6
:10ACB000E9E70A4BE7E70A4BE5E70A4BE3E70A4B0C
:10ACC000E1E70A4BDFE700BF814300309629060821
:10ACD0009C2906088429060887290608E41906081D
:10ACE0008A29060890290608782906087E29060878
:10ACF00001EB8101054B4A00D97B063219B1044BA7
:10AD00000021FFF76FBF034BFBE700BF814300301B
:10AD1000B0290608BD29060870B58AB00C4606465B
:10AD200006F07AF803680DF11301002205461B684E
:10AD300098470146D0B10021284606F05FF8B7EEEB
:10AD4000C00A9DF8133013210F4A05A802938DED18
:10AD5000000B02F0ADFD04EB840405AB002130468E
:10AD600062000632FFF73EFF0AB070BD284606F0CB
:10AD700045F8B7EEC00A054A132105A88DED000B72
:10AD800002F096FDE7E700BFCC290608DE29060899
:10AD900030B50C4687B04368054604EB8404074A87
:10ADA0004833132101A802F083FD01AB62000021AA
:10ADB00028460632FFF716FF07B030BDF029060817
:10ADC00070B5002686B00C46054631460F2202A813
:10ADD00004EB840411F0F0F81222202101A811F0F4
:10ADE000EBF801AB620031462846AE810632FFF730
:10ADF000F9FE06B070BD000070B5002594B00446A1
:10AE00000F220E4603A82946029511F0D5F82F22ED
:10AE1000294608A8079511F0CFF805F06DFA636888
:10AE20005A6C801A228A904205D331462046FFF799
:10AE3000C7FF14B070BD627B12B1013A6273F8E7CC
:10AE40000F33164A332107A802F032FD12222021C7
:10AE500002A811F0B1F807AB257B591908460191FA
:10AE6000F5F7F4FF0646C2B2019902A8122A28BFDC
:10AE7000122211F093F8122E4FF006024FF000014B
:10AE800094BF4FF480630135204698BFA38102AB85
:10AE900088BF2573FFF7A6FECBE700BFF1200608A9
:10AEA00010B504460021FFF7A7FF01212046FFF758
:10AEB0006FFF20460221FFF72FFF20460321FFF7F7
:10AEC000D3FE20460421FFF7BBFE20460521BDE846
:10AED0001040FFF70DBF0000164A10B51378044666
:10AEE000182B02D80133137010BD00231370124ABF
:10AEF000837B12798AB1012BF6D080680368DB6806
:10AF0000984703212046FFF787FE0123A373A0681B
:10AF10000368BDE810401B681847022B05D0806805
:10AF20000368DB6898470223A3732046FFF7B8FF46
:10AF3000EDE700BFBC430030814300302DE9F04F06
:10AF4000856889B004463DBB304B4FF0010ADFF8FD
:10AF5000C0901E68F06A03689B68984707460AFA23
:10AF600005F33B4207D10135202DF8D1A06860B927
:10AF700009B0BDE8F08F636893F90330012B0DD061
:10AF8000022B2CD0A368002BEDD02046FFF788FFC2
:10AF9000A06803681B6898470120E9E7F16A4FF051
:10AFA0000008042207A80B68CDF80090CDE90182C3
:10AFB000EAB2D3F800B03C23D847079B05A8059315
:10AFC000CDE9068800F0B2F9A06005A8FFF774F893
:10AFD00006A8FFF771F807A8FFF764F8D2E7F16A4F
:10AFE0004FF00008042207A80B68CDF80090CDE9C7
:10AFF0000182EAB2D3F800B03C23D847079B05A8EA
:10B000000593CDE9068800F09BF8DDE7282A00309B
:10B01000801A0600012380F828347047054B10B5CC
:10B0200004460360406810B103685B689847204697
:10B0300010BD00BF0C2C060810B50446FFF7EEFF4C
:10B040002046F8F7BDFA204610BD00004FF4846298
:10B050000021083010F0B0BFF0B58DB0224B04468F
:10B0600005AA03F1180716461868083353F8041C9C
:10B070001546BB4203C52A46F6D119884FF48462AF
:10B080009B7804F1080029800021AB7010F094FF38
:10B09000606818B9002528460DB0F0BD03685B6AEA
:10B0A000984703689B6898476068002331460268A8
:10B0B000009315691B22A8470546606803685B6A10
:10B0C00098470368DB689847002DE3D00123606848
:10B0D000224644F6206184F82834036803949E6A6B
:10B0E000024B0493B047D6E728F205080DB20408D6
:10B0F000832910B50ED83F2A0CD8D308842402F037
:10B10000070204FB03110123084403FA02F2037A45
:10B110001A43027210BD0000832910B50ED83F2AD1
:10B120000CD8D308842402F0070204FB0311012386
:10B1300008449340027A22EA0302027210BD000022
:10B1400038B500230568036040F22C40F8F732FA66
:10B15000074B0446C0E90035FFF77EFF054620B9DE
:10B16000236820462C465B699847204638BD00BFBF
:10B170000C2C06082DE9F04190F8283494B00446D0
:10B18000002B3DD02049002504F10807432280F818
:10B1900028541F3151F8040C029003A810F0FEFE51
:10B1A00065F04F036068002604228DF80B3002A979
:10B1B000036801350096D3F810803346C0473946FE
:10B1C00042220DF10D0010F0E9FE6068432203A950
:10B1D00003680096D3F810803346C04742220DF131
:10B1E0000D00B918843710F0D9FE6068432203A916
:10B1F00003680096D3F810803346C047082DCFD19E
:10B2000014B0BDE8F08100BF28F20508FFF7B2BF17
:10B21000012380F808347047054B10B504460360DD
:10B22000406810B103685B689847204610BD00BFB6
:10B23000302C060810B50446FFF7EEFF2046F8F75D
:10B24000BFF9204610BD00004FF480620021083095
:10B2500010F0B2BEF0B58DB0204B044604AA03F145
:10B26000200716461868083353F8041C1546BB42DD
:10B2700003C52A46F6D14FF48062002104F108008C
:10B2800010F09AFE606818B9002528460DB0F0BD90
:10B2900003685B6A984703689B6898476068002367
:10B2A00031460268009315692022A8470546606868
:10B2B00003685B6A98470368DB689847002DE3D012
:10B2C00001236068224644F6206184F8083403684C
:10B2D00002949E6A024B0393B047D6E78CF20508AE
:10B2E00015B404087F290DD83F2A0BD8D30802F0E3
:10B2F000070201EBC3110123084403FA02F2037AA7
:10B300001A430272704700007F290DD83F2A0BD8DC
:10B31000D30802F0070201EBC31101230844934054
:10B32000027A22EA030202727047000038B5002355
:10B330000568036040F20C40F8F73CF9074B0446FF
:10B34000C0E90035FFF786FF054620B9236820468F
:10B350002C465B699847204638BD00BF302C060854
:10B360002DE9F04390F8083497B00646002B4CD0F6
:10B370002749002506F108078A8CA84680F808545A
:10B38000273151F8070C11F8013C039005A8ADF8DE
:10B39000102041228DF8123010F000FE7068072254
:10B3A0008DF8115003A90368CDF800801C690023B3
:10B3B000A0473C460DF1150307F1400254F8041B69
:10B3C000944243F8041BF9D17068412205A903682F
:10B3D000CDF80080D3F810900023C8470DF1150375
:10B3E00004F1400254F8041B944243F8041BF9D1C1
:10B3F00070680135412205A903688037CDF80080C7
:10B400001C690023A047082DC8D117B0BDE8F08300
:10B410008CF20508FFF7A4BF80F85230012380F8B2
:10B42000501080F8512080F85330184670470000C3
:10B430000F2337B50D4600931F2218230021044621
:10B4400000F0DEFB044B204684F8545023600023B8
:10B45000E36403B030BD00BF542C06081FB51F23A2
:10B46000C2EB022201F0E001C06CB2FBF3F21A4021
:10B4700000230A4303A98DF80C2002680093146985
:10B480000122A04704B010BD70B506464D1E4024F1
:10B4900015F8012F21463046FFF7E0FF18B12034A0
:10B4A000E4B2A02CF4D170BD90F8533001462BB11A
:10B4B0000023503180F85330FFF7E6BF704700009B
:10B4C000FFF7F2BF044B10B5044640F84C3BFEF7C3
:10B4D000E9FD204610BD00BF542C060810B50446F7
:10B4E000FFF7F0FF2046F8F76BF8204610BD00008C
:10B4F0002DE9F04B43F638138AB004464FF00208AA
:10B50000ADF818300DF11809354B08AE354F1B68F2
:10B510000593059B002504223046D96A0B680097E5
:10B52000CDE9015294F85420D3F800B019F8013B4A
:10B53000D847089BE06C0895E36410B103685B682A
:10B5400098473046FEF7AEFDE06CC0B103685B6A19
:10B55000984703689B689847E06C0A2103689B6CD6
:10B5600098471F2220212046FFF778FF054670B933
:10B57000E06C03685B6A98470368DB689847B8F13A
:10B58000010F01D1002526E04FF00108C1E7E37A61
:10B5900007A920468DF81C308DF81D308DF81E301F
:10B5A000FFF772FF0746E06C012103689B6C984728
:10B5B000E06C03685B6A98470368DB68984757B19B
:10B5C000E06C44F6206103689F6A074B0894099376
:10B5D00096E80C00B84728460AB0BDE8F08B00BFDB
:10B5E000282A0030801A0600C1B404087047000001
:10B5F000F8B506467824002527B23846FEF784FFC2
:10B6000020B13846FEF76AFF284385B20134A4B260
:10B610007C2CF1D185B10023084F25FA03F25C1C84
:10B6200012F0010F05D07368E1B238469A7B01F041
:10B630000BF8102C2346F0D12846F8BDBD4300304E
:10B6400010B50446F7F7BCFF204610BD3323FF2298
:10B6500013B50446009300217F2300F06DFC024BDC
:10B660002046236002B010BD8C2C060880F85230B2
:10B67000012380F8501080F8512080F8533018468C
:10B68000704700004F23002213B5FF2100937F2352
:10B69000044600F0B5FA034B204623600023E36420
:10B6A00002B010BDC82C060830B590F8533087B0F2
:10B6B00043B390F85020002390F85110062590F8DD
:10B6C00052401201090180F853302401C06C8DF8FA
:10B6D0001320120ACDE90233CDF80F308DF80B405C
:10B6E000240A8DF80F10090A8DF80C408DF81010FF
:10B6F00002A98DF808508DF814200268009314698F
:10B700000D22A04707B030BDFFF7CEBF044B10B5E8
:10B71000044640F84C3BFEF7C5FC204610BD00BF78
:10B72000C82C060810B50446FFF7F0FF2046F7F7CF
:10B7300047FF204610BD0000374B04221B68F0B5C0
:10B74000002489B0D96A064606AF0B683846CDE9B1
:10B750000142324A009201221D684023A847069BFD
:10B76000F06C0694F36410B103685B689847384640
:10B77000FEF798FCF06C00284CD0036800255B6A4B
:10B78000984703689B689847F06C052103689B6C99
:10B79000984701230DF113022946F06C8DF81350E0
:10B7A00004F0ACFE0446F06C44B903685B6A984749
:10B7B0000368DB689847204609B0F0BD9DF8133058
:10B7C00002228DF8145005A923F0300343F0200322
:10B7D0008DF81530036800951C692B46A047044678
:10B7E000F06C0368002CE1D001219B6C9847F06C51
:10B7F00003685B6A98470368DB689847F06C44F617
:10B80000206103689D6A064B0696079397E80C0033
:10B81000A847D0E70446CEE7282A0030801A060061
:10B8200009B7040870B5B0F84A509DF81040AC4212
:10B8300009DAC66C04EB44043355351901236970E9
:10B84000AA7080F8503070BDF0B50025B0F84A609D
:10B85000ACB2A64208D9C76C04EB440401353E19CA
:10B860003B557170B270F1E7012380F850301846F3
:10B87000F0BD000070470000F8B5064681240025A1
:10B8800027B23846FEF740FE20B13846FEF726FEC6
:10B89000284385B20134A4B2842CF1D185B10023B0
:10B8A000084F25FA03F25C1C12F0010F05D07368F3
:10B8B000E1B238469A7B00F0DFFE102C2346F0D12F
:10B8C0002846F8BDBD43003010B50446F7F778FEB2
:10B8D000204610BD3323FF2213B5044600930021F8
:10B8E0007F2300F029FB024B2046236002B010BDED
:10B8F000602D06083323FF2213B5002100937F2318
:10B90000044600F07DF9034B204623600023636565
:10B9100002B010BD282D06082DE9F04F0446B0F8FE
:10B920004A50406D19278FB003687D435B6A05F16B
:10B93000320698477522014605A8F7F78BFF39357F
:10B94000E36C06F00706ED081A88C6F13A069B7804
:10B95000F6B2ADF810208DF81230EB0000250393FD
:10B960002946A8460022A5EB060A4FF0180E944679
:10B97000AB189E425DD80AEB0203B3FBF7F007FB5E
:10B980001039B9F1000F56D01B1AB3FBFEF0404539
:10B990000DD0D4F84C9000EB400809EB080B39F8B7
:10B9A00008809BF80290ADF810808DF812900DF190
:10B9B0003809B3FBFEF80EFB183803F0070309EB58
:10B9C000D808C3F1080318F8288C48FA03F3804616
:10B9D00003F00103C2F1070001328340082A43EA61
:10B9E0000C0C5FFA8CFCC3D14A1C0EABD2B21944CA
:10B9F0001F2A01F820CC20D9606D00210368009136
:10BA0000D3F810900B4606A9C84700210835039BC0
:10BA1000AB42A7D139B1606D00230268009314696D
:10BA20000A4606A9A04705A8F7F71AFF0FB0BDE818
:10BA3000F08F0023CEE70123CCE71146E6E70000B4
:10BA4000002280F85020FFF767BF0000FFF7F8BF23
:10BA500010B50446006810B103685B68984720463B
:10BA600010BD0000044B10B5044640F8543BFFF7EE
:10BA7000EFFF204610BD00BF282D060810B5044674
:10BA8000FFF7F0FF2046F7F79BFD204610BD0000B2
:10BA90007FB54368044602AD987B0130A4F84A00A4
:10BAA00000EB4000F7F790FDB4F84A200021E06475
:10BAB00002EB420210F080FA1A4B1B4A28461B6820
:10BAC000196B0B681B689847029B606D00226365C9
:10BAD000029210B103685B6898472846FFF7B8FFE9
:10BAE000606DE0B103685B6A98475122014601A886
:10BAF000F7F7B0FE606D42F2107103689E6A0B4B5F
:10BB00000294039395E80C000125B047084884F897
:10BB10005050F7F7F5F801A8F7F7A2FE284604B051
:10BB200070BD00BF282A0030F82C06084DBA040862
:10BB3000012D06082DE9F0411D46037A04460F4603
:10BB40008B42164605D1437A934202D1837AAB42A7
:10BB50000BD02368324639462046D3F828802B463E
:10BB6000C04710B127726672A572BDE8F08100006F
:10BB700030B4456895F90150012D04D00468E46A99
:10BB8000A44630BC604730BC7047000010B59DF83B
:10BB900008400174C4744274837410BD70B5436866
:10BBA00088B004460D4693F90130012B17D1CE78A9
:10BBB0001D22002168461D2E28BF1D2610F0FCF90D
:10BBC00005F10C016846324610F0E8F904F094FBE8
:10BBD0009DF804306061032B03D0042B0DD008B016
:10BBE00070BD0023E3749DF8053023749DF8063082
:10BBF00063749DF80730A374F1E79DF80830F1E70E
:10BC000030B543739DF80C30027346F6B652837319
:10BC1000124B134D836103F17643C17203F5AB43BD
:10BC200010490560C361104B104D0362A3F1DB5353
:10BC3000A3F558234362A3F1DB53A3F55823836292
:10BC40000B4BC0E90B230B4BC0E90D1342F292439F
:10BC5000C0E90F5341F24923436430BD0CC3300C9B
:10BC60009C2D060849922409B6EDFF3F8220080268
:10BC7000922449123660030038B543680446057BB8
:10BC800093F90030012B10D0022B10D003B9C57AE4
:10BC9000084B1B68586C03689B6B984718B1A37BD3
:10BCA0009D4228BF1D46284638BD857BF0E7457B71
:10BCB000EEE700BF282A0030244B1A780AB18069C9
:10BCC00070471A7A2AB95A7A1AB99A7C0AB9DA7E6E
:10BCD0000AB1C0697047997ADA7C91B9197B81B948
:10BCE000D97A71B9D97B002926D1597D002926D16D
:10BCF00042B91A7972B15B78022B8CBF006B406B32
:10BD000070470AB1006A7047DA7BD2B1406A704767
:10BD1000C06A70479A790AB9806B70475A78032ACB
:10BD200003D9DB7933B1C06B704703D1DB790BB139
:10BD3000006C7047406C7047002AE7D0E2E7002AA9
:10BD4000E0D15B7D002BE3D0806A704781430030F7
:10BD500010B5104C2378C3B92379C3B90E4B1B68B7
:10BD6000586D03681B6A98470128A37906D00B48D1
:10BD700046F6B652002B18BF104610BD42F2924054
:10BD8000074A002B08BF1046F7E70648F5E744F6D8
:10BD90002410F2E781430030282A0030866118061B
:10BDA0008220080254A8500170B5C37C044643B9F0
:10BDB0000368427CDD6A017C837CAC46BDE8704050
:10BDC00060474FF47A75B5FBF3F504F095FA6369B3
:10BDD000C01AB0FBF5F305FB13002368B0EB550F59
:10BDE000DD6A204691BF0023A37C627C217C9CBF3E
:10BDF0001A461946E1E7000070B54368044693F916
:10BE00000130032B48D8DFE803F006020A44BDE8FE
:10BE10007040FFF7C9BFFFF74FFF054606E01F4B15
:10BE20001F4D1B791F48002B18BF05462046FFF702
:10BE300023FF064604F060FA64220A2394F84810AF
:10BE4000B0FBF2F2B2FBF3F003FB1022D2B291424C
:10BE500007D04A1CB2FBF3F103FB1122D2B284F8E3
:10BE6000482002EB4202204625FA02F2D3B25107E3
:10BE700054BFE17A31469A0754BFE27A3246DB0773
:10BE8000236858BFE67A5D6A3346AC46BDE8704029
:10BE90006047FFF75DFFC0E70025C7E7814300303B
:10BEA00092244912244992240020704710B5036857
:10BEB00004461B6B9847A4F84C00012010BD0000FD
:10BEC0007047000010B50446F7F77AFB204610BD16
:10BED0002DE9F7439846B0F84C3005460E46174614
:10BEE00023B30024DFF84C90B5F84C30E340013424
:10BEF00013F0010F08D033464FF0FF32E1B248464D
:10BF0000CDE9007800F0DAFB102CEDD10023094ECA
:10BF1000B5F84C205C1CDA4012F0010F03D0E1B2FE
:10BF2000304600F0E5FB102C2346F1D1012003B090
:10BF3000BDE8F083BD43003037B59DF81850044686
:10BF40000095FFF75DFE2046034B40F8503B01F0A3
:10BF500099FC204603B030BDD42D06087047000080
:10BF600073B504460D46A72200F1140104F12C0616
:10BF700001A8F7F753FC304605F0E8FE04F1500342
:10BF800029466322184610F08BFB002201463046FA
:10BF900084F8B32006F03CF901A8F7F761FC02B081
:10BFA00070BD00002DE9F041CE78BCB004460D46CE
:10BFB000E82E4FF0E8024FF0000102A828BFE82663
:10BFC00004F12C070FF0F8FF05F10C01324602A82E
:10BFD0000FF0E4FF04F1500604F114014FF4E7728E
:10BFE00001A84FF00008F7F719FC384605F0AEFE3F
:10BFF0001E220DF10A01304610F052FB304684F843
:10C00000B380F4F723FF0546C8210AA8EDB210F06B
:10C010005BFB0AA9C5F16302C0B2824228BF024697
:10C02000701910F03DFB3146384684F8B38006F0B5
:10C03000EFF801A8F7F714FC3CB0BDE8F081000070
:10C0400010B50446F7F7BCFA204610BD13B5426898
:10C05000034692F90200F8B1104A197A1079009358
:10C0600060F300011972C9B2D27A21F00A015200BC
:10C0700042F0080202F00A020A431A72FF22DA7240
:10C08000074A084B1268019302AB106D0268546AAC
:10C0900013E90600A047012002B010BD8143003023
:10C0A000282A003001C1040870B504460D4604F08A
:10C0B00023F9094B6AB2206103EBC50120462273C4
:10C0C0000979C90753F8351048BFE2722268BDE804
:10C0D00070409269104700BF8C30060813B50446C3
:10C0E00000F11401A12201A8F7F798FB04F12C003C
:10C0F00006F07CF801A8F7F7B3FB02B010BD000012
:10C10000FFF7ECBF90F90B2090F90C309A4210B574
:10C11000044605D1036804499B699847FF232373AC
:10C12000FF23E37210BD00BFF2F8050810B5044606
:10C1300004F0E2F894F90B104B1C0ED094F90C307B
:10C140008B420AD02369C01AB0F5FA6F05D9204690
:10C15000C9B2BDE81040FFF7A7BF10BD70B5436876
:10C16000044693F9023083B1394DFFF7DFFF637A5C
:10C170006A7E5AB1180703D41B212046FFF794FFAB
:10C180006A7E637A62F3C303637270BDAA7C03F0B4
:10C190000103934208D0BAB10E212046FFF784FF75
:10C1A00004212046FFF780FFAA7C637A294E62F3C0
:10C1B00000036372737813F0120F0DD00221204632
:10C1C000BDE87040FFF770BF94F90B300E2BEBD138
:10C1D0002046FFF797FFE7E733681F49194001D072
:10C1E0000721ECE71D4A1342E9D1B3781907E5D4DA
:10C1F000637AEA7EC3F30013934208D002B30E21A0
:10C200002046FFF751FF04212046FFF74DFFEA7E4D
:10C21000637A62F304136372AB7C002BB5D1EB7EBF
:10C22000002BB2D12B7913B3337813F0900F17D1C1
:10C2300033789A061BD501212046FFF735FF16E01B
:10C2400094F90B300E2BE2D12046FFF75BFFDEE7BF
:10C2500081430030A043003000041000000820009B
:10C2600006212046FFF720FF2B79002BE0D17378C1
:10C27000DB0703D50A212046FFF716FF337898071E
:10C2800007D52B79002B00F0EA8003212046FFF729
:10C290000BFF3378590705D5297901B101212046D3
:10C2A000FFF702FF33781A0703D508212046FFF76E
:10C2B000FBFE3378DB0703D500212046FFF7F4FEB1
:10C2C000237AAA7AC3F3001191420AD062F30413CD
:10C2D0002979D806237240F1C48011B92046FFF7AE
:10C2E000E3FE237A2A7BC3F3401191420AD062F322
:10C2F000451329799A06237240F1B88011B9204676
:10C30000FFF7D2FE237AAA79C3F3C00191420DD080
:10C3100062F3C30323721B0740F1AD80072120465F
:10C32000FFF7C2FEA37A43F00103A372237A2A79AE
:10C3300003F00101914209D062F30003D90723728F
:10C3400040F1A28009212046FFF7AEFE237AEA7A67
:10C35000C3F34001914208D062F3410323729B076B
:10C3600003D50D212046FFF79FFE237AAA7BC3F356
:10C370008001914208D062F382035807237203D5EB
:10C3800008212046FFF790FEEA7D237AB2EBD31F07
:10C3900009D062F3C7131906237240F181800C2182
:10C3A0002046FFF781FE637A2A7EC3F34001914263
:10C3B00008D062F341039A07637275D50F212046B6
:10C3C000FFF772FE637AEA7CC3F38001914208D0E2
:10C3D00062F3820363725B076AD51A212046FFF776
:10C3E00063FE7378980607D517212046FFF75CFE99
:10C3F00073786FF345137370316811F4E03F09D01F
:10C40000C1F3823120460F31FFF74EFE33686FF3E0
:10C4100090333360B378990707D518212046FFF78A
:10C4200043FEB3786FF34103B370B3785A0707D56F
:10C4300019212046FFF738FEB3786FF38203B370FB
:10C44000237A6A7BC3F3801191423FF49EAE62F37C
:10C45000861323725B067FF598AE1F21AFE602219B
:10C4600014E709B1052139E7042137E709B10521AE
:10C4700045E7042143E7A37AD8077FF557AF1C218E
:10C480002046FFF711FE51E702212046FFF70CFE80
:10C49000637A5A073FF55AAF2046FFF733FE55E758
:10C4A0002046FFF72FFE7EE72046FFF72BFE89E7A9
:10C4B0002046FFF727FE94E780F85330012380F8E9
:10C4C000511080F8522080F8503018467047000014
:10C4D000112337B50D460093FF2280230021044627
:10C4E000FFF78EFB044B204684F854502360002352
:10C4F000E36403B030BD00BFC03106081FB590F83B
:10C500005030DBB10122002303A98DF80C2090F8F4
:10C51000532080F8503012098DF80D2090F85220E9
:10C5200012098DF80E2090F85120C06C12098DF878
:10C530000F200268009314690422A04704B010BDC4
:10C54000FFF7DCBF044B10B5044640F84C3BFDF749
:10C55000A9FD204610BD00BFC031060810B5044635
:10C56000FFF7F0FF2046F7F72BF8204610BD00003C
:10C57000324B04221B68F0B5002589B0D96A044605
:10C5800006AE0B68CDE901522D4A00921F68552373
:10C5900090F854203046B847069BE06C0695E3645B
:10C5A00010B103685B6898473046FDF77BFDE06C8F
:10C5B000002840D003685B6A98473622014604A8E9
:10C5C000F7F748F9E06C0A2103689B6C9847002351
:10C5D00003220421E06C03F06DFF30B9002504A8AC
:10C5E000F7F73EF9284609B0F0BDE37A0127E06C81
:10C5F00005A98DF815308DF816308DF81730002309
:10C600008DF814700268009315690422A847054646
:10C61000E06C394603689B6C9847002DDED0E06CD7
:10C6200044F6206103689F6A064B0694079396E8D8
:10C630000C00B847D3E70546D4E700BF282A0030EE
:10C64000801A060041C5040813B50139C8B20F2885
:10C650000ED8802A0CD8074B002489B21B68D86CEE
:10C6600003680094D3F8B0400923A04702B010BD7E
:10C670000020FBE7282A0030F7B54C1E1546E3B230
:10C680000F2B02D9002003B0F0BD7E2AFAD88420F7
:10C69000FDF73AFF0028F5D08420FDF71FFF064B79
:10C6A0002A46A1B21B68DE6C336800903046D3F88E
:10C6B000B0700A23B847E6E7282A00300139C8B22B
:10C6C0000F2870B49DF80C509DF810600BD80748E7
:10C6D00089B20068C06C0468CDE90356D4F8B44050
:10C6E000A44670BC604770BC704700BF282A003069
:10C6F0000139CBB20F2B07D8044B89B21B68D86C19
:10C700000368D3F8B8301847704700BF282A0030B4
:10C71000202383F3118862B670470000002383F35F
:10C72000118862B67047000010B41346026814689E
:10C730000022A4465DF8044B6047000000F540501D
:10C7400090F859077047000000F5405090F85207E4
:10C750007047000000F5405090F9580770470000FE
:10C760004E20704700F5405208B5FFF7D1FFD2F8D0
:10C770009837D2F894071844D2F890371844D2F872
:10C7800078371844D2F888371844D2F884371844D8
:10C79000FFF7C4FF08BD000010B50446FFF7B8FF5F
:10C7A000084604F54054C4F854170B6807491B6841
:10C7B0009847D4F8540794F858270121036891400A
:10C7C0005B689847FFF7AAFF10BD00BFCC4300305D
:10C7D0002DE9F14F0C4600F540511F46054691F8F2
:10C7E00052379046BDF82890ABB1D1F87437013379
:10C7F000C1F8743723689A0008D494F84430082BA1
:10C800000CD994F845200AB10F2B07D9D1F8783705
:10C810000133C1F878374FF0FF300FE0FFF778FFB2
:10C82000EB6AD3F8C42012F4001A0AD0D1F87C378E
:10C8300000200133C1F87C37FFF770FF01B0BDE87D
:10C84000F08F22684FF0480BD3F8C460002A6B6A5F
:10C85000C6F30446B4BF42F0804292041BFB063B81
:10C86000CBF8002023685B004FEA066344BF42F028
:10C870000052CBF8002094F8442043EA0243CBF85E
:10C88000043094F8452032B343F44013CBF804301D
:10C89000D1F8A4370133C1F8A437582303FB06535A
:10C8A00003F5325393F8242042F0200283F8242029
:10C8B00094F84400F6F7F6FE033080105FFA8AF32E
:10C8C0000AF1010A834212DA04EB83020BEB8303C1
:10C8D00052689A60F2E7582303FB065303F532537C
:10C8E00093F8241062F3451183F82410E0E75820F0
:10C8F0000123EA6A214600FB065AB3400AF531508B
:10C90000C2F8D0300AF5315346221830C3E9048703
:10C910000FF044FB42F6A043214628464AF8036044
:10C920000AF5005A09F003039AF8A42C43F0100307
:10C9300022F01F02134342468AF8A43CFFF7EEFEA2
:10C940003B46CDF8289001B0BDE8F04FF6F760BE49
:10C950000246F2EE046A0846334900B59FB0FFF77D
:10C96000D7FE02F54053B3F85A2707EE902AD3F8C2
:10C97000A8271C92F8EEE77AD3F8A4271B9287EE3B
:10C98000A67AD3F8AC271A92D3F8A0271992D3F835
:10C990009C271892D3F898271792D3F894271692C9
:10C9A000D3F89027B7EEC77A1592D3F88C27149254
:10C9B000D3F888271392D3F884271292D3F88027CC
:10C9C0001192D3F87C271092D3F878270F92D3F8DE
:10C9D00074278DED0C7B0E9293F868270A9293F8DA
:10C9E0006727099293F866270892B3F8642707929D
:10C9F000D3F870278DED047B069293F8602703929D
:10CA000093F85F27029293F85E270192B3F85C27B0
:10CA100000925022D3F86C3703F0B2FC1FB05DF8DF
:10CA200004EBFFF77BBE00BFF03106082DE9F047AD
:10CA300000F54056044696F85257002D40F001810B
:10CA4000037C032B40F092802B4628462F465FFA4A
:10CA500083FC944510DA01EBCC0E51F83CC0BCF1DC
:10CA6000000F04DBDEF804C0BCF1000F02DB01376D
:10CA70000133ECE70130FBE7FFF74AFEE36AF0B968
:10CA8000D3F8800040F00200C3F880004E23E06A33
:10CA9000002F6ED1D0F8803043F00103C0F8803011
:10CAA000694B6A4A1B6803F1805303F52C539B00C2
:10CAB0009342A36240F2AF80654803F0EBFB4D2840
:10CAC00042D8DFF884814FEA004EDFF88891D8F829
:10CAD00000C04EEA8C0EC3F884E00CF1805303F5DD
:10CAE0002C539B00636100EB0C03D4F82CC0C8F8F6
:10CAF0000030C0F14E03DCF8800040F03000CCF88C
:10CB000080004FF0000CD4F81480E6465FFA8CF0F9
:10CB10008242BCDD01EBC00A51F83000002810DB76
:10CB2000DAF804A0BAF1000F0BDA09EA00400AF0C3
:10CB30007F0A40EA0A0040F0084048F82E000EF153
:10CB4000010E0CF1010CE1E79A6922F001029A61F1
:10CB500003F0D2FB0646E36A9B69D90704D503F0CC
:10CB6000CBFB831BFA2BF6D9FFF7D8FD2846BDE88F
:10CB7000F087B7EB530F3DD2DFF8CCE04FEA074C1C
:10CB8000DEF800304CEA830CC0F888C003F1805016
:10CB900003EB4703002700F52C50CEF80030BC46CD
:10CBA0008000A061E06AD0F8803043F00C03C0F848
:10CBB0008030D4F818E0FBB29A427FF771AF51F899
:10CBC000330001EBC3080028D8F8043001DB002B48
:10CBD0000EDB20F0604023F0604340F0005043F053
:10CBE00000434EF83C000EEBCC000CF1010C43600E
:10CBF0000137E0E7836923F00103836103F07CFBE5
:10CC00000646E36A9B69DA07AED503F075FB831B22
:10CC1000FA2BF6D9A8E7E26A936923F0010393613E
:10CC200003F06AFB0746E36A9B69DB0705D503F05F
:10CC300063FBC31BFA2BF6D996E7012586F85257FA
:10CC400092E7002592E700BFC8430030FCB50040E2
:10CC5000083406080000FF0713B500F500540191E1
:10CC6000D4F8440C03F0E0FD57280BD95822019961
:10CC7000D4F8440C03F04EFEA0F15803584258413A
:10CC800002B010BD0020FBE700F5005008B5FFF72B
:10CC90003FFDD0F8440C03F09BFDBDE80840FFF7D2
:10CCA0003DBD00000021402210B504460160A0F8FF
:10CCB000441004300FF080F9204610BD00220023FC
:10CCC00010B5C0E90023002304460C3020F8043CD2
:10CCD000FFF7E8FF204610BD2DE9F041044696B06D
:10CCE0001F460D4604F5005868461646FFF710FD2E
:10CCF000FFF7E4FFD8F8440C03F07CFD572823D954
:10CD000058226946D8F8440C03F088FE58281BD1F5
:10CD100004F5405393F85237B3B103A9462228468D
:10CD20000FF03CF929462046DDE90023C6E900233F
